 cuda_support

 Timestamp is 5c7622d4 (Wed Feb 27 12:40:36 2019)

 Preferred load address is 10000000

 Start         Length     Name                   Class
 0001:00000000 00000a1bH .text$di                CODE
 0001:00000a20 0000530eH .text$mn                CODE
 0001:00005d30 00000b83H .text$x                 CODE
 0001:000068c0 000001ebH .text$yd                CODE
 0002:00000000 0000041cH .idata$5                DATA
 0002:0000041c 00000004H .CRT$XCA                DATA
 0002:00000420 00000068H .CRT$XCU                DATA
 0002:00000488 00000004H .CRT$XCZ                DATA
 0002:0000048c 00000004H .CRT$XIA                DATA
 0002:00000490 00000004H .CRT$XIAA               DATA
 0002:00000494 00000004H .CRT$XIC                DATA
 0002:00000498 00000004H .CRT$XIZ                DATA
 0002:000004a0 00000ca8H .rdata                  DATA
 0002:00001148 00000074H .rdata$debug            DATA
 0002:000011bc 000007fcH .rdata$r                DATA
 0002:000019c0 000000c4H .rdata$sxdata           DATA
 0002:00001a84 00000004H .rtc$IAA                DATA
 0002:00001a88 00000004H .rtc$IZZ                DATA
 0002:00001a8c 00000004H .rtc$TAA                DATA
 0002:00001a90 00000004H .rtc$TZZ                DATA
 0002:00001a98 00000e4cH .xdata$x                DATA
 0002:000028f0 00000055H .edata                  DATA
 0002:00002948 000000a0H .idata$2                DATA
 0002:000029e8 00000014H .idata$3                DATA
 0002:000029fc 0000041cH .idata$4                DATA
 0002:00002e18 000029beH .idata$6                DATA
 0003:00000000 000000a4H .data                   DATA
 0003:000000a4 0000039cH .data$r                 DATA
 0003:00000440 000003ecH .bss                    DATA
 0004:00000000 00000058H .rsrc$01                DATA
 0004:00000060 00000180H .rsrc$02                DATA

  Address         Publics by Value              Rva+Base       Lib:Object

 0000:00000000       ___guard_fids_count        00000000     <absolute>
 0000:00000000       ___guard_fids_table        00000000     <absolute>
 0000:00000000       ___guard_flags             00000000     <absolute>
 0000:00000000       __except_list              00000000     <absolute>
 0000:00000031       ___safe_se_handler_count   00000031     <absolute>
 0000:00009876       __fltused                  00009876     <absolute>
 0000:00009876       __ldused                   00009876     <absolute>
 0000:00000000       ___ImageBase               10000000     <linker-defined>
 0001:00000a20       ??$_Allocate@D@std@@YAPADIPAD@Z 10001a20 f i CudaSupportPlugin.obj
 0001:00000a50       ??$addressof@D@std@@YAPADAAD@Z 10001a50 f i CudaSupportPlugin.obj
 0001:00000a60       ??$atomic@H@?$QAtomicOpsBySize@$03@@CAPAJPAH@Z 10001a60 f i CudaSupportPlugin.obj
 0001:00000a70       ??$construct@PADAAPAD@?$_Wrap_alloc@V?$allocator@D@std@@@std@@QAEXPAPADAAPAD@Z 10001a70 f i CudaSupportPlugin.obj
 0001:00000a90       ??$construct@PADAAPAD@?$allocator@D@std@@QAEXPAPADAAPAD@Z 10001a90 f i CudaSupportPlugin.obj
 0001:00000ab0       ??$construct@PADAAPAD@?$allocator_traits@V?$allocator@D@std@@@std@@SAXAAV?$allocator@D@1@PAPADAAPAD@Z 10001ab0 f i CudaSupportPlugin.obj
 0001:00000ad0       ??$deref@H@?$QAtomicOpsBySize@$03@@SA_NAAH@Z 10001ad0 f i CudaSupportPlugin.obj
 0001:00000af0       ??$destroy@PAD@?$_Wrap_alloc@V?$allocator@D@std@@@std@@QAEXPAPAD@Z 10001af0 f i CudaSupportPlugin.obj
 0001:00000b00       ??$destroy@PAD@?$allocator@D@std@@QAEXPAPAD@Z 10001b00 f i CudaSupportPlugin.obj
 0001:00000b10       ??$destroy@PAD@?$allocator_traits@V?$allocator@D@std@@@std@@SAXAAV?$allocator@D@1@PAPAD@Z 10001b10 f i CudaSupportPlugin.obj
 0001:00000b20       ??$forward@AAPAD@std@@YAAAPADAAPAD@Z 10001b20 f i CudaSupportPlugin.obj
 0001:00000b30       ??$load@H@?$QGenericAtomicOps@U?$QAtomicOpsBySize@$03@@@@SAHABH@Z 10001b30 f i CudaSupportPlugin.obj
 0001:00000b40       ??$ref@H@?$QAtomicOpsBySize@$03@@SA_NAAH@Z 10001b40 f i CudaSupportPlugin.obj
 0001:00000b60       ??0?$QForeachContainer@V?$QList@PAVCudaGpuModel@U2@@@@@@QAE@ABV?$QList@PAVCudaGpuModel@U2@@@@@Z 10001b60 f i CudaSupportPlugin.obj
 0001:00000ba0       ??0?$QList@PAVCudaGpuModel@U2@@@@QAE@ABV0@@Z 10001ba0 f i CudaSupportPlugin.obj
 0001:00000c60       ??0?$QList@PAVCudaGpuModel@U2@@@@QAE@XZ 10001c60 f i CudaSupportPlugin.obj
 0001:00000c70       ??0?$_String_alloc@$0A@U?$_String_base_types@DV?$allocator@D@std@@@std@@@std@@QAE@ABV?$allocator@D@1@@Z 10001c70 f i CudaSupportPlugin.obj
 0001:00000c90       ??0?$_String_val@U?$_Simple_types@D@std@@@std@@QAE@XZ 10001c90 f i CudaSupportPlugin.obj
 0001:00000cb0       ??0?$_Wrap_alloc@V?$allocator@D@std@@@std@@QAE@XZ 10001cb0 f i CudaSupportPlugin.obj
 0001:00000cc0       ??0?$allocator@D@std@@QAE@XZ 10001cc0 f i CudaSupportPlugin.obj
 0001:00000cd0       ??0?$basic_string@DU?$char_traits@D@std@@V?$allocator@D@2@@std@@QAE@PBD@Z 10001cd0 f i CudaSupportPlugin.obj
 0001:00000d30       ??0CudaSupportPlugin@U2@@QAE@XZ 10001d30 f   CudaSupportPlugin.obj
 0001:00000fb0       ??0QLatin1Char@@QAE@D@Z    10001fb0 f i CudaSupportPlugin.obj
 0001:00000fc0       ??0_Generic_error_category@std@@QAE@XZ 10001fc0 f i CudaSupportPlugin.obj
 0001:00000fd0       ??0_Ignore@std@@QAE@XZ     10001fd0 f i CudaSupportPlugin.obj
 0001:00000fe0       ??0_Iostream_error_category@std@@QAE@XZ 10001fe0 f i CudaSupportPlugin.obj
 0001:00000ff0       ??0_System_error_category@std@@QAE@XZ 10001ff0 f i CudaSupportPlugin.obj
 0001:00001000       ??0const_iterator@?$QList@PAVCudaGpuModel@U2@@@@QAE@PAUNode@1@@Z 10002000 f i CudaSupportPlugin.obj
 0001:00001010       ??0error_category@std@@QAE@XZ 10002010 f i CudaSupportPlugin.obj
 0001:00001020       ??0error_condition@std@@QAE@HABVerror_category@1@@Z 10002020 f i CudaSupportPlugin.obj
 0001:00001040       ??1?$QForeachContainer@V?$QList@PAVCudaGpuModel@U2@@@@@@QAE@XZ 10002040 f i CudaSupportPlugin.obj
 0001:00001070       ??1?$QList@PAVCudaGpuModel@U2@@@@QAE@XZ 10002070 f i CudaSupportPlugin.obj
 0001:000010a0       ??1?$basic_string@DU?$char_traits@D@std@@V?$allocator@D@2@@std@@QAE@XZ 100020a0 f i CudaSupportPlugin.obj
 0001:000010d0       ??1CudaSupportPlugin@U2@@UAE@XZ 100020d0 f i CudaSupportPlugin.obj
 0001:00001150       ??1_Generic_error_category@std@@UAE@XZ 10002150 f i CudaSupportPlugin.obj
 0001:00001160       ??1_Iostream_error_category@std@@UAE@XZ 10002160 f i CudaSupportPlugin.obj
 0001:00001170       ??1_System_error_category@std@@UAE@XZ 10002170 f i CudaSupportPlugin.obj
 0001:00001180       ??1error_category@std@@UAE@XZ 10002180 f i CudaSupportPlugin.obj
 0001:00001190       ??2@YAPAXIPAX@Z            10002190 f i CudaSupportPlugin.obj
 0001:000011a0       ??3@YAXPAX0@Z              100021a0 f i CudaSupportPlugin.obj
 0001:000011b0       ??8error_category@std@@QBE_NABV01@@Z 100021b0 f i CudaSupportPlugin.obj
 0001:000011c0       ??8error_condition@std@@QBE_NABV01@@Z 100021c0 f i CudaSupportPlugin.obj
 0001:000011e0       ??9const_iterator@?$QList@PAVCudaGpuModel@U2@@@@QBE_NABV01@@Z 100021e0 f i CudaSupportPlugin.obj
 0001:00001200       ??Dconst_iterator@?$QList@PAVCudaGpuModel@U2@@@@QBEABQAVCudaGpuModel@U2@@XZ 10002200 f i CudaSupportPlugin.obj
 0001:00001210       ??Econst_iterator@?$QList@PAVCudaGpuModel@U2@@@@QAEAAV01@XZ 10002210 f i CudaSupportPlugin.obj
 0001:00001220       ??H@YA?BVQString@@ABV0@0@Z 10002220 f i CudaSupportPlugin.obj
 0001:00001290       ??H@YA?BVQString@@ABV0@PBD@Z 10002290 f i CudaSupportPlugin.obj
 0001:00001330       ??H@YA?BVQString@@PBDABV0@@Z 10002330 f i CudaSupportPlugin.obj
 0001:000013a0       ??_EAppResourceSemaphore@U2@@UAEPAXI@Z 100023a0 f i CudaSupportPlugin.obj
 0001:000013a0       ??_GAppResourceSemaphore@U2@@UAEPAXI@Z 100023a0 f i CudaSupportPlugin.obj
 0001:000013d0       ??_GCudaSupportPlugin@U2@@UAEPAXI@Z 100023d0 f i CudaSupportPlugin.obj
 0001:000013d0       ??_ECudaSupportPlugin@U2@@UAEPAXI@Z 100023d0 f i CudaSupportPlugin.obj
 0001:00001460       ??_E_Generic_error_category@std@@UAEPAXI@Z 10002460 f i CudaSupportPlugin.obj
 0001:00001460       ??_G_Generic_error_category@std@@UAEPAXI@Z 10002460 f i CudaSupportPlugin.obj
 0001:00001490       ??_G_Iostream_error_category@std@@UAEPAXI@Z 10002490 f i CudaSupportPlugin.obj
 0001:00001490       ??_E_Iostream_error_category@std@@UAEPAXI@Z 10002490 f i CudaSupportPlugin.obj
 0001:000014c0       ??_E_System_error_category@std@@UAEPAXI@Z 100024c0 f i CudaSupportPlugin.obj
 0001:000014c0       ??_G_System_error_category@std@@UAEPAXI@Z 100024c0 f i CudaSupportPlugin.obj
 0001:000014f0       ??_Gerror_category@std@@UAEPAXI@Z 100024f0 f i CudaSupportPlugin.obj
 0001:000014f0       ??_Eerror_category@std@@UAEPAXI@Z 100024f0 f i CudaSupportPlugin.obj
 0001:00001520       ?_Copy@?$basic_string@DU?$char_traits@D@std@@V?$allocator@D@2@@std@@QAEXII@Z 10002520 f i CudaSupportPlugin.obj
 0001:00001670       ?_Eos@?$basic_string@DU?$char_traits@D@std@@V?$allocator@D@2@@std@@QAEXI@Z 10002670 f i CudaSupportPlugin.obj
 0001:000016a0       ?_Getal@?$_String_alloc@$0A@U?$_String_base_types@DV?$allocator@D@std@@@std@@@std@@QBE?AU?$_Wrap_alloc@V?$allocator@D@std@@@2@XZ 100026a0 f i CudaSupportPlugin.obj
 0001:000016b0       ?_Grow@?$basic_string@DU?$char_traits@D@std@@V?$allocator@D@2@@std@@QAE_NI_N@Z 100026b0 f i CudaSupportPlugin.obj
 0001:00001760       ?_Inside@?$basic_string@DU?$char_traits@D@std@@V?$allocator@D@2@@std@@QAE_NPBD@Z 10002760 f i CudaSupportPlugin.obj
 0001:000017a0       ?_Myptr@?$_String_val@U?$_Simple_types@D@std@@@std@@QAEPADXZ 100027a0 f i CudaSupportPlugin.obj
 0001:000017b0       ?_Myptr@?$_String_val@U?$_Simple_types@D@std@@@std@@QBEPBDXZ 100027b0 f i CudaSupportPlugin.obj
 0001:000017c0       ?_Tidy@?$basic_string@DU?$char_traits@D@std@@V?$allocator@D@2@@std@@QAEX_NI@Z 100027c0 f i CudaSupportPlugin.obj
 0001:00001810       ?_Xlen@?$basic_string@DU?$char_traits@D@std@@V?$allocator@D@2@@std@@QBEXXZ 10002810 f i CudaSupportPlugin.obj
 0001:00001820       ?_Xran@?$basic_string@DU?$char_traits@D@std@@V?$allocator@D@2@@std@@QBEXXZ 10002820 f i CudaSupportPlugin.obj
 0001:00001830       ?allocate@?$_Wrap_alloc@V?$allocator@D@std@@@std@@QAEPADI@Z 10002830 f i CudaSupportPlugin.obj
 0001:00001860       ?allocate@?$allocator@D@std@@QAEPADI@Z 10002860 f i CudaSupportPlugin.obj
 0001:00001890       ?append@?$QList@PAVCudaGpuModel@U2@@@@QAEXABQAVCudaGpuModel@U2@@@Z 10002890 f i CudaSupportPlugin.obj
 0001:00001920       ?assign@?$basic_string@DU?$char_traits@D@std@@V?$allocator@D@2@@std@@QAEAAV12@ABV12@II@Z 10002920 f i CudaSupportPlugin.obj
 0001:00001a40       ?assign@?$basic_string@DU?$char_traits@D@std@@V?$allocator@D@2@@std@@QAEAAV12@PBD@Z 10002a40 f i CudaSupportPlugin.obj
 0001:00001a80       ?assign@?$basic_string@DU?$char_traits@D@std@@V?$allocator@D@2@@std@@QAEAAV12@PBDI@Z 10002a80 f i CudaSupportPlugin.obj
 0001:00001b80       ?assign@?$char_traits@D@std@@SAXAADABD@Z 10002b80 f i CudaSupportPlugin.obj
 0001:00001b90       ?begin@?$QList@PAVCudaGpuModel@U2@@@@QBE?AVconst_iterator@1@XZ 10002b90 f i CudaSupportPlugin.obj
 0001:00001bb0       ?category@error_code@std@@QBEABVerror_category@2@XZ 10002bb0 f i CudaSupportPlugin.obj
 0001:00001bc0       ?category@error_condition@std@@QBEABVerror_category@2@XZ 10002bc0 f i CudaSupportPlugin.obj
 0001:00001bd0       ?copy@?$char_traits@D@std@@SAPADPADPBDI@Z 10002bd0 f i CudaSupportPlugin.obj
 0001:00001bf0       ?dealloc@?$QList@PAVCudaGpuModel@U2@@@@AAEXPAUData@QListData@@@Z 10002bf0 f i CudaSupportPlugin.obj
 0001:00001c10       ?deallocate@?$_Wrap_alloc@V?$allocator@D@std@@@std@@QAEXPADI@Z 10002c10 f i CudaSupportPlugin.obj
 0001:00001c30       ?deallocate@?$allocator@D@std@@QAEXPADI@Z 10002c30 f i CudaSupportPlugin.obj
 0001:00001c50       ?default_error_condition@_System_error_category@std@@UBE?AVerror_condition@2@H@Z 10002c50 f i CudaSupportPlugin.obj
 0001:00001c90       ?default_error_condition@error_category@std@@UBE?AVerror_condition@2@H@Z 10002c90 f i CudaSupportPlugin.obj
 0001:00001cb0       ?deref@?$QBasicAtomicInteger@H@@QAE_NXZ 10002cb0 f i CudaSupportPlugin.obj
 0001:00001cc0       ?deref@RefCount@QtPrivate@@QAE_NXZ 10002cc0 f i CudaSupportPlugin.obj
 0001:00001ce0       ?detach_helper_grow@?$QList@PAVCudaGpuModel@U2@@@@AAEPAUNode@1@HH@Z 10002ce0 f i CudaSupportPlugin.obj
 0001:00001df0       ?empty@?$QList@PAVCudaGpuModel@U2@@@@QBE_NXZ 10002df0 f i CudaSupportPlugin.obj
 0001:00001e00       ?end@?$QList@PAVCudaGpuModel@U2@@@@QBE?AVconst_iterator@1@XZ 10002e00 f i CudaSupportPlugin.obj
 0001:00001e20       ?equivalent@error_category@std@@UBE_NABVerror_code@2@H@Z 10002e20 f i CudaSupportPlugin.obj
 0001:00001e40       ?equivalent@error_category@std@@UBE_NHABVerror_condition@2@@Z 10002e40 f i CudaSupportPlugin.obj
 0001:00001e80       ?erase@?$basic_string@DU?$char_traits@D@std@@V?$allocator@D@2@@std@@QAEAAV12@I@Z 10002e80 f i CudaSupportPlugin.obj
 0001:00001ec0       ?erase@?$basic_string@DU?$char_traits@D@std@@V?$allocator@D@2@@std@@QAEAAV12@II@Z 10002ec0 f i CudaSupportPlugin.obj
 0001:00001f60       ?generic_category@std@@YAABVerror_category@1@XZ 10002f60 f i CudaSupportPlugin.obj
 0001:00001f70       ?getCudaErrorString@CudaSupportPlugin@U2@@CA?AVQString@@W4cudaError_enum@@@Z 10002f70 f   CudaSupportPlugin.obj
 0001:00001ff0       ?getSettingsErrorString@CudaSupportPlugin@U2@@CA?AVQString@@W4Error@12@@Z 10002ff0 f   CudaSupportPlugin.obj
 0001:000020a0       ?isEmpty@?$QList@PAVCudaGpuModel@U2@@@@QBE_NXZ 100030a0 f i CudaSupportPlugin.obj
 0001:000020b0       ?isShared@RefCount@QtPrivate@@QBE_NXZ 100030b0 f i CudaSupportPlugin.obj
 0001:000020d0       ?length@?$char_traits@D@std@@SAIPBD@Z 100030d0 f i CudaSupportPlugin.obj
 0001:000020f0       ?load@?$QBasicAtomicInteger@H@@QBEHXZ 100030f0 f i CudaSupportPlugin.obj
 0001:00002100       ?loadGpusSettings@CudaSupportPlugin@U2@@AAEXXZ 10003100 f   CudaSupportPlugin.obj
 0001:00002290       ?max_size@?$_Wrap_alloc@V?$allocator@D@std@@@std@@QBEIXZ 10003290 f i CudaSupportPlugin.obj
 0001:000022a0       ?max_size@?$allocator@D@std@@QBEIXZ 100032a0 f i CudaSupportPlugin.obj
 0001:000022b0       ?max_size@?$allocator_traits@V?$allocator@D@std@@@std@@SAIABV?$allocator@D@2@@Z 100032b0 f i CudaSupportPlugin.obj
 0001:000022c0       ?max_size@?$basic_string@DU?$char_traits@D@std@@V?$allocator@D@2@@std@@QBEIXZ 100032c0 f i CudaSupportPlugin.obj
 0001:000022d0       ?message@_Generic_error_category@std@@UBE?AV?$basic_string@DU?$char_traits@D@std@@V?$allocator@D@2@@2@H@Z 100032d0 f i CudaSupportPlugin.obj
 0001:00002350       ?message@_Iostream_error_category@std@@UBE?AV?$basic_string@DU?$char_traits@D@std@@V?$allocator@D@2@@2@H@Z 10003350 f i CudaSupportPlugin.obj
 0001:000023a0       ?message@_System_error_category@std@@UBE?AV?$basic_string@DU?$char_traits@D@std@@V?$allocator@D@2@@2@H@Z 100033a0 f i CudaSupportPlugin.obj
 0001:00002420       ?move@?$char_traits@D@std@@SAPADPADPBDI@Z 10003420 f i CudaSupportPlugin.obj
 0001:00002440       ?name@_Generic_error_category@std@@UBEPBDXZ 10003440 f i CudaSupportPlugin.obj
 0001:00002450       ?name@_Iostream_error_category@std@@UBEPBDXZ 10003450 f i CudaSupportPlugin.obj
 0001:00002460       ?name@_System_error_category@std@@UBEPBDXZ 10003460 f i CudaSupportPlugin.obj
 0001:00002470       ?node_construct@?$QList@PAVCudaGpuModel@U2@@@@AAEXPAUNode@1@ABQAVCudaGpuModel@U2@@@Z 10003470 f i CudaSupportPlugin.obj
 0001:00002490       ?node_copy@?$QList@PAVCudaGpuModel@U2@@@@AAEXPAUNode@1@00@Z 10003490 f i CudaSupportPlugin.obj
 0001:000024c0       ?node_destruct@?$QList@PAVCudaGpuModel@U2@@@@AAEXPAUNode@1@0@Z 100034c0 f i CudaSupportPlugin.obj
 0001:000024d0       ?node_destruct@?$QList@PAVCudaGpuModel@U2@@@@AAEXPAUNode@1@@Z 100034d0 f i CudaSupportPlugin.obj
 0001:000024e0       ?obtainGpusInfo@CudaSupportPlugin@U2@@AAE?AW4Error@12@AAVQString@@@Z 100034e0 f   CudaSupportPlugin.obj
 0001:00002c20       ?push_back@?$QList@PAVCudaGpuModel@U2@@@@QAEXABQAVCudaGpuModel@U2@@@Z 10003c20 f i CudaSupportPlugin.obj
 0001:00002c30       ?ref@?$QBasicAtomicInteger@H@@QAE_NXZ 10003c30 f i CudaSupportPlugin.obj
 0001:00002c50       ?ref@RefCount@QtPrivate@@QAE_NXZ 10003c50 f i CudaSupportPlugin.obj
 0001:00002c70       ?registerAvailableGpus@CudaSupportPlugin@U2@@AAEXXZ 10003c70 f   CudaSupportPlugin.obj
 0001:00002d40       ?size@?$QList@PAVCudaGpuModel@U2@@@@QBEHXZ 10003d40 f i CudaSupportPlugin.obj
 0001:00002d50       ?size@?$basic_string@DU?$char_traits@D@std@@V?$allocator@D@2@@std@@QBEIXZ 10003d50 f i CudaSupportPlugin.obj
 0001:00002d60       ?system_category@std@@YAABVerror_category@1@XZ 10003d60 f i CudaSupportPlugin.obj
 0001:00002d70       ?t@Node@?$QList@PAVCudaGpuModel@U2@@@@QAEAAPAVCudaGpuModel@U2@@XZ 10003d70 f i CudaSupportPlugin.obj
 0001:00002d80       ?tr@CudaSupportPlugin@U2@@SA?AVQString@@PBD0H@Z 10003d80 f i CudaSupportPlugin.obj
 0001:00002db0       ?value@error_code@std@@QBEHXZ 10003db0 f i CudaSupportPlugin.obj
 0001:00002dc0       ?value@error_condition@std@@QBEHXZ 10003dc0 f i CudaSupportPlugin.obj
 0001:00002dd0       _hypot                     10003dd0 f i CudaSupportPlugin.obj
 0001:00002e00       _ugene_plugin_init         10003e00 f   CudaSupportPlugin.obj
 0001:00002e20       ??$_Count_np@PB_N_N@std@@YAHPB_N0AB_N@Z 10003e20 f i CudaSupportSettingsController.obj
 0001:00002e60       ??$_Unchecked@PB_N@std@@YAPB_NPB_N@Z 10003e60 f i CudaSupportSettingsController.obj
 0001:00002e70       ??$count@PB_N_N@std@@YAHPB_N0AB_N@Z 10003e70 f i CudaSupportSettingsController.obj
 0001:00002eb0       ??$qobject_cast@PAVCudaSupportSettingsPageState@U2@@@@YAPAVCudaSupportSettingsPageState@U2@@PAVQObject@@@Z 10003eb0 f i CudaSupportSettingsController.obj
 0001:00002ed0       ??0?$QFlags@W4AlignmentFlag@Qt@@@@QAE@PQPrivate@0@H@Z 10003ed0 f i CudaSupportSettingsController.obj
 0001:00002ee0       ??0?$QFlags@W4AlignmentFlag@Qt@@@@QAE@VQFlag@@@Z 10003ee0 f i CudaSupportSettingsController.obj
 0001:00002ef0       ??0?$QFlags@W4AlignmentFlag@Qt@@@@QAE@W4AlignmentFlag@Qt@@@Z 10003ef0 f i CudaSupportSettingsController.obj
 0001:00002f00       ??0?$QFlags@W4AllocationOption@QArrayData@@@@QAE@PQPrivate@0@H@Z 10003f00 f i CudaSupportSettingsController.obj
 0001:00002f10       ??0?$QFlags@W4AllocationOption@QArrayData@@@@QAE@W4AllocationOption@QArrayData@@@Z 10003f10 f i CudaSupportSettingsController.obj
 0001:00002f20       ??0?$QFlags@W4WindowType@Qt@@@@QAE@PQPrivate@0@H@Z 10003f20 f i CudaSupportSettingsController.obj
 0001:00002f30       ??0?$QList@PAVQCheckBox@@@@QAE@XZ 10003f30 f i CudaSupportSettingsController.obj
 0001:00002f40       ??0?$QVector@_N@@QAE@XZ    10003f40 f i CudaSupportSettingsController.obj
 0001:00002f50       ??0CudaSupportSettingsPageController@U2@@QAE@ABVQString@@PAVQObject@@@Z 10003f50 f   CudaSupportSettingsController.obj
 0001:00003000       ??0CudaSupportSettingsPageState@U2@@QAE@H@Z 10004000 f   CudaSupportSettingsController.obj
 0001:000030a0       ??0CudaSupportSettingsPageWidget@U2@@QAE@ABVQString@@PAVCudaSupportSettingsPageController@1@@Z 100040a0 f   CudaSupportSettingsController.obj
 0001:00003550       ??0QFlag@@QAE@H@Z          10004550 f i CudaSupportSettingsController.obj
 0001:00003560       ??1?$QList@PAVQCheckBox@@@@QAE@XZ 10004560 f i CudaSupportSettingsController.obj
 0001:00003590       ??1?$QVector@_N@@QAE@XZ    10004590 f i CudaSupportSettingsController.obj
 0001:000035d0       ??1CudaSupportSettingsPageController@U2@@UAE@XZ 100045d0 f i CudaSupportSettingsController.obj
 0001:00003630       ??1CudaSupportSettingsPageState@U2@@UAE@XZ 10004630 f i CudaSupportSettingsController.obj
 0001:000036c0       ??1CudaSupportSettingsPageWidget@U2@@UAE@XZ 100046c0 f i CudaSupportSettingsController.obj
 0001:00003750       ??A?$QList@PAVCudaGpuModel@U2@@@@QAEAAPAVCudaGpuModel@U2@@H@Z 10004750 f i CudaSupportSettingsController.obj
 0001:00003780       ??A?$QVector@_N@@QAEAA_NH@Z 10004780 f i CudaSupportSettingsController.obj
 0001:000037f0       ??BQFlag@@QBEHXZ           100047f0 f i CudaSupportSettingsController.obj
 0001:00003800       ??U?$QFlags@W4AlignmentFlag@Qt@@@@QBE?AV0@W4AlignmentFlag@Qt@@@Z 10004800 f i CudaSupportSettingsController.obj
 0001:00003820       ??U@YA?AV?$QFlags@W4AlignmentFlag@Qt@@@@W4AlignmentFlag@Qt@@0@Z 10004820 f i CudaSupportSettingsController.obj
 0001:00003830       ??_ECudaSupportSettingsPageWidget@U2@@W7AEPAXI@Z 10004830 f i CudaSupportSettingsController.obj
 0001:00003838       ??_EQCheckBox@@W7AEPAXI@Z  10004838 f i CudaSupportSettingsController.obj
 0001:00003840       ??_EQHBoxLayout@@W7AEPAXI@Z 10004840 f i CudaSupportSettingsController.obj
 0001:00003848       ??_EQLabel@@W7AEPAXI@Z     10004848 f i CudaSupportSettingsController.obj
 0001:00003850       ??_EQVBoxLayout@@W7AEPAXI@Z 10004850 f i CudaSupportSettingsController.obj
 0001:00003860       ??_GCudaSupportSettingsPageController@U2@@UAEPAXI@Z 10004860 f i CudaSupportSettingsController.obj
 0001:00003860       ??_ECudaSupportSettingsPageController@U2@@UAEPAXI@Z 10004860 f i CudaSupportSettingsController.obj
 0001:000038d0       ??_GCudaSupportSettingsPageState@U2@@UAEPAXI@Z 100048d0 f i CudaSupportSettingsController.obj
 0001:000038d0       ??_ECudaSupportSettingsPageState@U2@@UAEPAXI@Z 100048d0 f i CudaSupportSettingsController.obj
 0001:00003980       ??_ECudaSupportSettingsPageWidget@U2@@UAEPAXI@Z 10004980 f i CudaSupportSettingsController.obj
 0001:00003980       ??_GCudaSupportSettingsPageWidget@U2@@UAEPAXI@Z 10004980 f i CudaSupportSettingsController.obj
 0001:00003a20       ??_GQCheckBox@@UAEPAXI@Z   10004a20 f i CudaSupportSettingsController.obj
 0001:00003a20       ??_EQCheckBox@@UAEPAXI@Z   10004a20 f i CudaSupportSettingsController.obj
 0001:00003a50       ??_EQHBoxLayout@@UAEPAXI@Z 10004a50 f i CudaSupportSettingsController.obj
 0001:00003a50       ??_GQHBoxLayout@@UAEPAXI@Z 10004a50 f i CudaSupportSettingsController.obj
 0001:00003a80       ??_GQLabel@@UAEPAXI@Z      10004a80 f i CudaSupportSettingsController.obj
 0001:00003a80       ??_EQLabel@@UAEPAXI@Z      10004a80 f i CudaSupportSettingsController.obj
 0001:00003ab0       ??_GQVBoxLayout@@UAEPAXI@Z 10004ab0 f i CudaSupportSettingsController.obj
 0001:00003ab0       ??_EQVBoxLayout@@UAEPAXI@Z 10004ab0 f i CudaSupportSettingsController.obj
 0001:00003ae0       ?allocate@?$QTypedArrayData@_N@@SAPAU1@IV?$QFlags@W4AllocationOption@QArrayData@@@@@Z 10004ae0 f i CudaSupportSettingsController.obj
 0001:00003b00       ?append@?$QList@PAVQCheckBox@@@@QAEXABQAVQCheckBox@@@Z 10004b00 f i CudaSupportSettingsController.obj
 0001:00003b90       ?at@?$QList@PAVCudaGpuModel@U2@@@@QBEABQAVCudaGpuModel@U2@@H@Z 10004b90 f i CudaSupportSettingsController.obj
 0001:00003bb0       ?at@?$QList@PAVQCheckBox@@@@QBEABQAVQCheckBox@@H@Z 10004bb0 f i CudaSupportSettingsController.obj
 0001:00003bd0       ?at@?$QVector@_N@@QBEAB_NH@Z 10004bd0 f i CudaSupportSettingsController.obj
 0001:00003bf0       ?begin@?$QTypedArrayData@_N@@QAEPA_NPA_N@Z 10004bf0 f i CudaSupportSettingsController.obj
 0001:00003c00       ?count@?$QVector@_N@@QBEHAB_N@Z 10004c00 f i CudaSupportSettingsController.obj
 0001:00003c60       ?createWidget@CudaSupportSettingsPageController@U2@@UAEPAVAppSettingsGUIPageWidget@2@PAVAppSettingsGUIPageState@2@@Z 10004c60 f   CudaSupportSettingsController.obj
 0001:00003ce0       ?data@?$QTypedArrayData@_N@@QAEPA_NXZ 10004ce0 f i CudaSupportSettingsController.obj
 0001:00003cf0       ?data@?$QVector@_N@@QAEPA_NXZ 10004cf0 f i CudaSupportSettingsController.obj
 0001:00003d50       ?dealloc@?$QList@PAVQCheckBox@@@@AAEXPAUData@QListData@@@Z 10004d50 f i CudaSupportSettingsController.obj
 0001:00003d70       ?deallocate@?$QTypedArrayData@_N@@SAXPAUQArrayData@@@Z 10004d70 f i CudaSupportSettingsController.obj
 0001:00003d90       ?defaultConstruct@?$QVector@_N@@AAEXPA_N0@Z 10004d90 f i CudaSupportSettingsController.obj
 0001:00003db0       ?destruct@?$QVector@_N@@AAEXPA_N0@Z 10004db0 f i CudaSupportSettingsController.obj
 0001:00003dc0       ?detach@?$QList@PAVCudaGpuModel@U2@@@@QAEXXZ 10004dc0 f i CudaSupportSettingsController.obj
 0001:00003de0       ?detach@?$QVector@_N@@QAEXXZ 10004de0 f i CudaSupportSettingsController.obj
 0001:00003e30       ?detach_helper@?$QList@PAVCudaGpuModel@U2@@@@AAEXH@Z 10004e30 f i CudaSupportSettingsController.obj
 0001:00003f00       ?detach_helper@?$QList@PAVCudaGpuModel@U2@@@@AAEXXZ 10004f00 f i CudaSupportSettingsController.obj
 0001:00003f10       ?detach_helper_grow@?$QList@PAVQCheckBox@@@@AAEPAUNode@1@HH@Z 10004f10 f i CudaSupportSettingsController.obj
 0001:00004020       ?end@?$QTypedArrayData@_N@@QAEPA_NPA_N@Z 10005020 f i CudaSupportSettingsController.obj
 0001:00004030       ?freeData@?$QVector@_N@@AAEXPAU?$QTypedArrayData@_N@@@Z 10005030 f i CudaSupportSettingsController.obj
 0001:00004060       ?getHelpPageId@CudaSupportSettingsPageController@U2@@UBEABVQString@@XZ 10005060 f i CudaSupportSettingsController.obj
 0001:00004070       ?getSavedState@CudaSupportSettingsPageController@U2@@UAEPAVAppSettingsGUIPageState@2@XZ 10005070 f   CudaSupportSettingsController.obj
 0001:000041c0       ?getState@CudaSupportSettingsPageWidget@U2@@UBEPAVAppSettingsGUIPageState@2@AAVQString@@@Z 100051c0 f   CudaSupportSettingsController.obj
 0001:000042f0       ?isDetached@?$QVector@_N@@QBE_NXZ 100052f0 f i CudaSupportSettingsController.obj
 0001:00004320       ?node_construct@?$QList@PAVQCheckBox@@@@AAEXPAUNode@1@ABQAVQCheckBox@@@Z 10005320 f i CudaSupportSettingsController.obj
 0001:00004340       ?node_copy@?$QList@PAVQCheckBox@@@@AAEXPAUNode@1@00@Z 10005340 f i CudaSupportSettingsController.obj
 0001:00004370       ?node_destruct@?$QList@PAVQCheckBox@@@@AAEXPAUNode@1@0@Z 10005370 f i CudaSupportSettingsController.obj
 0001:00004380       ?node_destruct@?$QList@PAVQCheckBox@@@@AAEXPAUNode@1@@Z 10005380 f i CudaSupportSettingsController.obj
 0001:00004390       ?push_back@?$QList@PAVQCheckBox@@@@QAEXABQAVQCheckBox@@@Z 10005390 f i CudaSupportSettingsController.obj
 0001:000043a0       ?qt_noop@@YAXXZ            100053a0 f i CudaSupportSettingsController.obj
 0001:000043b0       ?reallocData@?$QVector@_N@@AAEXHHV?$QFlags@W4AllocationOption@QArrayData@@@@@Z 100053b0 f i CudaSupportSettingsController.obj
 0001:000045e0       ?resize@?$QVector@_N@@QAEXH@Z 100055e0 f i CudaSupportSettingsController.obj
 0001:00004630       ?saveState@CudaSupportSettingsPageController@U2@@UAEXPAVAppSettingsGUIPageState@2@@Z 10005630 f   CudaSupportSettingsController.obj
 0001:000047d0       ?setState@CudaSupportSettingsPageWidget@U2@@UAEXPAVAppSettingsGUIPageState@2@@Z 100057d0 f   CudaSupportSettingsController.obj
 0001:00004830       ?sharedNull@?$QTypedArrayData@_N@@SAPAU1@XZ 10005830 f i CudaSupportSettingsController.obj
 0001:00004840       ?size@?$QList@PAVQCheckBox@@@@QBEHXZ 10005840 f i CudaSupportSettingsController.obj
 0001:00004850       ?size@?$QVector@_N@@QBEHXZ 10005850 f i CudaSupportSettingsController.obj
 0001:00004860       ?t@Node@?$QList@PAVQCheckBox@@@@QAEAAPAVQCheckBox@@XZ 10005860 f i CudaSupportSettingsController.obj
 0001:00004870       ?tr@CudaSupportSettingsPageController@U2@@SA?AVQString@@PBD0H@Z 10005870 f i CudaSupportSettingsController.obj
 0001:000048a0       ?tr@CudaSupportSettingsPageWidget@U2@@SA?AVQString@@PBD0H@Z 100058a0 f i CudaSupportSettingsController.obj
 0001:000048d0       ?unsharableEmpty@?$QTypedArrayData@_N@@SAPAU1@XZ 100058d0 f i CudaSupportSettingsController.obj
 0001:000048f0       ??C?$QScopedPointer@VQObjectData@@U?$QScopedPointerDeleter@VQObjectData@@@@@@QBEPAVQObjectData@@XZ 100058f0 f i moc_CudaSupportPlugin.obj
 0001:00004900       ?metaObject@CudaSupportPlugin@U2@@UBEPBUQMetaObject@@XZ 10005900 f   moc_CudaSupportPlugin.obj
 0001:00004920       ?qt_metacall@CudaSupportPlugin@U2@@UAEHW4Call@QMetaObject@@HPAPAX@Z 10005920 f   moc_CudaSupportPlugin.obj
 0001:00004930       ?qt_metacast@CudaSupportPlugin@U2@@UAEPAXPBD@Z 10005930 f   moc_CudaSupportPlugin.obj
 0001:00004990       ?qt_static_metacall@CudaSupportPlugin@U2@@CAXPAVQObject@@W4Call@QMetaObject@@HPAPAX@Z 10005990 f   moc_CudaSupportPlugin.obj
 0001:000049a0       ?metaObject@CudaSupportSettingsPageController@U2@@UBEPBUQMetaObject@@XZ 100059a0 f   moc_CudaSupportSettingsController.obj
 0001:000049c0       ?metaObject@CudaSupportSettingsPageState@U2@@UBEPBUQMetaObject@@XZ 100059c0 f   moc_CudaSupportSettingsController.obj
 0001:000049e0       ?metaObject@CudaSupportSettingsPageWidget@U2@@UBEPBUQMetaObject@@XZ 100059e0 f   moc_CudaSupportSettingsController.obj
 0001:00004a00       ?qt_metacall@CudaSupportSettingsPageController@U2@@UAEHW4Call@QMetaObject@@HPAPAX@Z 10005a00 f   moc_CudaSupportSettingsController.obj
 0001:00004a10       ?qt_metacall@CudaSupportSettingsPageState@U2@@UAEHW4Call@QMetaObject@@HPAPAX@Z 10005a10 f   moc_CudaSupportSettingsController.obj
 0001:00004a20       ?qt_metacall@CudaSupportSettingsPageWidget@U2@@UAEHW4Call@QMetaObject@@HPAPAX@Z 10005a20 f   moc_CudaSupportSettingsController.obj
 0001:00004a30       ?qt_metacast@CudaSupportSettingsPageController@U2@@UAEPAXPBD@Z 10005a30 f   moc_CudaSupportSettingsController.obj
 0001:00004a90       ?qt_metacast@CudaSupportSettingsPageState@U2@@UAEPAXPBD@Z 10005a90 f   moc_CudaSupportSettingsController.obj
 0001:00004af0       ?qt_metacast@CudaSupportSettingsPageWidget@U2@@UAEPAXPBD@Z 10005af0 f   moc_CudaSupportSettingsController.obj
 0001:00004b50       ?qt_static_metacall@CudaSupportSettingsPageController@U2@@CAXPAVQObject@@W4Call@QMetaObject@@HPAPAX@Z 10005b50 f   moc_CudaSupportSettingsController.obj
 0001:00004b60       ?qt_static_metacall@CudaSupportSettingsPageState@U2@@CAXPAVQObject@@W4Call@QMetaObject@@HPAPAX@Z 10005b60 f   moc_CudaSupportSettingsController.obj
 0001:00004b70       ?qt_static_metacall@CudaSupportSettingsPageWidget@U2@@CAXPAVQObject@@W4Call@QMetaObject@@HPAPAX@Z 10005b70 f   moc_CudaSupportSettingsController.obj
 0001:00004b72       ?getSettings@AppContext@U2@@SAPAVSettings@2@XZ 10005b72 f   U2Core:U2Core.dll
 0001:00004b78       ?getAppSettingsGUI@AppContext@U2@@SAPAVAppSettingsGUI@2@XZ 10005b78 f   U2Core:U2Core.dll
 0001:00004b7e       ?getMainWindow@AppContext@U2@@SAPAVMainWindow@2@XZ 10005b7e f   U2Core:U2Core.dll
 0001:00004b84       ?getCudaGpuRegistry@AppContext@U2@@SAPAVCudaGpuRegistry@2@XZ 10005b84 f   U2Core:U2Core.dll
 0001:00004b8a       ??0Logger@U2@@QAE@ABVQString@@@Z 10005b8a f   U2Core:U2Core.dll
 0001:00004b90       ??1Logger@U2@@UAE@XZ       10005b90 f   U2Core:U2Core.dll
 0001:00004b96       ?details@Logger@U2@@QAEXABVQString@@@Z 10005b96 f   U2Core:U2Core.dll
 0001:00004b9c       ??0AppResourceSemaphore@U2@@QAE@HHABVQString@@0@Z 10005b9c f   U2Core:U2Core.dll
 0001:00004ba2       ??1AppResourceSemaphore@U2@@UAE@XZ 10005ba2 f   U2Core:U2Core.dll
 0001:00004ba8       ?registerResource@AppResourcePool@U2@@QAEXPAVAppResource@2@@Z 10005ba8 f   U2Core:U2Core.dll
 0001:00004bae       ?instance@AppResourcePool@U2@@SAPAV12@XZ 10005bae f   U2Core:U2Core.dll
 0001:00004bb4       ??0Plugin@U2@@QAE@ABVQString@@0_NW4PluginState@1@@Z 10005bb4 f   U2Core:U2Core.dll
 0001:00004bba       ??1Plugin@U2@@UAE@XZ       10005bba f   U2Core:U2Core.dll
 0001:00004bc0       ?acquire@AppResourceSemaphore@U2@@UAEXHW4MemoryLockType@AppResource@2@@Z 10005bc0 f   U2Core:U2Core.dll
 0001:00004bc6       ?available@AppResourceSemaphore@U2@@UBEHXZ 10005bc6 f   U2Core:U2Core.dll
 0001:00004bcc       ?release@AppResourceSemaphore@U2@@UAEXHW4MemoryLockType@AppResource@2@@Z 10005bcc f   U2Core:U2Core.dll
 0001:00004bd2       ?tryAcquire@AppResourceSemaphore@U2@@UAE_NHHW4MemoryLockType@AppResource@2@@Z 10005bd2 f   U2Core:U2Core.dll
 0001:00004bd8       ?tryAcquire@AppResourceSemaphore@U2@@UAE_NHW4MemoryLockType@AppResource@2@@Z 10005bd8 f   U2Core:U2Core.dll
 0001:00004bde       ?setMaxUse@AppResourceSemaphore@U2@@QAEXH@Z 10005bde f   U2Core:U2Core.dll
 0001:00004be4       ?getResource@AppResourcePool@U2@@QBEPAVAppResource@2@H@Z 10005be4 f   U2Core:U2Core.dll
 0001:00004bea       ?qt_metacast@Plugin@U2@@UAEPAXPBD@Z 10005bea f   U2Core:U2Core.dll
 0001:00004bf0       ?qt_metacall@Plugin@U2@@UAEHW4Call@QMetaObject@@HPAPAX@Z 10005bf0 f   U2Core:U2Core.dll
 0001:00004bf6       ??0CudaGpuModel@U2@@QAE@ABVQString@@ABH_K_N@Z 10005bf6 f   U2Algorithm:U2Algorithm.dll
 0001:00004bfc       ?getName@CudaGpuModel@U2@@QBE?AVQString@@XZ 10005bfc f   U2Algorithm:U2Algorithm.dll
 0001:00004c02       ?registerCudaGpu@CudaGpuRegistry@U2@@QAEXPAVCudaGpuModel@2@@Z 10005c02 f   U2Algorithm:U2Algorithm.dll
 0001:00004c08       ?getRegisteredGpus@CudaGpuRegistry@U2@@QBE?AV?$QList@PAVCudaGpuModel@U2@@@@XZ 10005c08 f   U2Algorithm:U2Algorithm.dll
 0001:00004c0e       ??1AppSettingsGUIPageState@U2@@UAE@XZ 10005c0e f   U2Gui:U2Gui.dll
 0001:00004c14       ??0AppSettingsGUIPageWidget@U2@@QAE@PAVQWidget@@@Z 10005c14 f   U2Gui:U2Gui.dll
 0001:00004c1a       ??1AppSettingsGUIPageWidget@U2@@UAE@XZ 10005c1a f   U2Gui:U2Gui.dll
 0001:00004c20       ??0AppSettingsGUIPageController@U2@@QAE@ABVQString@@0PAVQObject@@@Z 10005c20 f   U2Gui:U2Gui.dll
 0001:00004c26       ??1AppSettingsGUIPageController@U2@@UAE@XZ 10005c26 f   U2Gui:U2Gui.dll
 0001:00004c2c       ?qt_metacast@AppSettingsGUIPageState@U2@@UAEPAXPBD@Z 10005c2c f   U2Gui:U2Gui.dll
 0001:00004c32       ?qt_metacall@AppSettingsGUIPageState@U2@@UAEHW4Call@QMetaObject@@HPAPAX@Z 10005c32 f   U2Gui:U2Gui.dll
 0001:00004c38       ?qt_metacast@AppSettingsGUIPageWidget@U2@@UAEPAXPBD@Z 10005c38 f   U2Gui:U2Gui.dll
 0001:00004c3e       ?qt_metacall@AppSettingsGUIPageWidget@U2@@UAEHW4Call@QMetaObject@@HPAPAX@Z 10005c3e f   U2Gui:U2Gui.dll
 0001:00004c44       ?qt_metacast@AppSettingsGUIPageController@U2@@UAEPAXPBD@Z 10005c44 f   U2Gui:U2Gui.dll
 0001:00004c4a       ?qt_metacall@AppSettingsGUIPageController@U2@@UAEHW4Call@QMetaObject@@HPAPAX@Z 10005c4a f   U2Gui:U2Gui.dll
 0001:00004c50       ??1QWidget@@UAE@XZ         10005c50 f   Qt5Widgets:Qt5Widgets.dll
 0001:00004c56       ?setLayout@QWidget@@QAEXPAVQLayout@@@Z 10005c56 f   Qt5Widgets:Qt5Widgets.dll
 0001:00004c5c       ??0QLabel@@QAE@ABVQString@@PAVQWidget@@V?$QFlags@W4WindowType@Qt@@@@@Z 10005c5c f   Qt5Widgets:Qt5Widgets.dll
 0001:00004c62       ??1QLabel@@UAE@XZ          10005c62 f   Qt5Widgets:Qt5Widgets.dll
 0001:00004c68       ?setAlignment@QLabel@@QAEXV?$QFlags@W4AlignmentFlag@Qt@@@@@Z 10005c68 f   Qt5Widgets:Qt5Widgets.dll
 0001:00004c6e       ?setAlignment@QLayoutItem@@QAEXV?$QFlags@W4AlignmentFlag@Qt@@@@@Z 10005c6e f   Qt5Widgets:Qt5Widgets.dll
 0001:00004c74       ?addStretch@QBoxLayout@@QAEXH@Z 10005c74 f   Qt5Widgets:Qt5Widgets.dll
 0001:00004c7a       ?addWidget@QBoxLayout@@QAEXPAVQWidget@@HV?$QFlags@W4AlignmentFlag@Qt@@@@@Z 10005c7a f   Qt5Widgets:Qt5Widgets.dll
 0001:00004c80       ?addLayout@QBoxLayout@@QAEXPAVQLayout@@H@Z 10005c80 f   Qt5Widgets:Qt5Widgets.dll
 0001:00004c86       ??0QHBoxLayout@@QAE@PAVQWidget@@@Z 10005c86 f   Qt5Widgets:Qt5Widgets.dll
 0001:00004c8c       ??1QHBoxLayout@@UAE@XZ     10005c8c f   Qt5Widgets:Qt5Widgets.dll
 0001:00004c92       ??0QVBoxLayout@@QAE@PAVQWidget@@@Z 10005c92 f   Qt5Widgets:Qt5Widgets.dll
 0001:00004c98       ??1QVBoxLayout@@UAE@XZ     10005c98 f   Qt5Widgets:Qt5Widgets.dll
 0001:00004c9e       ?isChecked@QAbstractButton@@QBE_NXZ 10005c9e f   Qt5Widgets:Qt5Widgets.dll
 0001:00004ca4       ?setChecked@QAbstractButton@@QAEX_N@Z 10005ca4 f   Qt5Widgets:Qt5Widgets.dll
 0001:00004caa       ??0QCheckBox@@QAE@ABVQString@@PAVQWidget@@@Z 10005caa f   Qt5Widgets:Qt5Widgets.dll
 0001:00004cb0       ??1QCheckBox@@UAE@XZ       10005cb0 f   Qt5Widgets:Qt5Widgets.dll
 0001:00004cb6       ?actionEvent@QWidget@@MAEXPAVQActionEvent@@@Z 10005cb6 f   Qt5Widgets:Qt5Widgets.dll
 0001:00004cbc       ?addItem@QBoxLayout@@UAEXPAVQLayoutItem@@@Z 10005cbc f   Qt5Widgets:Qt5Widgets.dll
 0001:00004cc2       ?changeEvent@QAbstractButton@@MAEXPAVQEvent@@@Z 10005cc2 f   Qt5Widgets:Qt5Widgets.dll
 0001:00004cc8       ?changeEvent@QLabel@@MAEXPAVQEvent@@@Z 10005cc8 f   Qt5Widgets:Qt5Widgets.dll
 0001:00004cce       ?changeEvent@QWidget@@MAEXPAVQEvent@@@Z 10005cce f   Qt5Widgets:Qt5Widgets.dll
 0001:00004cd4       ?checkStateSet@QCheckBox@@MAEXXZ 10005cd4 f   Qt5Widgets:Qt5Widgets.dll
 0001:00004cda       ?childEvent@QLayout@@MAEXPAVQChildEvent@@@Z 10005cda f   Qt5Widgets:Qt5Widgets.dll
 0001:00004ce0       ?closeEvent@QWidget@@MAEXPAVQCloseEvent@@@Z 10005ce0 f   Qt5Widgets:Qt5Widgets.dll
 0001:00004ce6       ?contextMenuEvent@QLabel@@MAEXPAVQContextMenuEvent@@@Z 10005ce6 f   Qt5Widgets:Qt5Widgets.dll
 0001:00004cec       ?contextMenuEvent@QWidget@@MAEXPAVQContextMenuEvent@@@Z 10005cec f   Qt5Widgets:Qt5Widgets.dll
 0001:00004cf2       ?controlTypes@QLayout@@UBE?AV?$QFlags@W4ControlType@QSizePolicy@@@@XZ 10005cf2 f   Qt5Widgets:Qt5Widgets.dll
 0001:00004cf8       ?count@QBoxLayout@@UBEHXZ  10005cf8 f   Qt5Widgets:Qt5Widgets.dll
 0001:00004cfe       ?devType@QWidget@@UBEHXZ   10005cfe f   Qt5Widgets:Qt5Widgets.dll
 0001:00004d04       ?dragEnterEvent@QWidget@@MAEXPAVQDragEnterEvent@@@Z 10005d04 f   Qt5Widgets:Qt5Widgets.dll
 0001:00004d0a       ?dragLeaveEvent@QWidget@@MAEXPAVQDragLeaveEvent@@@Z 10005d0a f   Qt5Widgets:Qt5Widgets.dll
 0001:00004d10       ?dragMoveEvent@QWidget@@MAEXPAVQDragMoveEvent@@@Z 10005d10 f   Qt5Widgets:Qt5Widgets.dll
 0001:00004d16       ?dropEvent@QWidget@@MAEXPAVQDropEvent@@@Z 10005d16 f   Qt5Widgets:Qt5Widgets.dll
 0001:00004d1c       ?enterEvent@QWidget@@MAEXPAVQEvent@@@Z 10005d1c f   Qt5Widgets:Qt5Widgets.dll
 0001:00004d22       ?event@QCheckBox@@MAE_NPAVQEvent@@@Z 10005d22 f   Qt5Widgets:Qt5Widgets.dll
 0001:00004d28       ?event@QLabel@@MAE_NPAVQEvent@@@Z 10005d28 f   Qt5Widgets:Qt5Widgets.dll
 0001:00004d2e       ?event@QWidget@@MAE_NPAVQEvent@@@Z 10005d2e f   Qt5Widgets:Qt5Widgets.dll
 0001:00004d34       ?expandingDirections@QBoxLayout@@UBE?AV?$QFlags@W4Orientation@Qt@@@@XZ 10005d34 f   Qt5Widgets:Qt5Widgets.dll
 0001:00004d3a       ?focusInEvent@QAbstractButton@@MAEXPAVQFocusEvent@@@Z 10005d3a f   Qt5Widgets:Qt5Widgets.dll
 0001:00004d40       ?focusInEvent@QLabel@@MAEXPAVQFocusEvent@@@Z 10005d40 f   Qt5Widgets:Qt5Widgets.dll
 0001:00004d46       ?focusInEvent@QWidget@@MAEXPAVQFocusEvent@@@Z 10005d46 f   Qt5Widgets:Qt5Widgets.dll
 0001:00004d4c       ?focusNextPrevChild@QLabel@@MAE_N_N@Z 10005d4c f   Qt5Widgets:Qt5Widgets.dll
 0001:00004d52       ?focusNextPrevChild@QWidget@@MAE_N_N@Z 10005d52 f   Qt5Widgets:Qt5Widgets.dll
 0001:00004d58       ?focusOutEvent@QAbstractButton@@MAEXPAVQFocusEvent@@@Z 10005d58 f   Qt5Widgets:Qt5Widgets.dll
 0001:00004d5e       ?focusOutEvent@QLabel@@MAEXPAVQFocusEvent@@@Z 10005d5e f   Qt5Widgets:Qt5Widgets.dll
 0001:00004d64       ?focusOutEvent@QWidget@@MAEXPAVQFocusEvent@@@Z 10005d64 f   Qt5Widgets:Qt5Widgets.dll
 0001:00004d6a       ?geometry@QLayout@@UBE?AVQRect@@XZ 10005d6a f   Qt5Widgets:Qt5Widgets.dll
 0001:00004d70       ?hasHeightForWidth@QBoxLayout@@UBE_NXZ 10005d70 f   Qt5Widgets:Qt5Widgets.dll
 0001:00004d76       ?hasHeightForWidth@QWidget@@UBE_NXZ 10005d76 f   Qt5Widgets:Qt5Widgets.dll
 0001:00004d7c       ?heightForWidth@QBoxLayout@@UBEHH@Z 10005d7c f   Qt5Widgets:Qt5Widgets.dll
 0001:00004d82       ?heightForWidth@QLabel@@UBEHH@Z 10005d82 f   Qt5Widgets:Qt5Widgets.dll
 0001:00004d88       ?heightForWidth@QWidget@@UBEHH@Z 10005d88 f   Qt5Widgets:Qt5Widgets.dll
 0001:00004d8e       ?hideEvent@QWidget@@MAEXPAVQHideEvent@@@Z 10005d8e f   Qt5Widgets:Qt5Widgets.dll
 0001:00004d94       ?hitButton@QCheckBox@@MBE_NABVQPoint@@@Z 10005d94 f   Qt5Widgets:Qt5Widgets.dll
 0001:00004d9a       ?indexOf@QLayout@@UBEHPAVQWidget@@@Z 10005d9a f   Qt5Widgets:Qt5Widgets.dll
 0001:00004da0       ?initPainter@QWidget@@MBEXPAVQPainter@@@Z 10005da0 f   Qt5Widgets:Qt5Widgets.dll
 0001:00004da6       ?inputMethodEvent@QWidget@@MAEXPAVQInputMethodEvent@@@Z 10005da6 f   Qt5Widgets:Qt5Widgets.dll
 0001:00004dac       ?inputMethodQuery@QWidget@@UBE?AVQVariant@@W4InputMethodQuery@Qt@@@Z 10005dac f   Qt5Widgets:Qt5Widgets.dll
 0001:00004db2       ?invalidate@QBoxLayout@@UAEXXZ 10005db2 f   Qt5Widgets:Qt5Widgets.dll
 0001:00004db8       ?isEmpty@QLayout@@UBE_NXZ  10005db8 f   Qt5Widgets:Qt5Widgets.dll
 0001:00004dbe       ?itemAt@QBoxLayout@@UBEPAVQLayoutItem@@H@Z 10005dbe f   Qt5Widgets:Qt5Widgets.dll
 0001:00004dc4       ?keyPressEvent@QAbstractButton@@MAEXPAVQKeyEvent@@@Z 10005dc4 f   Qt5Widgets:Qt5Widgets.dll
 0001:00004dca       ?keyPressEvent@QLabel@@MAEXPAVQKeyEvent@@@Z 10005dca f   Qt5Widgets:Qt5Widgets.dll
 0001:00004dd0       ?keyPressEvent@QWidget@@MAEXPAVQKeyEvent@@@Z 10005dd0 f   Qt5Widgets:Qt5Widgets.dll
 0001:00004dd6       ?keyReleaseEvent@QAbstractButton@@MAEXPAVQKeyEvent@@@Z 10005dd6 f   Qt5Widgets:Qt5Widgets.dll
 0001:00004ddc       ?keyReleaseEvent@QWidget@@MAEXPAVQKeyEvent@@@Z 10005ddc f   Qt5Widgets:Qt5Widgets.dll
 0001:00004de2       ?layout@QLayout@@UAEPAV1@XZ 10005de2 f   Qt5Widgets:Qt5Widgets.dll
 0001:00004de8       ?leaveEvent@QWidget@@MAEXPAVQEvent@@@Z 10005de8 f   Qt5Widgets:Qt5Widgets.dll
 0001:00004dee       ?maximumSize@QBoxLayout@@UBE?AVQSize@@XZ 10005dee f   Qt5Widgets:Qt5Widgets.dll
 0001:00004df4       ?metaObject@QCheckBox@@UBEPBUQMetaObject@@XZ 10005df4 f   Qt5Widgets:Qt5Widgets.dll
 0001:00004dfa       ?metaObject@QHBoxLayout@@UBEPBUQMetaObject@@XZ 10005dfa f   Qt5Widgets:Qt5Widgets.dll
 0001:00004e00       ?metaObject@QLabel@@UBEPBUQMetaObject@@XZ 10005e00 f   Qt5Widgets:Qt5Widgets.dll
 0001:00004e06       ?metaObject@QVBoxLayout@@UBEPBUQMetaObject@@XZ 10005e06 f   Qt5Widgets:Qt5Widgets.dll
 0001:00004e0c       ?metric@QWidget@@MBEHW4PaintDeviceMetric@QPaintDevice@@@Z 10005e0c f   Qt5Widgets:Qt5Widgets.dll
 0001:00004e12       ?minimumHeightForWidth@QBoxLayout@@UBEHH@Z 10005e12 f   Qt5Widgets:Qt5Widgets.dll
 0001:00004e18       ?minimumSize@QBoxLayout@@UBE?AVQSize@@XZ 10005e18 f   Qt5Widgets:Qt5Widgets.dll
 0001:00004e1e       ?minimumSizeHint@QCheckBox@@UBE?AVQSize@@XZ 10005e1e f   Qt5Widgets:Qt5Widgets.dll
 0001:00004e24       ?minimumSizeHint@QLabel@@UBE?AVQSize@@XZ 10005e24 f   Qt5Widgets:Qt5Widgets.dll
 0001:00004e2a       ?minimumSizeHint@QWidget@@UBE?AVQSize@@XZ 10005e2a f   Qt5Widgets:Qt5Widgets.dll
 0001:00004e30       ?mouseDoubleClickEvent@QWidget@@MAEXPAVQMouseEvent@@@Z 10005e30 f   Qt5Widgets:Qt5Widgets.dll
 0001:00004e36       ?mouseMoveEvent@QCheckBox@@MAEXPAVQMouseEvent@@@Z 10005e36 f   Qt5Widgets:Qt5Widgets.dll
 0001:00004e3c       ?mouseMoveEvent@QLabel@@MAEXPAVQMouseEvent@@@Z 10005e3c f   Qt5Widgets:Qt5Widgets.dll
 0001:00004e42       ?mouseMoveEvent@QWidget@@MAEXPAVQMouseEvent@@@Z 10005e42 f   Qt5Widgets:Qt5Widgets.dll
 0001:00004e48       ?mousePressEvent@QAbstractButton@@MAEXPAVQMouseEvent@@@Z 10005e48 f   Qt5Widgets:Qt5Widgets.dll
 0001:00004e4e       ?mousePressEvent@QLabel@@MAEXPAVQMouseEvent@@@Z 10005e4e f   Qt5Widgets:Qt5Widgets.dll
 0001:00004e54       ?mousePressEvent@QWidget@@MAEXPAVQMouseEvent@@@Z 10005e54 f   Qt5Widgets:Qt5Widgets.dll
 0001:00004e5a       ?mouseReleaseEvent@QAbstractButton@@MAEXPAVQMouseEvent@@@Z 10005e5a f   Qt5Widgets:Qt5Widgets.dll
 0001:00004e60       ?mouseReleaseEvent@QLabel@@MAEXPAVQMouseEvent@@@Z 10005e60 f   Qt5Widgets:Qt5Widgets.dll
 0001:00004e66       ?mouseReleaseEvent@QWidget@@MAEXPAVQMouseEvent@@@Z 10005e66 f   Qt5Widgets:Qt5Widgets.dll
 0001:00004e6c       ?moveEvent@QWidget@@MAEXPAVQMoveEvent@@@Z 10005e6c f   Qt5Widgets:Qt5Widgets.dll
 0001:00004e72       ?nativeEvent@QWidget@@MAE_NABVQByteArray@@PAXPAJ@Z 10005e72 f   Qt5Widgets:Qt5Widgets.dll
 0001:00004e78       ?nextCheckState@QCheckBox@@MAEXXZ 10005e78 f   Qt5Widgets:Qt5Widgets.dll
 0001:00004e7e       ?paintEngine@QWidget@@UBEPAVQPaintEngine@@XZ 10005e7e f   Qt5Widgets:Qt5Widgets.dll
 0001:00004e84       ?paintEvent@QCheckBox@@MAEXPAVQPaintEvent@@@Z 10005e84 f   Qt5Widgets:Qt5Widgets.dll
 0001:00004e8a       ?paintEvent@QLabel@@MAEXPAVQPaintEvent@@@Z 10005e8a f   Qt5Widgets:Qt5Widgets.dll
 0001:00004e90       ?paintEvent@QWidget@@MAEXPAVQPaintEvent@@@Z 10005e90 f   Qt5Widgets:Qt5Widgets.dll
 0001:00004e96       ?qt_metacall@QCheckBox@@UAEHW4Call@QMetaObject@@HPAPAX@Z 10005e96 f   Qt5Widgets:Qt5Widgets.dll
 0001:00004e9c       ?qt_metacall@QHBoxLayout@@UAEHW4Call@QMetaObject@@HPAPAX@Z 10005e9c f   Qt5Widgets:Qt5Widgets.dll
 0001:00004ea2       ?qt_metacall@QLabel@@UAEHW4Call@QMetaObject@@HPAPAX@Z 10005ea2 f   Qt5Widgets:Qt5Widgets.dll
 0001:00004ea8       ?qt_metacall@QVBoxLayout@@UAEHW4Call@QMetaObject@@HPAPAX@Z 10005ea8 f   Qt5Widgets:Qt5Widgets.dll
 0001:00004eae       ?qt_metacast@QCheckBox@@UAEPAXPBD@Z 10005eae f   Qt5Widgets:Qt5Widgets.dll
 0001:00004eb4       ?qt_metacast@QHBoxLayout@@UAEPAXPBD@Z 10005eb4 f   Qt5Widgets:Qt5Widgets.dll
 0001:00004eba       ?qt_metacast@QLabel@@UAEPAXPBD@Z 10005eba f   Qt5Widgets:Qt5Widgets.dll
 0001:00004ec0       ?qt_metacast@QVBoxLayout@@UAEPAXPBD@Z 10005ec0 f   Qt5Widgets:Qt5Widgets.dll
 0001:00004ec6       ?redirected@QWidget@@MBEPAVQPaintDevice@@PAVQPoint@@@Z 10005ec6 f   Qt5Widgets:Qt5Widgets.dll
 0001:00004ecc       ?resizeEvent@QWidget@@MAEXPAVQResizeEvent@@@Z 10005ecc f   Qt5Widgets:Qt5Widgets.dll
 0001:00004ed2       ?setGeometry@QBoxLayout@@UAEXABVQRect@@@Z 10005ed2 f   Qt5Widgets:Qt5Widgets.dll
 0001:00004ed8       ?setVisible@QWidget@@UAEX_N@Z 10005ed8 f   Qt5Widgets:Qt5Widgets.dll
 0001:00004ede       ?sharedPainter@QWidget@@MBEPAVQPainter@@XZ 10005ede f   Qt5Widgets:Qt5Widgets.dll
 0001:00004ee4       ?showEvent@QWidget@@MAEXPAVQShowEvent@@@Z 10005ee4 f   Qt5Widgets:Qt5Widgets.dll
 0001:00004eea       ?sizeHint@QBoxLayout@@UBE?AVQSize@@XZ 10005eea f   Qt5Widgets:Qt5Widgets.dll
 0001:00004ef0       ?sizeHint@QCheckBox@@UBE?AVQSize@@XZ 10005ef0 f   Qt5Widgets:Qt5Widgets.dll
 0001:00004ef6       ?sizeHint@QLabel@@UBE?AVQSize@@XZ 10005ef6 f   Qt5Widgets:Qt5Widgets.dll
 0001:00004efc       ?sizeHint@QWidget@@UBE?AVQSize@@XZ 10005efc f   Qt5Widgets:Qt5Widgets.dll
 0001:00004f02       ?spacerItem@QLayoutItem@@UAEPAVQSpacerItem@@XZ 10005f02 f   Qt5Widgets:Qt5Widgets.dll
 0001:00004f08       ?tabletEvent@QWidget@@MAEXPAVQTabletEvent@@@Z 10005f08 f   Qt5Widgets:Qt5Widgets.dll
 0001:00004f0e       ?takeAt@QBoxLayout@@UAEPAVQLayoutItem@@H@Z 10005f0e f   Qt5Widgets:Qt5Widgets.dll
 0001:00004f14       ?timerEvent@QAbstractButton@@MAEXPAVQTimerEvent@@@Z 10005f14 f   Qt5Widgets:Qt5Widgets.dll
 0001:00004f1a       ?wheelEvent@QWidget@@MAEXPAVQWheelEvent@@@Z 10005f1a f   Qt5Widgets:Qt5Widgets.dll
 0001:00004f20       ?widget@QLayoutItem@@UAEPAVQWidget@@XZ 10005f20 f   Qt5Widgets:Qt5Widgets.dll
 0001:00004f26       ?tr@QMetaObject@@QBE?AVQString@@PBD0H@Z 10005f26 f   Qt5Core:Qt5Core.dll
 0001:00004f2c       ??0QChar@@QAE@UQLatin1Char@@@Z 10005f2c f   Qt5Core:Qt5Core.dll
 0001:00004f32       ??0QByteArray@@QAE@HD@Z    10005f32 f   Qt5Core:Qt5Core.dll
 0001:00004f38       ??1QByteArray@@QAE@XZ      10005f38 f   Qt5Core:Qt5Core.dll
 0001:00004f3e       ?data@QByteArray@@QAEPADXZ 10005f3e f   Qt5Core:Qt5Core.dll
 0001:00004f44       ??0QString@@QAE@XZ         10005f44 f   Qt5Core:Qt5Core.dll
 0001:00004f4a       ??0QString@@QAE@ABV0@@Z    10005f4a f   Qt5Core:Qt5Core.dll
 0001:00004f50       ??1QString@@QAE@XZ         10005f50 f   Qt5Core:Qt5Core.dll
 0001:00004f56       ??4QString@@QAEAAV0@ABV0@@Z 10005f56 f   Qt5Core:Qt5Core.dll
 0001:00004f5c       ??4QString@@QAEAAV0@$$QAV0@@Z 10005f5c f   Qt5Core:Qt5Core.dll
 0001:00004f62       ?arg@QString@@QBE?AV1@ABV1@HVQChar@@@Z 10005f62 f   Qt5Core:Qt5Core.dll
 0001:00004f68       ?arg@QString@@QBE?AV1@ABV1@0@Z 10005f68 f   Qt5Core:Qt5Core.dll
 0001:00004f6e       ?append@QString@@QAEAAV1@ABV1@@Z 10005f6e f   Qt5Core:Qt5Core.dll
 0001:00004f74       ?fromUtf8@QString@@SA?AV1@PBDH@Z 10005f74 f   Qt5Core:Qt5Core.dll
 0001:00004f7a       ?number@QString@@SA?AV1@HH@Z 10005f7a f   Qt5Core:Qt5Core.dll
 0001:00004f80       ??0QString@@QAE@ABVQByteArray@@@Z 10005f80 f   Qt5Core:Qt5Core.dll
 0001:00004f86       ??4QString@@QAEAAV0@PBD@Z  10005f86 f   Qt5Core:Qt5Core.dll
 0001:00004f8c       ?fromAscii_helper@QString@@CAPAU?$QTypedArrayData@G@@PBDH@Z 10005f8c f   Qt5Core:Qt5Core.dll
 0001:00004f92       ?detach@QListData@@QAEPAUData@1@H@Z 10005f92 f   Qt5Core:Qt5Core.dll
 0001:00004f98       ?detach_grow@QListData@@QAEPAUData@1@PAHH@Z 10005f98 f   Qt5Core:Qt5Core.dll
 0001:00004f9e       ?dispose@QListData@@SAXPAUData@1@@Z 10005f9e f   Qt5Core:Qt5Core.dll
 0001:00004fa4       ?append@QListData@@QAEPAPAXXZ 10005fa4 f   Qt5Core:Qt5Core.dll
 0001:00004faa       ??0QLibrary@@QAE@ABVQString@@PAVQObject@@@Z 10005faa f   Qt5Core:Qt5Core.dll
 0001:00004fb0       ??1QLibrary@@UAE@XZ        10005fb0 f   Qt5Core:Qt5Core.dll
 0001:00004fb6       ?resolve@QLibrary@@QAEP6AXXZPBD@Z 10005fb6 f   Qt5Core:Qt5Core.dll
 0001:00004fbc       ?load@QLibrary@@QAE_NXZ    10005fbc f   Qt5Core:Qt5Core.dll
 0001:00004fc2       ?isLoaded@QLibrary@@QBE_NXZ 10005fc2 f   Qt5Core:Qt5Core.dll
 0001:00004fc8       ?fileName@QLibrary@@QBE?AVQString@@XZ 10005fc8 f   Qt5Core:Qt5Core.dll
 0001:00004fce       ?errorString@QLibrary@@QBE?AVQString@@XZ 10005fce f   Qt5Core:Qt5Core.dll
 0001:00004fd4       ??0QVariant@@QAE@XZ        10005fd4 f   Qt5Core:Qt5Core.dll
 0001:00004fda       ??1QVariant@@QAE@XZ        10005fda f   Qt5Core:Qt5Core.dll
 0001:00004fe0       ?isNull@QVariant@@QBE_NXZ  10005fe0 f   Qt5Core:Qt5Core.dll
 0001:00004fe6       ?toBool@QVariant@@QBE_NXZ  10005fe6 f   Qt5Core:Qt5Core.dll
 0001:00004fec       ?childEvent@QObject@@MAEXPAVQChildEvent@@@Z 10005fec f   Qt5Core:Qt5Core.dll
 0001:00004ff2       ?connectNotify@QObject@@MAEXABVQMetaMethod@@@Z 10005ff2 f   Qt5Core:Qt5Core.dll
 0001:00004ff8       ?customEvent@QObject@@MAEXPAVQEvent@@@Z 10005ff8 f   Qt5Core:Qt5Core.dll
 0001:00004ffe       ?disconnectNotify@QObject@@MAEXABVQMetaMethod@@@Z 10005ffe f   Qt5Core:Qt5Core.dll
 0001:00005004       ?event@QObject@@UAE_NPAVQEvent@@@Z 10006004 f   Qt5Core:Qt5Core.dll
 0001:0000500a       ?eventFilter@QObject@@UAE_NPAV1@PAVQEvent@@@Z 1000600a f   Qt5Core:Qt5Core.dll
 0001:00005010       ?timerEvent@QObject@@MAEXPAVQTimerEvent@@@Z 10006010 f   Qt5Core:Qt5Core.dll
 0001:00005016       ?qBadAlloc@@YAXXZ          10006016 f   Qt5Core:Qt5Core.dll
 0001:0000501c       ?cast@QMetaObject@@QBEPAVQObject@@PAV2@@Z 1000601c f   Qt5Core:Qt5Core.dll
 0001:00005022       ?data@QArrayData@@QAEPAXXZ 10006022 f   Qt5Core:Qt5Core.dll
 0001:00005028       ?allocate@QArrayData@@SAPAU1@IIIV?$QFlags@W4AllocationOption@QArrayData@@@@@Z 10006028 f   Qt5Core:Qt5Core.dll
 0001:0000502e       ?deallocate@QArrayData@@SAXPAU1@II@Z 1000602e f   Qt5Core:Qt5Core.dll
 0001:00005034       ?number@QString@@SA?AV1@_KH@Z 10006034 f   Qt5Core:Qt5Core.dll
 0001:0000503a       ??0QObject@@QAE@PAV0@@Z    1000603a f   Qt5Core:Qt5Core.dll
 0001:00005040       ??1QObject@@UAE@XZ         10006040 f   Qt5Core:Qt5Core.dll
 0001:00005046       ?dynamicMetaObject@QObjectData@@QBEPAUQMetaObject@@XZ 10006046 f   Qt5Core:Qt5Core.dll
 0001:0000504c       ?_Xbad_alloc@std@@YAXXZ    1000604c f   msvcprt:MSVCP120.dll
 0001:00005052       ?_Xlength_error@std@@YAXPBD@Z 10006052 f   msvcprt:MSVCP120.dll
 0001:00005058       ?_Xout_of_range@std@@YAXPBD@Z 10006058 f   msvcprt:MSVCP120.dll
 0001:0000505e       ?_Syserror_map@std@@YAPBDH@Z 1000605e f   msvcprt:MSVCP120.dll
 0001:00005064       ?_Winerror_map@std@@YAPBDH@Z 10006064 f   msvcprt:MSVCP120.dll
 0001:0000506a       __purecall                 1000606a f   MSVCRT:MSVCR120.dll
 0001:00005070       ??2@YAPAXI@Z               10006070 f   MSVCRT:MSVCR120.dll
 0001:00005076       ??3@YAXPAX@Z               10006076 f   MSVCRT:MSVCR120.dll
 0001:0000507c       ___atonexitinit            1000607c f   MSVCRT:atonexit.obj
 0001:000050b8       __onexit                   100060b8 f   MSVCRT:atonexit.obj
 0001:00005161       _atexit                    10006161 f   MSVCRT:atonexit.obj
 0001:00005176       _memmove                   10006176 f   MSVCRT:MSVCR120.dll
 0001:0000517c       __hypot                    1000617c f   MSVCRT:MSVCR120.dll
 0001:00005182       @__security_check_cookie@4 10006182 f   MSVCRT:secchk.obj
 0001:00005192       __CxxThrowException@8      10006192 f   MSVCRT:MSVCR120.dll
 0001:00005198       ___CxxFrameHandler3        10006198 f   MSVCRT:MSVCR120.dll
 0001:0000519e       _memcpy                    1000619e f   MSVCRT:MSVCR120.dll
 0001:000051a4       ??0type_info@@AAE@ABV0@@Z  100061a4 f   MSVCRT:ti_inst.obj
 0001:000051af       ??4type_info@@AAEAAV0@ABV0@@Z 100061af f   MSVCRT:ti_inst.obj
 0001:000051b4       ??_Etype_info@@UAEPAXI@Z   100061b4 f i MSVCRT:ti_inst.obj
 0001:00005200       ___RTDynamicCast           10006200 f   MSVCRT:MSVCR120.dll
 0001:00005206       _memset                    10006206 f   MSVCRT:MSVCR120.dll
 0001:00005258       _NtCurrentTeb              10006258 f i MSVCRT:crtdll.obj
 0001:0000525f       __CRT_INIT@12              1000625f f   MSVCRT:crtdll.obj
 0001:00005456       __DllMainCRTStartup@12     10006456 f   MSVCRT:crtdll.obj
 0001:000055ac       __lock                     100065ac f   MSVCRT:MSVCR120.dll
 0001:000055b2       __unlock                   100065b2 f   MSVCRT:MSVCR120.dll
 0001:000055b8       __calloc_crt               100065b8 f   MSVCRT:MSVCR120.dll
 0001:000055be       ___dllonexit               100065be f   MSVCRT:MSVCR120.dll
 0001:000055d0       __SEH_prolog4              100065d0 f   MSVCRT:sehprolg4.obj
 0001:00005615       __SEH_epilog4              10006615 f   MSVCRT:sehprolg4.obj
 0001:00005629       __except_handler4          10006629 f   MSVCRT:chandler4gs.obj
 0001:0000564c       ___raise_securityfailure   1000664c f   MSVCRT:gs_report.obj
 0001:00005689       ___report_gsfailure        10006689 f   MSVCRT:gs_report.obj
 0001:00005784       ___report_rangecheckfailure 10006784 f   MSVCRT:gs_report.obj
 0001:00005790       ___report_securityfailure  10006790 f   MSVCRT:gs_report.obj
 0001:00005860       ___report_securityfailureEx 10006860 f   MSVCRT:gs_report.obj
 0001:00005976       ??_M@YGXPAXIHP6EX0@Z@Z     10006976 f   MSVCRT:ehvecdtr.obj
 0001:000059fe       ?__ArrayUnwind@@YGXPAXIHP6EX0@Z@Z 100069fe f   MSVCRT:ehvecdtr.obj
 0001:00005a5c       ??1type_info@@UAE@XZ       10006a5c f   MSVCRT:MSVCR120.dll
 0001:00005a62       ___CppXcptFilter           10006a62 f   MSVCRT:MSVCR120.dll
 0001:00005a68       __amsg_exit                10006a68 f   MSVCRT:MSVCR120.dll
 0001:00005a70       __FindPESection            10006a70 f   MSVCRT:pesect.obj
 0001:00005ac0       __IsNonwritableInCurrentImage 10006ac0 f   MSVCRT:pesect.obj
 0001:00005b80       __ValidateImageBase        10006b80 f   MSVCRT:pesect.obj
 0001:00005bb2       _free                      10006bb2 f   MSVCRT:MSVCR120.dll
 0001:00005bb8       ___security_init_cookie    10006bb8 f   MSVCRT:gs_support.obj
 0001:00005c54       _DllMain@12                10006c54 f   MSVCRT:dllmain.obj
 0001:00005c76       __malloc_crt               10006c76 f   MSVCRT:MSVCR120.dll
 0001:00005c7c       __RTC_Initialize           10006c7c f   MSVCRT:initsect.obj
 0001:00005c9c       __RTC_Terminate            10006c9c f   MSVCRT:initsect.obj
 0001:00005cbc       __initterm                 10006cbc f   MSVCRT:MSVCR120.dll
 0001:00005cc2       __initterm_e               10006cc2 f   MSVCRT:MSVCR120.dll
 0001:00005cc8       ___clean_type_info_names   10006cc8 f   MSVCRT:tncleanup.obj
 0001:00005cd4       __except_handler4_common   10006cd4 f   MSVCRT:MSVCR120.dll
 0001:00005cda       __crt_debugger_hook        10006cda f   MSVCRT:MSVCR120.dll
 0001:00005ce0       ___crtUnhandledException   10006ce0 f   MSVCRT:MSVCR120.dll
 0001:00005ce6       ___crtTerminateProcess     10006ce6 f   MSVCRT:MSVCR120.dll
 0001:00005cec       ?terminate@@YAXXZ          10006cec f   MSVCRT:MSVCR120.dll
 0001:00005cf2       ___clean_type_info_names_internal 10006cf2 f   MSVCRT:MSVCR120.dll
 0001:00005cf8       _EncodePointer@4           10006cf8 f   kernel32:KERNEL32.dll
 0001:00005cfe       _DecodePointer@4           10006cfe f   kernel32:KERNEL32.dll
 0001:00005d04       _IsDebuggerPresent@0       10006d04 f   kernel32:KERNEL32.dll
 0001:00005d0a       _IsProcessorFeaturePresent@4 10006d0a f   kernel32:KERNEL32.dll
 0001:00005d10       _QueryPerformanceCounter@4 10006d10 f   kernel32:KERNEL32.dll
 0001:00005d16       _GetCurrentProcessId@0     10006d16 f   kernel32:KERNEL32.dll
 0001:00005d1c       _GetCurrentThreadId@0      10006d1c f   kernel32:KERNEL32.dll
 0001:00005d22       _GetSystemTimeAsFileTime@4 10006d22 f   kernel32:KERNEL32.dll
 0001:00005d28       _DisableThreadLibraryCalls@4 10006d28 f   kernel32:KERNEL32.dll
 0002:00000000       __imp__DisableThreadLibraryCalls@4 10008000     kernel32:KERNEL32.dll
 0002:00000004       __imp__GetSystemTimeAsFileTime@4 10008004     kernel32:KERNEL32.dll
 0002:00000008       __imp__GetCurrentThreadId@0 10008008     kernel32:KERNEL32.dll
 0002:0000000c       __imp__GetCurrentProcessId@0 1000800c     kernel32:KERNEL32.dll
 0002:00000010       __imp__QueryPerformanceCounter@4 10008010     kernel32:KERNEL32.dll
 0002:00000014       __imp__IsProcessorFeaturePresent@4 10008014     kernel32:KERNEL32.dll
 0002:00000018       __imp__IsDebuggerPresent@0 10008018     kernel32:KERNEL32.dll
 0002:0000001c       __imp__DecodePointer@4     1000801c     kernel32:KERNEL32.dll
 0002:00000020       __imp__EncodePointer@4     10008020     kernel32:KERNEL32.dll
 0002:00000024       \177KERNEL32_NULL_THUNK_DATA 10008024     kernel32:KERNEL32.dll
 0002:00000028       __imp_?_Xbad_alloc@std@@YAXXZ 10008028     msvcprt:MSVCP120.dll
 0002:0000002c       __imp_?_Xlength_error@std@@YAXPBD@Z 1000802c     msvcprt:MSVCP120.dll
 0002:00000030       __imp_?_Xout_of_range@std@@YAXPBD@Z 10008030     msvcprt:MSVCP120.dll
 0002:00000034       __imp_?_Syserror_map@std@@YAPBDH@Z 10008034     msvcprt:MSVCP120.dll
 0002:00000038       __imp_?_Winerror_map@std@@YAPBDH@Z 10008038     msvcprt:MSVCP120.dll
 0002:0000003c       \177MSVCP120_NULL_THUNK_DATA 1000803c     msvcprt:MSVCP120.dll
 0002:00000040       __imp___initterm_e         10008040     MSVCRT:MSVCR120.dll
 0002:00000044       __imp___initterm           10008044     MSVCRT:MSVCR120.dll
 0002:00000048       __imp___malloc_crt         10008048     MSVCRT:MSVCR120.dll
 0002:0000004c       __imp__free                1000804c     MSVCRT:MSVCR120.dll
 0002:00000050       __imp___amsg_exit          10008050     MSVCRT:MSVCR120.dll
 0002:00000054       __imp____CppXcptFilter     10008054     MSVCRT:MSVCR120.dll
 0002:00000058       __imp_??1type_info@@UAE@XZ 10008058     MSVCRT:MSVCR120.dll
 0002:0000005c       __imp___onexit             1000805c     MSVCRT:MSVCR120.dll
 0002:00000060       __imp____dllonexit         10008060     MSVCRT:MSVCR120.dll
 0002:00000064       __imp___calloc_crt         10008064     MSVCRT:MSVCR120.dll
 0002:00000068       __imp___unlock             10008068     MSVCRT:MSVCR120.dll
 0002:0000006c       __imp___lock               1000806c     MSVCRT:MSVCR120.dll
 0002:00000070       __imp__memset              10008070     MSVCRT:MSVCR120.dll
 0002:00000074       __imp____RTDynamicCast     10008074     MSVCRT:MSVCR120.dll
 0002:00000078       __imp__memcpy              10008078     MSVCRT:MSVCR120.dll
 0002:0000007c       __imp____CxxFrameHandler3  1000807c     MSVCRT:MSVCR120.dll
 0002:00000080       __imp___CxxThrowException@8 10008080     MSVCRT:MSVCR120.dll
 0002:00000084       __imp___hypot              10008084     MSVCRT:MSVCR120.dll
 0002:00000088       __imp__memmove             10008088     MSVCRT:MSVCR120.dll
 0002:0000008c       __imp_??3@YAXPAX@Z         1000808c     MSVCRT:MSVCR120.dll
 0002:00000090       __imp_??2@YAPAXI@Z         10008090     MSVCRT:MSVCR120.dll
 0002:00000094       __imp___purecall           10008094     MSVCRT:MSVCR120.dll
 0002:00000098       __imp___except_handler4_common 10008098     MSVCRT:MSVCR120.dll
 0002:0000009c       __imp___crt_debugger_hook  1000809c     MSVCRT:MSVCR120.dll
 0002:000000a0       __imp____crtUnhandledException 100080a0     MSVCRT:MSVCR120.dll
 0002:000000a4       __imp____crtTerminateProcess 100080a4     MSVCRT:MSVCR120.dll
 0002:000000a8       __imp_?terminate@@YAXXZ    100080a8     MSVCRT:MSVCR120.dll
 0002:000000ac       __imp____clean_type_info_names_internal 100080ac     MSVCRT:MSVCR120.dll
 0002:000000b0       \177MSVCR120_NULL_THUNK_DATA 100080b0     MSVCRT:MSVCR120.dll
 0002:000000b4       __imp_?shared_null@QArrayData@@2QBU1@B 100080b4     Qt5Core:Qt5Core.dll
 0002:000000b8       __imp_??1QObject@@UAE@XZ   100080b8     Qt5Core:Qt5Core.dll
 0002:000000bc       __imp_??0QObject@@QAE@PAV0@@Z 100080bc     Qt5Core:Qt5Core.dll
 0002:000000c0       __imp_?number@QString@@SA?AV1@_KH@Z 100080c0     Qt5Core:Qt5Core.dll
 0002:000000c4       __imp_?deallocate@QArrayData@@SAXPAU1@II@Z 100080c4     Qt5Core:Qt5Core.dll
 0002:000000c8       __imp_?allocate@QArrayData@@SAPAU1@IIIV?$QFlags@W4AllocationOption@QArrayData@@@@@Z 100080c8     Qt5Core:Qt5Core.dll
 0002:000000cc       __imp_?data@QArrayData@@QAEPAXXZ 100080cc     Qt5Core:Qt5Core.dll
 0002:000000d0       __imp_?cast@QMetaObject@@QBEPAVQObject@@PAV2@@Z 100080d0     Qt5Core:Qt5Core.dll
 0002:000000d4       __imp_?qBadAlloc@@YAXXZ    100080d4     Qt5Core:Qt5Core.dll
 0002:000000d8       __imp_?shared_null@QListData@@2UData@1@B 100080d8     Qt5Core:Qt5Core.dll
 0002:000000dc       __imp_?timerEvent@QObject@@MAEXPAVQTimerEvent@@@Z 100080dc     Qt5Core:Qt5Core.dll
 0002:000000e0       __imp_?dynamicMetaObject@QObjectData@@QBEPAUQMetaObject@@XZ 100080e0     Qt5Core:Qt5Core.dll
 0002:000000e4       __imp_?event@QObject@@UAE_NPAVQEvent@@@Z 100080e4     Qt5Core:Qt5Core.dll
 0002:000000e8       __imp_?disconnectNotify@QObject@@MAEXABVQMetaMethod@@@Z 100080e8     Qt5Core:Qt5Core.dll
 0002:000000ec       __imp_?customEvent@QObject@@MAEXPAVQEvent@@@Z 100080ec     Qt5Core:Qt5Core.dll
 0002:000000f0       __imp_?connectNotify@QObject@@MAEXABVQMetaMethod@@@Z 100080f0     Qt5Core:Qt5Core.dll
 0002:000000f4       __imp_?childEvent@QObject@@MAEXPAVQChildEvent@@@Z 100080f4     Qt5Core:Qt5Core.dll
 0002:000000f8       __imp_?toBool@QVariant@@QBE_NXZ 100080f8     Qt5Core:Qt5Core.dll
 0002:000000fc       __imp_?isNull@QVariant@@QBE_NXZ 100080fc     Qt5Core:Qt5Core.dll
 0002:00000100       __imp_??1QVariant@@QAE@XZ  10008100     Qt5Core:Qt5Core.dll
 0002:00000104       __imp_??0QVariant@@QAE@XZ  10008104     Qt5Core:Qt5Core.dll
 0002:00000108       __imp_?errorString@QLibrary@@QBE?AVQString@@XZ 10008108     Qt5Core:Qt5Core.dll
 0002:0000010c       __imp_?fileName@QLibrary@@QBE?AVQString@@XZ 1000810c     Qt5Core:Qt5Core.dll
 0002:00000110       __imp_?isLoaded@QLibrary@@QBE_NXZ 10008110     Qt5Core:Qt5Core.dll
 0002:00000114       __imp_?load@QLibrary@@QAE_NXZ 10008114     Qt5Core:Qt5Core.dll
 0002:00000118       __imp_?resolve@QLibrary@@QAEP6AXXZPBD@Z 10008118     Qt5Core:Qt5Core.dll
 0002:0000011c       __imp_??1QLibrary@@UAE@XZ  1000811c     Qt5Core:Qt5Core.dll
 0002:00000120       __imp_??0QLibrary@@QAE@ABVQString@@PAVQObject@@@Z 10008120     Qt5Core:Qt5Core.dll
 0002:00000124       __imp_?append@QListData@@QAEPAPAXXZ 10008124     Qt5Core:Qt5Core.dll
 0002:00000128       __imp_?dispose@QListData@@SAXPAUData@1@@Z 10008128     Qt5Core:Qt5Core.dll
 0002:0000012c       __imp_?detach_grow@QListData@@QAEPAUData@1@PAHH@Z 1000812c     Qt5Core:Qt5Core.dll
 0002:00000130       __imp_?detach@QListData@@QAEPAUData@1@H@Z 10008130     Qt5Core:Qt5Core.dll
 0002:00000134       __imp_?fromAscii_helper@QString@@CAPAU?$QTypedArrayData@G@@PBDH@Z 10008134     Qt5Core:Qt5Core.dll
 0002:00000138       __imp_??4QString@@QAEAAV0@PBD@Z 10008138     Qt5Core:Qt5Core.dll
 0002:0000013c       __imp_??0QString@@QAE@ABVQByteArray@@@Z 1000813c     Qt5Core:Qt5Core.dll
 0002:00000140       __imp_?number@QString@@SA?AV1@HH@Z 10008140     Qt5Core:Qt5Core.dll
 0002:00000144       __imp_?fromUtf8@QString@@SA?AV1@PBDH@Z 10008144     Qt5Core:Qt5Core.dll
 0002:00000148       __imp_?append@QString@@QAEAAV1@ABV1@@Z 10008148     Qt5Core:Qt5Core.dll
 0002:0000014c       __imp_?arg@QString@@QBE?AV1@ABV1@0@Z 1000814c     Qt5Core:Qt5Core.dll
 0002:00000150       __imp_?arg@QString@@QBE?AV1@ABV1@HVQChar@@@Z 10008150     Qt5Core:Qt5Core.dll
 0002:00000154       __imp_??4QString@@QAEAAV0@$$QAV0@@Z 10008154     Qt5Core:Qt5Core.dll
 0002:00000158       __imp_??4QString@@QAEAAV0@ABV0@@Z 10008158     Qt5Core:Qt5Core.dll
 0002:0000015c       __imp_??1QString@@QAE@XZ   1000815c     Qt5Core:Qt5Core.dll
 0002:00000160       __imp_??0QString@@QAE@ABV0@@Z 10008160     Qt5Core:Qt5Core.dll
 0002:00000164       __imp_??0QString@@QAE@XZ   10008164     Qt5Core:Qt5Core.dll
 0002:00000168       __imp_?data@QByteArray@@QAEPADXZ 10008168     Qt5Core:Qt5Core.dll
 0002:0000016c       __imp_??1QByteArray@@QAE@XZ 1000816c     Qt5Core:Qt5Core.dll
 0002:00000170       __imp_??0QByteArray@@QAE@HD@Z 10008170     Qt5Core:Qt5Core.dll
 0002:00000174       __imp_??0QChar@@QAE@UQLatin1Char@@@Z 10008174     Qt5Core:Qt5Core.dll
 0002:00000178       __imp_?tr@QMetaObject@@QBE?AVQString@@PBD0H@Z 10008178     Qt5Core:Qt5Core.dll
 0002:0000017c       __imp_?eventFilter@QObject@@UAE_NPAV1@PAVQEvent@@@Z 1000817c     Qt5Core:Qt5Core.dll
 0002:00000180       \177Qt5Core_NULL_THUNK_DATA 10008180     Qt5Core:Qt5Core.dll
 0002:00000184       __imp_?hideEvent@QWidget@@MAEXPAVQHideEvent@@@Z 10008184     Qt5Widgets:Qt5Widgets.dll
 0002:00000188       __imp_?hitButton@QCheckBox@@MBE_NABVQPoint@@@Z 10008188     Qt5Widgets:Qt5Widgets.dll
 0002:0000018c       __imp_?indexOf@QLayout@@UBEHPAVQWidget@@@Z 1000818c     Qt5Widgets:Qt5Widgets.dll
 0002:00000190       __imp_?initPainter@QWidget@@MBEXPAVQPainter@@@Z 10008190     Qt5Widgets:Qt5Widgets.dll
 0002:00000194       __imp_?inputMethodEvent@QWidget@@MAEXPAVQInputMethodEvent@@@Z 10008194     Qt5Widgets:Qt5Widgets.dll
 0002:00000198       __imp_?inputMethodQuery@QWidget@@UBE?AVQVariant@@W4InputMethodQuery@Qt@@@Z 10008198     Qt5Widgets:Qt5Widgets.dll
 0002:0000019c       __imp_?invalidate@QBoxLayout@@UAEXXZ 1000819c     Qt5Widgets:Qt5Widgets.dll
 0002:000001a0       __imp_?isEmpty@QLayout@@UBE_NXZ 100081a0     Qt5Widgets:Qt5Widgets.dll
 0002:000001a4       __imp_?itemAt@QBoxLayout@@UBEPAVQLayoutItem@@H@Z 100081a4     Qt5Widgets:Qt5Widgets.dll
 0002:000001a8       __imp_?keyPressEvent@QAbstractButton@@MAEXPAVQKeyEvent@@@Z 100081a8     Qt5Widgets:Qt5Widgets.dll
 0002:000001ac       __imp_?keyPressEvent@QLabel@@MAEXPAVQKeyEvent@@@Z 100081ac     Qt5Widgets:Qt5Widgets.dll
 0002:000001b0       __imp_?keyPressEvent@QWidget@@MAEXPAVQKeyEvent@@@Z 100081b0     Qt5Widgets:Qt5Widgets.dll
 0002:000001b4       __imp_?heightForWidth@QWidget@@UBEHH@Z 100081b4     Qt5Widgets:Qt5Widgets.dll
 0002:000001b8       __imp_?keyReleaseEvent@QWidget@@MAEXPAVQKeyEvent@@@Z 100081b8     Qt5Widgets:Qt5Widgets.dll
 0002:000001bc       __imp_?layout@QLayout@@UAEPAV1@XZ 100081bc     Qt5Widgets:Qt5Widgets.dll
 0002:000001c0       __imp_?leaveEvent@QWidget@@MAEXPAVQEvent@@@Z 100081c0     Qt5Widgets:Qt5Widgets.dll
 0002:000001c4       __imp_?maximumSize@QBoxLayout@@UBE?AVQSize@@XZ 100081c4     Qt5Widgets:Qt5Widgets.dll
 0002:000001c8       __imp_?metaObject@QCheckBox@@UBEPBUQMetaObject@@XZ 100081c8     Qt5Widgets:Qt5Widgets.dll
 0002:000001cc       __imp_?metaObject@QHBoxLayout@@UBEPBUQMetaObject@@XZ 100081cc     Qt5Widgets:Qt5Widgets.dll
 0002:000001d0       __imp_?metaObject@QLabel@@UBEPBUQMetaObject@@XZ 100081d0     Qt5Widgets:Qt5Widgets.dll
 0002:000001d4       __imp_?heightForWidth@QLabel@@UBEHH@Z 100081d4     Qt5Widgets:Qt5Widgets.dll
 0002:000001d8       __imp_?metric@QWidget@@MBEHW4PaintDeviceMetric@QPaintDevice@@@Z 100081d8     Qt5Widgets:Qt5Widgets.dll
 0002:000001dc       __imp_?minimumHeightForWidth@QBoxLayout@@UBEHH@Z 100081dc     Qt5Widgets:Qt5Widgets.dll
 0002:000001e0       __imp_?minimumSize@QBoxLayout@@UBE?AVQSize@@XZ 100081e0     Qt5Widgets:Qt5Widgets.dll
 0002:000001e4       __imp_?minimumSizeHint@QCheckBox@@UBE?AVQSize@@XZ 100081e4     Qt5Widgets:Qt5Widgets.dll
 0002:000001e8       __imp_?minimumSizeHint@QLabel@@UBE?AVQSize@@XZ 100081e8     Qt5Widgets:Qt5Widgets.dll
 0002:000001ec       __imp_?minimumSizeHint@QWidget@@UBE?AVQSize@@XZ 100081ec     Qt5Widgets:Qt5Widgets.dll
 0002:000001f0       __imp_?mouseDoubleClickEvent@QWidget@@MAEXPAVQMouseEvent@@@Z 100081f0     Qt5Widgets:Qt5Widgets.dll
 0002:000001f4       __imp_?mouseMoveEvent@QCheckBox@@MAEXPAVQMouseEvent@@@Z 100081f4     Qt5Widgets:Qt5Widgets.dll
 0002:000001f8       __imp_?mouseMoveEvent@QLabel@@MAEXPAVQMouseEvent@@@Z 100081f8     Qt5Widgets:Qt5Widgets.dll
 0002:000001fc       __imp_?mouseMoveEvent@QWidget@@MAEXPAVQMouseEvent@@@Z 100081fc     Qt5Widgets:Qt5Widgets.dll
 0002:00000200       __imp_?mousePressEvent@QAbstractButton@@MAEXPAVQMouseEvent@@@Z 10008200     Qt5Widgets:Qt5Widgets.dll
 0002:00000204       __imp_?mousePressEvent@QLabel@@MAEXPAVQMouseEvent@@@Z 10008204     Qt5Widgets:Qt5Widgets.dll
 0002:00000208       __imp_?mousePressEvent@QWidget@@MAEXPAVQMouseEvent@@@Z 10008208     Qt5Widgets:Qt5Widgets.dll
 0002:0000020c       __imp_?mouseReleaseEvent@QAbstractButton@@MAEXPAVQMouseEvent@@@Z 1000820c     Qt5Widgets:Qt5Widgets.dll
 0002:00000210       __imp_?mouseReleaseEvent@QLabel@@MAEXPAVQMouseEvent@@@Z 10008210     Qt5Widgets:Qt5Widgets.dll
 0002:00000214       __imp_?mouseReleaseEvent@QWidget@@MAEXPAVQMouseEvent@@@Z 10008214     Qt5Widgets:Qt5Widgets.dll
 0002:00000218       __imp_?moveEvent@QWidget@@MAEXPAVQMoveEvent@@@Z 10008218     Qt5Widgets:Qt5Widgets.dll
 0002:0000021c       __imp_?nativeEvent@QWidget@@MAE_NABVQByteArray@@PAXPAJ@Z 1000821c     Qt5Widgets:Qt5Widgets.dll
 0002:00000220       __imp_?nextCheckState@QCheckBox@@MAEXXZ 10008220     Qt5Widgets:Qt5Widgets.dll
 0002:00000224       __imp_?paintEngine@QWidget@@UBEPAVQPaintEngine@@XZ 10008224     Qt5Widgets:Qt5Widgets.dll
 0002:00000228       __imp_?paintEvent@QCheckBox@@MAEXPAVQPaintEvent@@@Z 10008228     Qt5Widgets:Qt5Widgets.dll
 0002:0000022c       __imp_?paintEvent@QLabel@@MAEXPAVQPaintEvent@@@Z 1000822c     Qt5Widgets:Qt5Widgets.dll
 0002:00000230       __imp_?paintEvent@QWidget@@MAEXPAVQPaintEvent@@@Z 10008230     Qt5Widgets:Qt5Widgets.dll
 0002:00000234       __imp_?qt_metacall@QCheckBox@@UAEHW4Call@QMetaObject@@HPAPAX@Z 10008234     Qt5Widgets:Qt5Widgets.dll
 0002:00000238       __imp_?qt_metacall@QHBoxLayout@@UAEHW4Call@QMetaObject@@HPAPAX@Z 10008238     Qt5Widgets:Qt5Widgets.dll
 0002:0000023c       __imp_?qt_metacall@QLabel@@UAEHW4Call@QMetaObject@@HPAPAX@Z 1000823c     Qt5Widgets:Qt5Widgets.dll
 0002:00000240       __imp_?qt_metacall@QVBoxLayout@@UAEHW4Call@QMetaObject@@HPAPAX@Z 10008240     Qt5Widgets:Qt5Widgets.dll
 0002:00000244       __imp_?qt_metacast@QCheckBox@@UAEPAXPBD@Z 10008244     Qt5Widgets:Qt5Widgets.dll
 0002:00000248       __imp_?qt_metacast@QHBoxLayout@@UAEPAXPBD@Z 10008248     Qt5Widgets:Qt5Widgets.dll
 0002:0000024c       __imp_?qt_metacast@QLabel@@UAEPAXPBD@Z 1000824c     Qt5Widgets:Qt5Widgets.dll
 0002:00000250       __imp_?qt_metacast@QVBoxLayout@@UAEPAXPBD@Z 10008250     Qt5Widgets:Qt5Widgets.dll
 0002:00000254       __imp_?redirected@QWidget@@MBEPAVQPaintDevice@@PAVQPoint@@@Z 10008254     Qt5Widgets:Qt5Widgets.dll
 0002:00000258       __imp_?resizeEvent@QWidget@@MAEXPAVQResizeEvent@@@Z 10008258     Qt5Widgets:Qt5Widgets.dll
 0002:0000025c       __imp_?setGeometry@QBoxLayout@@UAEXABVQRect@@@Z 1000825c     Qt5Widgets:Qt5Widgets.dll
 0002:00000260       __imp_?setVisible@QWidget@@UAEX_N@Z 10008260     Qt5Widgets:Qt5Widgets.dll
 0002:00000264       __imp_?sharedPainter@QWidget@@MBEPAVQPainter@@XZ 10008264     Qt5Widgets:Qt5Widgets.dll
 0002:00000268       __imp_?showEvent@QWidget@@MAEXPAVQShowEvent@@@Z 10008268     Qt5Widgets:Qt5Widgets.dll
 0002:0000026c       __imp_?sizeHint@QBoxLayout@@UBE?AVQSize@@XZ 1000826c     Qt5Widgets:Qt5Widgets.dll
 0002:00000270       __imp_?sizeHint@QCheckBox@@UBE?AVQSize@@XZ 10008270     Qt5Widgets:Qt5Widgets.dll
 0002:00000274       __imp_?sizeHint@QLabel@@UBE?AVQSize@@XZ 10008274     Qt5Widgets:Qt5Widgets.dll
 0002:00000278       __imp_?sizeHint@QWidget@@UBE?AVQSize@@XZ 10008278     Qt5Widgets:Qt5Widgets.dll
 0002:0000027c       __imp_?spacerItem@QLayoutItem@@UAEPAVQSpacerItem@@XZ 1000827c     Qt5Widgets:Qt5Widgets.dll
 0002:00000280       __imp_?tabletEvent@QWidget@@MAEXPAVQTabletEvent@@@Z 10008280     Qt5Widgets:Qt5Widgets.dll
 0002:00000284       __imp_?takeAt@QBoxLayout@@UAEPAVQLayoutItem@@H@Z 10008284     Qt5Widgets:Qt5Widgets.dll
 0002:00000288       __imp_?timerEvent@QAbstractButton@@MAEXPAVQTimerEvent@@@Z 10008288     Qt5Widgets:Qt5Widgets.dll
 0002:0000028c       __imp_?wheelEvent@QWidget@@MAEXPAVQWheelEvent@@@Z 1000828c     Qt5Widgets:Qt5Widgets.dll
 0002:00000290       __imp_?widget@QLayoutItem@@UAEPAVQWidget@@XZ 10008290     Qt5Widgets:Qt5Widgets.dll
 0002:00000294       __imp_?heightForWidth@QBoxLayout@@UBEHH@Z 10008294     Qt5Widgets:Qt5Widgets.dll
 0002:00000298       __imp_?hasHeightForWidth@QWidget@@UBE_NXZ 10008298     Qt5Widgets:Qt5Widgets.dll
 0002:0000029c       __imp_?hasHeightForWidth@QBoxLayout@@UBE_NXZ 1000829c     Qt5Widgets:Qt5Widgets.dll
 0002:000002a0       __imp_?geometry@QLayout@@UBE?AVQRect@@XZ 100082a0     Qt5Widgets:Qt5Widgets.dll
 0002:000002a4       __imp_?focusOutEvent@QWidget@@MAEXPAVQFocusEvent@@@Z 100082a4     Qt5Widgets:Qt5Widgets.dll
 0002:000002a8       __imp_?focusOutEvent@QLabel@@MAEXPAVQFocusEvent@@@Z 100082a8     Qt5Widgets:Qt5Widgets.dll
 0002:000002ac       __imp_?focusOutEvent@QAbstractButton@@MAEXPAVQFocusEvent@@@Z 100082ac     Qt5Widgets:Qt5Widgets.dll
 0002:000002b0       __imp_?focusNextPrevChild@QWidget@@MAE_N_N@Z 100082b0     Qt5Widgets:Qt5Widgets.dll
 0002:000002b4       __imp_?focusNextPrevChild@QLabel@@MAE_N_N@Z 100082b4     Qt5Widgets:Qt5Widgets.dll
 0002:000002b8       __imp_?focusInEvent@QWidget@@MAEXPAVQFocusEvent@@@Z 100082b8     Qt5Widgets:Qt5Widgets.dll
 0002:000002bc       __imp_?focusInEvent@QLabel@@MAEXPAVQFocusEvent@@@Z 100082bc     Qt5Widgets:Qt5Widgets.dll
 0002:000002c0       __imp_?focusInEvent@QAbstractButton@@MAEXPAVQFocusEvent@@@Z 100082c0     Qt5Widgets:Qt5Widgets.dll
 0002:000002c4       __imp_?expandingDirections@QBoxLayout@@UBE?AV?$QFlags@W4Orientation@Qt@@@@XZ 100082c4     Qt5Widgets:Qt5Widgets.dll
 0002:000002c8       __imp_?event@QWidget@@MAE_NPAVQEvent@@@Z 100082c8     Qt5Widgets:Qt5Widgets.dll
 0002:000002cc       __imp_?event@QLabel@@MAE_NPAVQEvent@@@Z 100082cc     Qt5Widgets:Qt5Widgets.dll
 0002:000002d0       __imp_?event@QCheckBox@@MAE_NPAVQEvent@@@Z 100082d0     Qt5Widgets:Qt5Widgets.dll
 0002:000002d4       __imp_?enterEvent@QWidget@@MAEXPAVQEvent@@@Z 100082d4     Qt5Widgets:Qt5Widgets.dll
 0002:000002d8       __imp_?dropEvent@QWidget@@MAEXPAVQDropEvent@@@Z 100082d8     Qt5Widgets:Qt5Widgets.dll
 0002:000002dc       __imp_?dragMoveEvent@QWidget@@MAEXPAVQDragMoveEvent@@@Z 100082dc     Qt5Widgets:Qt5Widgets.dll
 0002:000002e0       __imp_?dragLeaveEvent@QWidget@@MAEXPAVQDragLeaveEvent@@@Z 100082e0     Qt5Widgets:Qt5Widgets.dll
 0002:000002e4       __imp_?dragEnterEvent@QWidget@@MAEXPAVQDragEnterEvent@@@Z 100082e4     Qt5Widgets:Qt5Widgets.dll
 0002:000002e8       __imp_?devType@QWidget@@UBEHXZ 100082e8     Qt5Widgets:Qt5Widgets.dll
 0002:000002ec       __imp_?count@QBoxLayout@@UBEHXZ 100082ec     Qt5Widgets:Qt5Widgets.dll
 0002:000002f0       __imp_?controlTypes@QLayout@@UBE?AV?$QFlags@W4ControlType@QSizePolicy@@@@XZ 100082f0     Qt5Widgets:Qt5Widgets.dll
 0002:000002f4       __imp_?contextMenuEvent@QWidget@@MAEXPAVQContextMenuEvent@@@Z 100082f4     Qt5Widgets:Qt5Widgets.dll
 0002:000002f8       __imp_?contextMenuEvent@QLabel@@MAEXPAVQContextMenuEvent@@@Z 100082f8     Qt5Widgets:Qt5Widgets.dll
 0002:000002fc       __imp_?closeEvent@QWidget@@MAEXPAVQCloseEvent@@@Z 100082fc     Qt5Widgets:Qt5Widgets.dll
 0002:00000300       __imp_?childEvent@QLayout@@MAEXPAVQChildEvent@@@Z 10008300     Qt5Widgets:Qt5Widgets.dll
 0002:00000304       __imp_?checkStateSet@QCheckBox@@MAEXXZ 10008304     Qt5Widgets:Qt5Widgets.dll
 0002:00000308       __imp_?changeEvent@QWidget@@MAEXPAVQEvent@@@Z 10008308     Qt5Widgets:Qt5Widgets.dll
 0002:0000030c       __imp_?changeEvent@QLabel@@MAEXPAVQEvent@@@Z 1000830c     Qt5Widgets:Qt5Widgets.dll
 0002:00000310       __imp_?changeEvent@QAbstractButton@@MAEXPAVQEvent@@@Z 10008310     Qt5Widgets:Qt5Widgets.dll
 0002:00000314       __imp_?addItem@QBoxLayout@@UAEXPAVQLayoutItem@@@Z 10008314     Qt5Widgets:Qt5Widgets.dll
 0002:00000318       __imp_?actionEvent@QWidget@@MAEXPAVQActionEvent@@@Z 10008318     Qt5Widgets:Qt5Widgets.dll
 0002:0000031c       __imp_??1QCheckBox@@UAE@XZ 1000831c     Qt5Widgets:Qt5Widgets.dll
 0002:00000320       __imp_??0QCheckBox@@QAE@ABVQString@@PAVQWidget@@@Z 10008320     Qt5Widgets:Qt5Widgets.dll
 0002:00000324       __imp_?setChecked@QAbstractButton@@QAEX_N@Z 10008324     Qt5Widgets:Qt5Widgets.dll
 0002:00000328       __imp_?isChecked@QAbstractButton@@QBE_NXZ 10008328     Qt5Widgets:Qt5Widgets.dll
 0002:0000032c       __imp_??1QVBoxLayout@@UAE@XZ 1000832c     Qt5Widgets:Qt5Widgets.dll
 0002:00000330       __imp_??0QVBoxLayout@@QAE@PAVQWidget@@@Z 10008330     Qt5Widgets:Qt5Widgets.dll
 0002:00000334       __imp_??1QHBoxLayout@@UAE@XZ 10008334     Qt5Widgets:Qt5Widgets.dll
 0002:00000338       __imp_??0QHBoxLayout@@QAE@PAVQWidget@@@Z 10008338     Qt5Widgets:Qt5Widgets.dll
 0002:0000033c       __imp_?addLayout@QBoxLayout@@QAEXPAVQLayout@@H@Z 1000833c     Qt5Widgets:Qt5Widgets.dll
 0002:00000340       __imp_?addWidget@QBoxLayout@@QAEXPAVQWidget@@HV?$QFlags@W4AlignmentFlag@Qt@@@@@Z 10008340     Qt5Widgets:Qt5Widgets.dll
 0002:00000344       __imp_?addStretch@QBoxLayout@@QAEXH@Z 10008344     Qt5Widgets:Qt5Widgets.dll
 0002:00000348       __imp_?setAlignment@QLayoutItem@@QAEXV?$QFlags@W4AlignmentFlag@Qt@@@@@Z 10008348     Qt5Widgets:Qt5Widgets.dll
 0002:0000034c       __imp_?setAlignment@QLabel@@QAEXV?$QFlags@W4AlignmentFlag@Qt@@@@@Z 1000834c     Qt5Widgets:Qt5Widgets.dll
 0002:00000350       __imp_??1QLabel@@UAE@XZ    10008350     Qt5Widgets:Qt5Widgets.dll
 0002:00000354       __imp_??0QLabel@@QAE@ABVQString@@PAVQWidget@@V?$QFlags@W4WindowType@Qt@@@@@Z 10008354     Qt5Widgets:Qt5Widgets.dll
 0002:00000358       __imp_?setLayout@QWidget@@QAEXPAVQLayout@@@Z 10008358     Qt5Widgets:Qt5Widgets.dll
 0002:0000035c       __imp_??1QWidget@@UAE@XZ   1000835c     Qt5Widgets:Qt5Widgets.dll
 0002:00000360       __imp_?metaObject@QVBoxLayout@@UBEPBUQMetaObject@@XZ 10008360     Qt5Widgets:Qt5Widgets.dll
 0002:00000364       __imp_?keyReleaseEvent@QAbstractButton@@MAEXPAVQKeyEvent@@@Z 10008364     Qt5Widgets:Qt5Widgets.dll
 0002:00000368       \177Qt5Widgets_NULL_THUNK_DATA 10008368     Qt5Widgets:Qt5Widgets.dll
 0002:0000036c       __imp_??0CudaGpuModel@U2@@QAE@ABVQString@@ABH_K_N@Z 1000836c     U2Algorithm:U2Algorithm.dll
 0002:00000370       __imp_?registerCudaGpu@CudaGpuRegistry@U2@@QAEXPAVCudaGpuModel@2@@Z 10008370     U2Algorithm:U2Algorithm.dll
 0002:00000374       __imp_?getRegisteredGpus@CudaGpuRegistry@U2@@QBE?AV?$QList@PAVCudaGpuModel@U2@@@@XZ 10008374     U2Algorithm:U2Algorithm.dll
 0002:00000378       __imp_?getName@CudaGpuModel@U2@@QBE?AVQString@@XZ 10008378     U2Algorithm:U2Algorithm.dll
 0002:0000037c       \177U2Algorithm_NULL_THUNK_DATA 1000837c     U2Algorithm:U2Algorithm.dll
 0002:00000380       __imp_??1Logger@U2@@UAE@XZ 10008380     U2Core:U2Core.dll
 0002:00000384       __imp_?details@Logger@U2@@QAEXABVQString@@@Z 10008384     U2Core:U2Core.dll
 0002:00000388       __imp_??0AppResourceSemaphore@U2@@QAE@HHABVQString@@0@Z 10008388     U2Core:U2Core.dll
 0002:0000038c       __imp_??1AppResourceSemaphore@U2@@UAE@XZ 1000838c     U2Core:U2Core.dll
 0002:00000390       __imp_??0Logger@U2@@QAE@ABVQString@@@Z 10008390     U2Core:U2Core.dll
 0002:00000394       __imp_?instance@AppResourcePool@U2@@SAPAV12@XZ 10008394     U2Core:U2Core.dll
 0002:00000398       __imp_??0Plugin@U2@@QAE@ABVQString@@0_NW4PluginState@1@@Z 10008398     U2Core:U2Core.dll
 0002:0000039c       __imp_??1Plugin@U2@@UAE@XZ 1000839c     U2Core:U2Core.dll
 0002:000003a0       __imp_?acquire@AppResourceSemaphore@U2@@UAEXHW4MemoryLockType@AppResource@2@@Z 100083a0     U2Core:U2Core.dll
 0002:000003a4       __imp_?available@AppResourceSemaphore@U2@@UBEHXZ 100083a4     U2Core:U2Core.dll
 0002:000003a8       __imp_?getCudaGpuRegistry@AppContext@U2@@SAPAVCudaGpuRegistry@2@XZ 100083a8     U2Core:U2Core.dll
 0002:000003ac       __imp_?getMainWindow@AppContext@U2@@SAPAVMainWindow@2@XZ 100083ac     U2Core:U2Core.dll
 0002:000003b0       __imp_?getAppSettingsGUI@AppContext@U2@@SAPAVAppSettingsGUI@2@XZ 100083b0     U2Core:U2Core.dll
 0002:000003b4       __imp_?registerResource@AppResourcePool@U2@@QAEXPAVAppResource@2@@Z 100083b4     U2Core:U2Core.dll
 0002:000003b8       __imp_?qt_metacall@Plugin@U2@@UAEHW4Call@QMetaObject@@HPAPAX@Z 100083b8     U2Core:U2Core.dll
 0002:000003bc       __imp_?staticMetaObject@Plugin@U2@@2UQMetaObject@@B 100083bc     U2Core:U2Core.dll
 0002:000003c0       __imp_?getSettings@AppContext@U2@@SAPAVSettings@2@XZ 100083c0     U2Core:U2Core.dll
 0002:000003c4       __imp_?qt_metacast@Plugin@U2@@UAEPAXPBD@Z 100083c4     U2Core:U2Core.dll
 0002:000003c8       __imp_?getResource@AppResourcePool@U2@@QBEPAVAppResource@2@H@Z 100083c8     U2Core:U2Core.dll
 0002:000003cc       __imp_?setMaxUse@AppResourceSemaphore@U2@@QAEXH@Z 100083cc     U2Core:U2Core.dll
 0002:000003d0       __imp_?tryAcquire@AppResourceSemaphore@U2@@UAE_NHW4MemoryLockType@AppResource@2@@Z 100083d0     U2Core:U2Core.dll
 0002:000003d4       __imp_?tryAcquire@AppResourceSemaphore@U2@@UAE_NHHW4MemoryLockType@AppResource@2@@Z 100083d4     U2Core:U2Core.dll
 0002:000003d8       __imp_?release@AppResourceSemaphore@U2@@UAEXHW4MemoryLockType@AppResource@2@@Z 100083d8     U2Core:U2Core.dll
 0002:000003dc       \177U2Core_NULL_THUNK_DATA 100083dc     U2Core:U2Core.dll
 0002:000003e0       __imp_??1AppSettingsGUIPageState@U2@@UAE@XZ 100083e0     U2Gui:U2Gui.dll
 0002:000003e4       __imp_??0AppSettingsGUIPageWidget@U2@@QAE@PAVQWidget@@@Z 100083e4     U2Gui:U2Gui.dll
 0002:000003e8       __imp_??1AppSettingsGUIPageWidget@U2@@UAE@XZ 100083e8     U2Gui:U2Gui.dll
 0002:000003ec       __imp_??0AppSettingsGUIPageController@U2@@QAE@ABVQString@@0PAVQObject@@@Z 100083ec     U2Gui:U2Gui.dll
 0002:000003f0       __imp_??1AppSettingsGUIPageController@U2@@UAE@XZ 100083f0     U2Gui:U2Gui.dll
 0002:000003f4       __imp_?qt_metacast@AppSettingsGUIPageState@U2@@UAEPAXPBD@Z 100083f4     U2Gui:U2Gui.dll
 0002:000003f8       __imp_?qt_metacall@AppSettingsGUIPageState@U2@@UAEHW4Call@QMetaObject@@HPAPAX@Z 100083f8     U2Gui:U2Gui.dll
 0002:000003fc       __imp_?qt_metacast@AppSettingsGUIPageWidget@U2@@UAEPAXPBD@Z 100083fc     U2Gui:U2Gui.dll
 0002:00000400       __imp_?qt_metacall@AppSettingsGUIPageWidget@U2@@UAEHW4Call@QMetaObject@@HPAPAX@Z 10008400     U2Gui:U2Gui.dll
 0002:00000404       __imp_?qt_metacast@AppSettingsGUIPageController@U2@@UAEPAXPBD@Z 10008404     U2Gui:U2Gui.dll
 0002:00000408       __imp_?qt_metacall@AppSettingsGUIPageController@U2@@UAEHW4Call@QMetaObject@@HPAPAX@Z 10008408     U2Gui:U2Gui.dll
 0002:0000040c       __imp_?staticMetaObject@AppSettingsGUIPageState@U2@@2UQMetaObject@@B 1000840c     U2Gui:U2Gui.dll
 0002:00000410       __imp_?staticMetaObject@AppSettingsGUIPageWidget@U2@@2UQMetaObject@@B 10008410     U2Gui:U2Gui.dll
 0002:00000414       __imp_?staticMetaObject@AppSettingsGUIPageController@U2@@2UQMetaObject@@B 10008414     U2Gui:U2Gui.dll
 0002:00000418       \177U2Gui_NULL_THUNK_DATA  10008418     U2Gui:U2Gui.dll
 0002:0000041c       ___xc_a                    1000841c     MSVCRT:cinitexe.obj
 0002:00000488       ___xc_z                    10008488     MSVCRT:cinitexe.obj
 0002:0000048c       ___xi_a                    1000848c     MSVCRT:cinitexe.obj
 0002:00000498       ___xi_z                    10008498     MSVCRT:cinitexe.obj
 0002:000004d8       ??_C@_07LENCIMMC@CudaGpu?$AA@ 100084d8     CudaSupportPlugin.obj
 0002:000004e0       ??_C@_06BGNBMNO@cuInit?$AA@ 100084e0     CudaSupportPlugin.obj
 0002:000004e8       ??_C@_0BB@FHDBPPFB@cuDeviceGetCount?$AA@ 100084e8     CudaSupportPlugin.obj
 0002:000004fc       ??_C@_0M@HNBJNLLN@cuDeviceGet?$AA@ 100084fc     CudaSupportPlugin.obj
 0002:00000508       ??_C@_0BA@OHKMFJNA@cuDeviceGetName?$AA@ 10008508     CudaSupportPlugin.obj
 0002:00000518       ??_C@_0BB@PMLCNFHH@cuDeviceTotalMem?$AA@ 10008518     CudaSupportPlugin.obj
 0002:0000052c       ??_C@_0BG@DJIPABBC@cuDeviceGetProperties?$AA@ 1000852c     CudaSupportPlugin.obj
 0002:00000542       ??_C@_00CNPNBAHC@?$AA@     10008542     CudaSupportPlugin.obj
 0002:00000548       ??_7error_category@std@@6B@ 10008548     CudaSupportPlugin.obj
 0002:00000564       ??_7_Generic_error_category@std@@6B@ 10008564     CudaSupportPlugin.obj
 0002:0000057c       ??_C@_07DCLBNMLN@generic?$AA@ 1000857c     CudaSupportPlugin.obj
 0002:00000584       ??_C@_0O@BFJCFAAK@unknown?5error?$AA@ 10008584     CudaSupportPlugin.obj
 0002:00000598       ??_7_Iostream_error_category@std@@6B@ 10008598     CudaSupportPlugin.obj
 0002:000005b0       ??_C@_08LLGCOLLL@iostream?$AA@ 100085b0     CudaSupportPlugin.obj
 0002:000005bc       ??_C@_0BG@PADBLCHM@iostream?5stream?5error?$AA@ 100085bc     CudaSupportPlugin.obj
 0002:000005d8       ??_7_System_error_category@std@@6B@ 100085d8     CudaSupportPlugin.obj
 0002:000005f0       ??_C@_06FHFOAHML@system?$AA@ 100085f0     CudaSupportPlugin.obj
 0002:000005f8       ??_C@_0L@JLHNEGIN@Algorithms?$AA@ 100085f8     CudaSupportPlugin.obj
 0002:00000604       ??_C@_07PGLPGHFC@Console?$AA@ 10008604     CudaSupportPlugin.obj
 0002:0000060c       ??_C@_0O@BOFHOPCF@Core?5Services?$AA@ 1000860c     CudaSupportPlugin.obj
 0002:0000061c       ??_C@_0N@PPADAKBM@Input?1Output?$AA@ 1000861c     CudaSupportPlugin.obj
 0002:0000062c       ??_C@_0M@KPPBKPKK@Performance?$AA@ 1000862c     CudaSupportPlugin.obj
 0002:00000638       ??_C@_07BFDHHBBI@Scripts?$AA@ 10008638     CudaSupportPlugin.obj
 0002:00000640       ??_C@_05EEGKELMG@Tasks?$AA@ 10008640     CudaSupportPlugin.obj
 0002:00000648       ??_C@_0P@NIIOBHGA@User?5Interface?$AA@ 10008648     CudaSupportPlugin.obj
 0002:00000658       ??_C@_0N@JINCGGMN@User?5Actions?$AA@ 10008658     CudaSupportPlugin.obj
 0002:0000066c       ??_SAppResourceSemaphore@U2@@6B@ 1000866c     CudaSupportPlugin.obj
 0002:00000688       ??_7CudaSupportPlugin@U2@@6B@ 10008688     CudaSupportPlugin.obj
 0002:000006b4       ??_C@_0CN@NKKDJLJA@Utility?5plugin?5for?5CUDA?9enabled?5@ 100086b4     CudaSupportPlugin.obj
 0002:000006e4       ??_C@_0N@CJGGOMGK@CUDA?5Support?$AA@ 100086e4     CudaSupportPlugin.obj
 0002:000006f4       ??_C@_0BM@DCIKBKKJ@No?5CUDA?9enabled?5GPUs?5found?4?$AA@ 100086f4     CudaSupportPlugin.obj
 0002:00000710       ??_C@_0P@LAKHOBEE@Invalid?5device?$AA@ 10008710     CudaSupportPlugin.obj
 0002:00000720       ??_C@_0BO@KFGIBNNB@No?5cuda?9enabled?5devices?5found?$AA@ 10008720     CudaSupportPlugin.obj
 0002:00000740       ??_C@_0O@NIPGCINC@Unknown?5error?$AA@ 10008740     CudaSupportPlugin.obj
 0002:00000750       ??_C@_0JN@HINAMOPG@Cannot?5load?5CUDA?5driver?5dynamic?5@ 10008750     CudaSupportPlugin.obj
 0002:000007f0       ??_C@_0IB@LHOJFDKK@Cannot?5obtain?5needed?5info?5about?5@ 100087f0     CudaSupportPlugin.obj
 0002:00000878       ??_C@_0HG@JAEBHIDI@An?5error?5occurred?5while?5obtainin@ 10008878     CudaSupportPlugin.obj
 0002:000008f0       ??_C@_0BM@LJCGEHBJ@Loading?5CUDA?5driver?5library?$AA@ 100088f0     CudaSupportPlugin.obj
 0002:0000090c       ??_C@_06NFCKJNMM@nvcuda?$AA@ 1000890c     CudaSupportPlugin.obj
 0002:00000914       ??_C@_0DF@PFBMFLDJ@Cannot?5load?5driver?5library?4?5Erro@ 10008914     CudaSupportPlugin.obj
 0002:0000094c       ??_C@_0BC@JHJIFAJM@Initializing?5CUDA?$AA@ 1000894c     CudaSupportPlugin.obj
 0002:00000960       ??_C@_0BH@EKFKEGAP@Cannot?5resolve?5symbol?5?$AA@ 10008960     CudaSupportPlugin.obj
 0002:00000978       ??_C@_0CJ@KHGHIDMD@Obtaining?5number?5of?5CUDA?9enabled@ 10008978     CudaSupportPlugin.obj
 0002:000009a4       ??_C@_0BG@LOINGOKM@Cannot?5resolve?5symbol?$AA@ 100089a4     CudaSupportPlugin.obj
 0002:000009bc       ??_C@_0CJ@CEJJNFKM@Registering?5CUDA?9enabled?5GPU?3?5?$CF1@ 100089bc     CudaSupportPlugin.obj
 0002:000009e8       ??_C@_08BJBLCIEF@?1enabled?$AA@ 100089e8     CudaSupportPlugin.obj
 0002:000009f4       ??_C@_0CA@JCLEACLE@?1cuda_gpu_registry?1gpu_specific?$AA@ 100089f4     CudaSupportPlugin.obj
 0002:00000a14       ??_C@_0BA@JFNIOLAK@string?5too?5long?$AA@ 10008a14     CudaSupportPlugin.obj
 0002:00000a24       ??_C@_0BI@CFPLBAOH@invalid?5string?5position?$AA@ 10008a24     CudaSupportPlugin.obj
 0002:00000a40       ??_C@_0HF@HEMHJLFF@The?5following?5CUDA?9enabled?5GPUs?5@ 10008a40     CudaSupportSettingsController.obj
 0002:00000ab8       ??_C@_0BO@FPJKGMGJ@No?5CUDA?9enabled?5GPU?5detected?4?$AA@ 10008ab8     CudaSupportSettingsController.obj
 0002:00000adc       ??_SQLabel@@6BQObject@@@   10008adc     CudaSupportSettingsController.obj
 0002:00000b94       ??_SQLabel@@6BQPaintDevice@@@ 10008b94     CudaSupportSettingsController.obj
 0002:00000bb4       ??_SQHBoxLayout@@6BQObject@@@ 10008bb4     CudaSupportSettingsController.obj
 0002:00000bfc       ??_SQHBoxLayout@@6BQLayoutItem@@@ 10008bfc     CudaSupportSettingsController.obj
 0002:00000c44       ??_SQVBoxLayout@@6BQObject@@@ 10008c44     CudaSupportSettingsController.obj
 0002:00000c8c       ??_SQVBoxLayout@@6BQLayoutItem@@@ 10008c8c     CudaSupportSettingsController.obj
 0002:00000cd4       ??_SQCheckBox@@6BQObject@@@ 10008cd4     CudaSupportSettingsController.obj
 0002:00000d98       ??_SQCheckBox@@6BQPaintDevice@@@ 10008d98     CudaSupportSettingsController.obj
 0002:00000db8       ??_7CudaSupportSettingsPageController@U2@@6B@ 10008db8     CudaSupportSettingsController.obj
 0002:00000df8       ??_7CudaSupportSettingsPageState@U2@@6B@ 10008df8     CudaSupportSettingsController.obj
 0002:00000e28       ??_7CudaSupportSettingsPageWidget@U2@@6BQObject@@@ 10008e28     CudaSupportSettingsController.obj
 0002:00000ee8       ??_7CudaSupportSettingsPageWidget@U2@@6BQPaintDevice@@@ 10008ee8     CudaSupportSettingsController.obj
 0002:00000f04       ??_C@_03KFINIEDC@css?$AA@  10008f04     CudaSupportSettingsController.obj
 0002:00000f08       ??_C@_04EEKMIOLD@CUDA?$AA@ 10008f08     CudaSupportSettingsController.obj
 0002:00000f10       ??_C@_03DJLKPBKO@444?$AA@  10008f10     CudaSupportSettingsController.obj
 0002:00000f14       ??_C@_03FBAAJIGL@?5Mb?$AA@ 10008f14     CudaSupportSettingsController.obj
 0002:00000f18       ??_C@_01CLKCMJKC@?5?$AA@   10008f18     CudaSupportSettingsController.obj
 0002:000010d4       ?value@?$integral_constant@_N$0A@@std@@2_NB 100090d4     MSVCRT:ti_inst.obj
 0002:000010d5       ?value@?$integral_constant@_N$00@std@@2_NB 100090d5     MSVCRT:ti_inst.obj
 0002:000010dc       ??_7type_info@@6B@         100090dc     MSVCRT:ti_inst.obj
 0002:000010e0       __pDefaultRawDllMain       100090e0     MSVCRT:crtdll.obj
 0002:000010e0       __pRawDllMain              100090e0     MSVCRT:crtdll.obj
 0002:000010ec       ?ProcessDetach@NativeDll@<CrtImplementationDetails>@@0IB 100090ec     MSVCRT:initsect.obj
 0002:000010f0       ?ProcessAttach@NativeDll@<CrtImplementationDetails>@@0IB 100090f0     MSVCRT:initsect.obj
 0002:000010f4       ?ThreadAttach@NativeDll@<CrtImplementationDetails>@@0IB 100090f4     MSVCRT:initsect.obj
 0002:000010f8       ?ThreadDetach@NativeDll@<CrtImplementationDetails>@@0IB 100090f8     MSVCRT:initsect.obj
 0002:000010fc       ?ProcessVerifier@NativeDll@<CrtImplementationDetails>@@0IB 100090fc     MSVCRT:initsect.obj
 0002:00001100       __load_config_used         10009100     MSVCRT:loadcfg.obj
 0002:000011bc       ??_R4error_category@std@@6B@ 100091bc     CudaSupportPlugin.obj
 0002:000011d0       ??_R3error_category@std@@8 100091d0     CudaSupportPlugin.obj
 0002:000011e0       ??_R2error_category@std@@8 100091e0     CudaSupportPlugin.obj
 0002:000011e8       ??_R1A@?0A@EA@error_category@std@@8 100091e8     CudaSupportPlugin.obj
 0002:00001204       ??_R4_Generic_error_category@std@@6B@ 10009204     CudaSupportPlugin.obj
 0002:00001218       ??_R3_Generic_error_category@std@@8 10009218     CudaSupportPlugin.obj
 0002:00001228       ??_R2_Generic_error_category@std@@8 10009228     CudaSupportPlugin.obj
 0002:00001234       ??_R1A@?0A@EA@_Generic_error_category@std@@8 10009234     CudaSupportPlugin.obj
 0002:00001250       ??_R4_Iostream_error_category@std@@6B@ 10009250     CudaSupportPlugin.obj
 0002:00001264       ??_R3_Iostream_error_category@std@@8 10009264     CudaSupportPlugin.obj
 0002:00001274       ??_R2_Iostream_error_category@std@@8 10009274     CudaSupportPlugin.obj
 0002:00001284       ??_R1A@?0A@EA@_Iostream_error_category@std@@8 10009284     CudaSupportPlugin.obj
 0002:000012a0       ??_R4_System_error_category@std@@6B@ 100092a0     CudaSupportPlugin.obj
 0002:000012b4       ??_R3_System_error_category@std@@8 100092b4     CudaSupportPlugin.obj
 0002:000012c4       ??_R2_System_error_category@std@@8 100092c4     CudaSupportPlugin.obj
 0002:000012d4       ??_R1A@?0A@EA@_System_error_category@std@@8 100092d4     CudaSupportPlugin.obj
 0002:000012f0       ??_R4AppResourceSemaphore@U2@@6B@ 100092f0     CudaSupportPlugin.obj
 0002:00001304       ??_R3AppResourceSemaphore@U2@@8 10009304     CudaSupportPlugin.obj
 0002:00001314       ??_R2AppResourceSemaphore@U2@@8 10009314     CudaSupportPlugin.obj
 0002:00001320       ??_R1A@?0A@EA@AppResourceSemaphore@U2@@8 10009320     CudaSupportPlugin.obj
 0002:0000133c       ??_R1A@?0A@EA@AppResource@U2@@8 1000933c     CudaSupportPlugin.obj
 0002:00001358       ??_R3AppResource@U2@@8     10009358     CudaSupportPlugin.obj
 0002:00001368       ??_R2AppResource@U2@@8     10009368     CudaSupportPlugin.obj
 0002:00001370       ??_R4CudaSupportPlugin@U2@@6B@ 10009370     CudaSupportPlugin.obj
 0002:00001384       ??_R3CudaSupportPlugin@U2@@8 10009384     CudaSupportPlugin.obj
 0002:00001394       ??_R2CudaSupportPlugin@U2@@8 10009394     CudaSupportPlugin.obj
 0002:000013a4       ??_R1A@?0A@EA@CudaSupportPlugin@U2@@8 100093a4     CudaSupportPlugin.obj
 0002:000013c0       ??_R1A@?0A@EA@Plugin@U2@@8 100093c0     CudaSupportPlugin.obj
 0002:000013dc       ??_R3Plugin@U2@@8          100093dc     CudaSupportPlugin.obj
 0002:000013ec       ??_R2Plugin@U2@@8          100093ec     CudaSupportPlugin.obj
 0002:000013f8       ??_R1A@?0A@EA@QObject@@8   100093f8     CudaSupportPlugin.obj
 0002:00001414       ??_R3QObject@@8            10009414     CudaSupportPlugin.obj
 0002:00001424       ??_R2QObject@@8            10009424     CudaSupportPlugin.obj
 0002:0000142c       ??_R4QLabel@@6BQObject@@@  1000942c     CudaSupportSettingsController.obj
 0002:00001440       ??_R3QLabel@@8             10009440     CudaSupportSettingsController.obj
 0002:00001450       ??_R2QLabel@@8             10009450     CudaSupportSettingsController.obj
 0002:00001468       ??_R1A@?0A@EA@QLabel@@8    10009468     CudaSupportSettingsController.obj
 0002:00001484       ??_R1A@?0A@EA@QFrame@@8    10009484     CudaSupportSettingsController.obj
 0002:000014a0       ??_R3QFrame@@8             100094a0     CudaSupportSettingsController.obj
 0002:000014b0       ??_R2QFrame@@8             100094b0     CudaSupportSettingsController.obj
 0002:000014c4       ??_R1A@?0A@EA@QWidget@@8   100094c4     CudaSupportSettingsController.obj
 0002:000014e0       ??_R3QWidget@@8            100094e0     CudaSupportSettingsController.obj
 0002:000014f0       ??_R2QWidget@@8            100094f0     CudaSupportSettingsController.obj
 0002:00001500       ??_R17?0A@EA@QPaintDevice@@8 10009500     CudaSupportSettingsController.obj
 0002:0000151c       ??_R3QPaintDevice@@8       1000951c     CudaSupportSettingsController.obj
 0002:0000152c       ??_R2QPaintDevice@@8       1000952c     CudaSupportSettingsController.obj
 0002:00001534       ??_R1A@?0A@EA@QPaintDevice@@8 10009534     CudaSupportSettingsController.obj
 0002:00001550       ??_R4QLabel@@6BQPaintDevice@@@ 10009550     CudaSupportSettingsController.obj
 0002:00001564       ??_R4QHBoxLayout@@6BQObject@@@ 10009564     CudaSupportSettingsController.obj
 0002:00001578       ??_R3QHBoxLayout@@8        10009578     CudaSupportSettingsController.obj
 0002:00001588       ??_R2QHBoxLayout@@8        10009588     CudaSupportSettingsController.obj
 0002:000015a0       ??_R1A@?0A@EA@QHBoxLayout@@8 100095a0     CudaSupportSettingsController.obj
 0002:000015bc       ??_R1A@?0A@EA@QBoxLayout@@8 100095bc     CudaSupportSettingsController.obj
 0002:000015d8       ??_R3QBoxLayout@@8         100095d8     CudaSupportSettingsController.obj
 0002:000015e8       ??_R2QBoxLayout@@8         100095e8     CudaSupportSettingsController.obj
 0002:000015fc       ??_R1A@?0A@EA@QLayout@@8   100095fc     CudaSupportSettingsController.obj
 0002:00001618       ??_R3QLayout@@8            10009618     CudaSupportSettingsController.obj
 0002:00001628       ??_R2QLayout@@8            10009628     CudaSupportSettingsController.obj
 0002:00001638       ??_R17?0A@EA@QLayoutItem@@8 10009638     CudaSupportSettingsController.obj
 0002:00001654       ??_R3QLayoutItem@@8        10009654     CudaSupportSettingsController.obj
 0002:00001664       ??_R2QLayoutItem@@8        10009664     CudaSupportSettingsController.obj
 0002:0000166c       ??_R1A@?0A@EA@QLayoutItem@@8 1000966c     CudaSupportSettingsController.obj
 0002:00001688       ??_R4QHBoxLayout@@6BQLayoutItem@@@ 10009688     CudaSupportSettingsController.obj
 0002:0000169c       ??_R4QVBoxLayout@@6BQObject@@@ 1000969c     CudaSupportSettingsController.obj
 0002:000016b0       ??_R3QVBoxLayout@@8        100096b0     CudaSupportSettingsController.obj
 0002:000016c0       ??_R2QVBoxLayout@@8        100096c0     CudaSupportSettingsController.obj
 0002:000016d8       ??_R1A@?0A@EA@QVBoxLayout@@8 100096d8     CudaSupportSettingsController.obj
 0002:000016f4       ??_R4QVBoxLayout@@6BQLayoutItem@@@ 100096f4     CudaSupportSettingsController.obj
 0002:00001708       ??_R4QCheckBox@@6BQObject@@@ 10009708     CudaSupportSettingsController.obj
 0002:0000171c       ??_R3QCheckBox@@8          1000971c     CudaSupportSettingsController.obj
 0002:0000172c       ??_R2QCheckBox@@8          1000972c     CudaSupportSettingsController.obj
 0002:00001744       ??_R1A@?0A@EA@QCheckBox@@8 10009744     CudaSupportSettingsController.obj
 0002:00001760       ??_R1A@?0A@EA@QAbstractButton@@8 10009760     CudaSupportSettingsController.obj
 0002:0000177c       ??_R3QAbstractButton@@8    1000977c     CudaSupportSettingsController.obj
 0002:0000178c       ??_R2QAbstractButton@@8    1000978c     CudaSupportSettingsController.obj
 0002:000017a0       ??_R4QCheckBox@@6BQPaintDevice@@@ 100097a0     CudaSupportSettingsController.obj
 0002:000017b4       ??_R4CudaSupportSettingsPageController@U2@@6B@ 100097b4     CudaSupportSettingsController.obj
 0002:000017c8       ??_R3CudaSupportSettingsPageController@U2@@8 100097c8     CudaSupportSettingsController.obj
 0002:000017d8       ??_R2CudaSupportSettingsPageController@U2@@8 100097d8     CudaSupportSettingsController.obj
 0002:000017e8       ??_R1A@?0A@EA@CudaSupportSettingsPageController@U2@@8 100097e8     CudaSupportSettingsController.obj
 0002:00001804       ??_R1A@?0A@EA@AppSettingsGUIPageController@U2@@8 10009804     CudaSupportSettingsController.obj
 0002:00001820       ??_R3AppSettingsGUIPageController@U2@@8 10009820     CudaSupportSettingsController.obj
 0002:00001830       ??_R2AppSettingsGUIPageController@U2@@8 10009830     CudaSupportSettingsController.obj
 0002:0000183c       ??_R4CudaSupportSettingsPageState@U2@@6B@ 1000983c     CudaSupportSettingsController.obj
 0002:00001850       ??_R3CudaSupportSettingsPageState@U2@@8 10009850     CudaSupportSettingsController.obj
 0002:00001860       ??_R2CudaSupportSettingsPageState@U2@@8 10009860     CudaSupportSettingsController.obj
 0002:00001870       ??_R1A@?0A@EA@CudaSupportSettingsPageState@U2@@8 10009870     CudaSupportSettingsController.obj
 0002:0000188c       ??_R1A@?0A@EA@AppSettingsGUIPageState@U2@@8 1000988c     CudaSupportSettingsController.obj
 0002:000018a8       ??_R3AppSettingsGUIPageState@U2@@8 100098a8     CudaSupportSettingsController.obj
 0002:000018b8       ??_R2AppSettingsGUIPageState@U2@@8 100098b8     CudaSupportSettingsController.obj
 0002:000018c4       ??_R4CudaSupportSettingsPageWidget@U2@@6BQObject@@@ 100098c4     CudaSupportSettingsController.obj
 0002:000018d8       ??_R3CudaSupportSettingsPageWidget@U2@@8 100098d8     CudaSupportSettingsController.obj
 0002:000018e8       ??_R2CudaSupportSettingsPageWidget@U2@@8 100098e8     CudaSupportSettingsController.obj
 0002:00001900       ??_R1A@?0A@EA@CudaSupportSettingsPageWidget@U2@@8 10009900     CudaSupportSettingsController.obj
 0002:0000191c       ??_R1A@?0A@EA@AppSettingsGUIPageWidget@U2@@8 1000991c     CudaSupportSettingsController.obj
 0002:00001938       ??_R3AppSettingsGUIPageWidget@U2@@8 10009938     CudaSupportSettingsController.obj
 0002:00001948       ??_R2AppSettingsGUIPageWidget@U2@@8 10009948     CudaSupportSettingsController.obj
 0002:0000195c       ??_R4CudaSupportSettingsPageWidget@U2@@6BQPaintDevice@@@ 1000995c     CudaSupportSettingsController.obj
 0002:00001970       ??_R4type_info@@6B@        10009970     MSVCRT:ti_inst.obj
 0002:00001984       ??_R3type_info@@8          10009984     MSVCRT:ti_inst.obj
 0002:00001994       ??_R2type_info@@8          10009994     MSVCRT:ti_inst.obj
 0002:0000199c       ??_R1A@?0A@EA@type_info@@8 1000999c     MSVCRT:ti_inst.obj
 0002:000019c0       ___safe_se_handler_table   100099c0     <linker-defined>
 0002:00001a84       ___rtc_iaa                 10009a84     MSVCRT:initsect.obj
 0002:00001a88       ___rtc_izz                 10009a88     MSVCRT:initsect.obj
 0002:00001a8c       ___rtc_taa                 10009a8c     MSVCRT:initsect.obj
 0002:00001a90       ___rtc_tzz                 10009a90     MSVCRT:initsect.obj
 0002:00002948       __IMPORT_DESCRIPTOR_U2Core 1000a948     U2Core:U2Core.dll
 0002:0000295c       __IMPORT_DESCRIPTOR_U2Algorithm 1000a95c     U2Algorithm:U2Algorithm.dll
 0002:00002970       __IMPORT_DESCRIPTOR_U2Gui  1000a970     U2Gui:U2Gui.dll
 0002:00002984       __IMPORT_DESCRIPTOR_Qt5Widgets 1000a984     Qt5Widgets:Qt5Widgets.dll
 0002:00002998       __IMPORT_DESCRIPTOR_Qt5Core 1000a998     Qt5Core:Qt5Core.dll
 0002:000029ac       __IMPORT_DESCRIPTOR_MSVCP120 1000a9ac     msvcprt:MSVCP120.dll
 0002:000029c0       __IMPORT_DESCRIPTOR_MSVCR120 1000a9c0     MSVCRT:MSVCR120.dll
 0002:000029d4       __IMPORT_DESCRIPTOR_KERNEL32 1000a9d4     kernel32:KERNEL32.dll
 0002:000029e8       __NULL_IMPORT_DESCRIPTOR   1000a9e8     U2Core:U2Core.dll
 0003:0000001c       ?_Generic_object@?$_Error_objects@H@std@@2V_Generic_error_category@2@A 1000e01c     CudaSupportPlugin.obj
 0003:00000020       ?_Iostream_object@?$_Error_objects@H@std@@2V_Iostream_error_category@2@A 1000e020     CudaSupportPlugin.obj
 0003:00000024       ?_System_object@?$_Error_objects@H@std@@2V_System_error_category@2@A 1000e024     CudaSupportPlugin.obj
 0003:00000030       ?staticMetaObject@CudaSupportPlugin@U2@@2UQMetaObject@@B 1000e030     moc_CudaSupportPlugin.obj
 0003:00000048       ?staticMetaObject@CudaSupportSettingsPageController@U2@@2UQMetaObject@@B 1000e048     moc_CudaSupportSettingsController.obj
 0003:00000060       ?staticMetaObject@CudaSupportSettingsPageState@U2@@2UQMetaObject@@B 1000e060     moc_CudaSupportSettingsController.obj
 0003:00000078       ?staticMetaObject@CudaSupportSettingsPageWidget@U2@@2UQMetaObject@@B 1000e078     moc_CudaSupportSettingsController.obj
 0003:00000090       ___security_cookie         1000e090     MSVCRT:gs_cookie.obj
 0003:00000094       ___security_cookie_complement 1000e094     MSVCRT:gs_cookie.obj
 0003:000000a0       ___native_dllmain_reason   1000e0a0     MSVCRT:natstart.obj
 0003:000000a4       ??_R0?AVerror_category@std@@@8 1000e0a4     CudaSupportPlugin.obj
 0003:000000c8       ??_R0?AV_Generic_error_category@std@@@8 1000e0c8     CudaSupportPlugin.obj
 0003:000000f4       ??_R0?AV_Iostream_error_category@std@@@8 1000e0f4     CudaSupportPlugin.obj
 0003:00000120       ??_R0?AV_System_error_category@std@@@8 1000e120     CudaSupportPlugin.obj
 0003:0000014c       ??_R0?AVAppResourceSemaphore@U2@@@8 1000e14c     CudaSupportPlugin.obj
 0003:00000174       ??_R0?AVAppResource@U2@@@8 1000e174     CudaSupportPlugin.obj
 0003:00000194       ??_R0?AVCudaSupportPlugin@U2@@@8 1000e194     CudaSupportPlugin.obj
 0003:000001b8       ??_R0?AVPlugin@U2@@@8      1000e1b8     CudaSupportPlugin.obj
 0003:000001d0       ??_R0?AVQObject@@@8        1000e1d0     CudaSupportPlugin.obj
 0003:000001e8       ??_R0?AVQLabel@@@8         1000e1e8     CudaSupportSettingsController.obj
 0003:00000200       ??_R0?AVQFrame@@@8         1000e200     CudaSupportSettingsController.obj
 0003:00000218       ??_R0?AVQWidget@@@8        1000e218     CudaSupportSettingsController.obj
 0003:00000230       ??_R0?AVQPaintDevice@@@8   1000e230     CudaSupportSettingsController.obj
 0003:0000024c       ??_R0?AVQHBoxLayout@@@8    1000e24c     CudaSupportSettingsController.obj
 0003:00000268       ??_R0?AVQBoxLayout@@@8     1000e268     CudaSupportSettingsController.obj
 0003:00000284       ??_R0?AVQLayout@@@8        1000e284     CudaSupportSettingsController.obj
 0003:0000029c       ??_R0?AVQLayoutItem@@@8    1000e29c     CudaSupportSettingsController.obj
 0003:000002b8       ??_R0?AVQVBoxLayout@@@8    1000e2b8     CudaSupportSettingsController.obj
 0003:000002d4       ??_R0?AVQCheckBox@@@8      1000e2d4     CudaSupportSettingsController.obj
 0003:000002ec       ??_R0?AVQAbstractButton@@@8 1000e2ec     CudaSupportSettingsController.obj
 0003:0000030c       ??_R0?AVCudaSupportSettingsPageController@U2@@@8 1000e30c     CudaSupportSettingsController.obj
 0003:00000340       ??_R0?AVAppSettingsGUIPageController@U2@@@8 1000e340     CudaSupportSettingsController.obj
 0003:00000370       ??_R0?AVCudaSupportSettingsPageState@U2@@@8 1000e370     CudaSupportSettingsController.obj
 0003:000003a0       ??_R0?AVAppSettingsGUIPageState@U2@@@8 1000e3a0     CudaSupportSettingsController.obj
 0003:000003cc       ??_R0?AVCudaSupportSettingsPageWidget@U2@@@8 1000e3cc     CudaSupportSettingsController.obj
 0003:000003fc       ??_R0?AVAppSettingsGUIPageWidget@U2@@@8 1000e3fc     CudaSupportSettingsController.obj
 0003:00000428       ??_R0?AVtype_info@@@8      1000e428     MSVCRT:ti_inst.obj
 0003:0000048c       ?id@?$num_put@DV?$back_insert_iterator@V?$basic_string@DU?$char_traits@D@std@@V?$allocator@D@2@@std@@@std@@@std@@2V0locale@2@A 1000e48c     CudaSupportPlugin.obj
 0003:00000490       ?id@?$num_put@_WV?$back_insert_iterator@V?$basic_string@_WU?$char_traits@_W@std@@V?$allocator@_W@2@@std@@@std@@@std@@2V0locale@2@A 1000e490     CudaSupportPlugin.obj
 0003:000004d0       ?helpPageId@CudaSupportSettingsPageController@U2@@0VQString@@B 1000e4d0     CudaSupportSettingsController.obj
 0003:00000810       ?__type_info_root_node@@3U__type_info_node@@A 1000e810     MSVCRT:tncleanup.obj
 0003:00000818       ___native_startup_lock     1000e818     <common>
 0003:0000081c       ___native_startup_state    1000e81c     <common>
 0003:00000820       ___dyn_tls_init_callback   1000e820     <common>
 0003:00000824       ___onexitend               1000e824     <common>
 0003:00000828       ___onexitbegin             1000e828     <common>

 entry point at        0001:00005456

 Static symbols

 0000:fffee000       .debug$S                   10000000     MSVCRT:MSVCR120.dll
 0000:fffee000       .debug$S                   10000000     MSVCRT:MSVCR120.dll
 0000:fffee000       .debug$S                   10000000     MSVCRT:MSVCR120.dll
 0000:fffee000       .debug$S                   10000000     MSVCRT:MSVCR120.dll
 0000:fffee000       .debug$S                   10000000     MSVCRT:MSVCR120.dll
 0000:fffee000       .debug$S                   10000000     MSVCRT:MSVCR120.dll
 0000:fffee000       .debug$S                   10000000     MSVCRT:MSVCR120.dll
 0000:fffee000       .debug$S                   10000000     MSVCRT:MSVCR120.dll
 0000:fffee000       .debug$S                   10000000     MSVCRT:MSVCR120.dll
 0000:fffee000       .debug$S                   10000000     MSVCRT:MSVCR120.dll
 0000:fffee000       .debug$S                   10000000     MSVCRT:MSVCR120.dll
 0000:fffee000       .debug$S                   10000000     MSVCRT:MSVCR120.dll
 0000:fffee000       .debug$S                   10000000     MSVCRT:MSVCR120.dll
 0000:fffee000       .debug$S                   10000000     U2Core:U2Core.dll
 0000:fffee000       .debug$S                   10000000     U2Core:U2Core.dll
 0000:fffee000       .debug$S                   10000000     U2Core:U2Core.dll
 0000:fffee000       .debug$S                   10000000     U2Core:U2Core.dll
 0000:fffee000       .debug$S                   10000000     MSVCRT:MSVCR120.dll
 0000:fffee000       .debug$S                   10000000     U2Core:U2Core.dll
 0000:fffee000       .debug$S                   10000000     MSVCRT:MSVCR120.dll
 0000:fffee000       .debug$S                   10000000     U2Core:U2Core.dll
 0000:fffee000       .debug$S                   10000000     MSVCRT:MSVCR120.dll
 0001:fffff000       __ehhandler$?_Copy@?$basic_string@DU?$char_traits@D@std@@V?$allocator@D@2@@std@@QAEXII@Z 10000000 f   moc_CudaSupportSettingsController.obj
 0000:fffee000       .debug$S                   10000000     U2Core:U2Core.dll
 0000:fffee000       .debug$S                   10000000     U2Core:U2Core.dll
 0000:fffee000       .debug$S                   10000000     U2Core:U2Core.dll
 0000:fffee000       .debug$S                   10000000     U2Core:U2Core.dll
 0000:fffee000       .debug$S                   10000000     U2Core:U2Core.dll
 0000:fffee000       .debug$S                   10000000     U2Core:U2Core.dll
 0002:ffff8000       __catchsym$?_Copy@?$basic_string@DU?$char_traits@D@std@@V?$allocator@D@2@@std@@QAEXII@Z$5 10000000     moc_CudaSupportSettingsController.obj
 0000:fffee000       .debug$S                   10000000     MSVCRT:MSVCR120.dll
 0000:fffee000       .debug$S                   10000000     MSVCRT:MSVCR120.dll
 0000:fffee000       .debug$S                   10000000     MSVCRT:MSVCR120.dll
 0000:fffee000       .debug$S                   10000000     MSVCRT:MSVCR120.dll
 0000:fffee000       .debug$S                   10000000     MSVCRT:MSVCR120.dll
 0000:fffee000       .debug$S                   10000000     MSVCRT:MSVCR120.dll
 0000:fffee000       .debug$S                   10000000     MSVCRT:MSVCR120.dll
 0002:ffff8000       ?_Generic_object$initializer$@?$_Error_objects@H@std@@2P6AXXZA 10000000     moc_CudaSupportSettingsController.obj
 0002:ffff8000       ?_Iostream_object$initializer$@?$_Error_objects@H@std@@2P6AXXZA 10000000     moc_CudaSupportSettingsController.obj
 0002:ffff8000       ?_System_object$initializer$@?$_Error_objects@H@std@@2P6AXXZA 10000000     moc_CudaSupportSettingsController.obj
 0000:fffee000       .debug$S                   10000000     MSVCRT:MSVCR120.dll
 0000:fffee000       .debug$S                   10000000     MSVCRT:MSVCR120.dll
 0000:fffee000       .debug$S                   10000000     U2Core:U2Core.dll
 0000:fffee000       .debug$S                   10000000     U2Core:U2Core.dll
 0000:fffee000       .debug$S                   10000000     MSVCRT:MSVCR120.dll
 0000:fffee000       .debug$S                   10000000     U2Core:U2Core.dll
 0000:fffee000       .debug$S                   10000000     MSVCRT:MSVCR120.dll
 0000:fffee000       .debug$S                   10000000     U2Core:U2Core.dll
 0000:fffee000       .debug$S                   10000000     MSVCRT:MSVCR120.dll
 0001:fffff000       __ehhandler$?_Copy@?$basic_string@DU?$char_traits@D@std@@V?$allocator@D@2@@std@@QAEXII@Z 10000000 f   moc_CudaSupportPlugin.obj
 0000:fffee000       .debug$S                   10000000     U2Core:U2Core.dll
 0000:fffee000       .debug$S                   10000000     U2Core:U2Core.dll
 0000:fffee000       .debug$S                   10000000     U2Core:U2Core.dll
 0000:fffee000       .debug$S                   10000000     U2Core:U2Core.dll
 0000:fffee000       .debug$S                   10000000     U2Core:U2Core.dll
 0000:fffee000       .debug$S                   10000000     U2Core:U2Core.dll
 0002:ffff8000       __catchsym$?_Copy@?$basic_string@DU?$char_traits@D@std@@V?$allocator@D@2@@std@@QAEXII@Z$5 10000000     moc_CudaSupportPlugin.obj
 0000:fffee000       .debug$S                   10000000     U2Algorithm:U2Algorithm.dll
 0000:fffee000       .debug$S                   10000000     U2Algorithm:U2Algorithm.dll
 0000:fffee000       .debug$S                   10000000     U2Algorithm:U2Algorithm.dll
 0000:fffee000       .debug$S                   10000000     U2Algorithm:U2Algorithm.dll
 0000:fffee000       .debug$S                   10000000     msvcprt:MSVCP120.dll
 0002:ffff8000       ?_Generic_object$initializer$@?$_Error_objects@H@std@@2P6AXXZA 10000000     moc_CudaSupportPlugin.obj
 0002:ffff8000       ?_Iostream_object$initializer$@?$_Error_objects@H@std@@2P6AXXZA 10000000     moc_CudaSupportPlugin.obj
 0002:ffff8000       ?_System_object$initializer$@?$_Error_objects@H@std@@2P6AXXZA 10000000     moc_CudaSupportPlugin.obj
 0000:fffee000       .debug$S                   10000000     msvcprt:MSVCP120.dll
 0000:fffee000       .debug$S                   10000000     msvcprt:MSVCP120.dll
 0000:fffee000       .debug$S                   10000000     U2Gui:U2Gui.dll
 0000:fffee000       .debug$S                   10000000     msvcprt:MSVCP120.dll
 0000:fffee000       .debug$S                   10000000     U2Gui:U2Gui.dll
 0000:fffee000       .debug$S                   10000000     msvcprt:MSVCP120.dll
 0000:fffee000       .debug$S                   10000000     U2Gui:U2Gui.dll
 0000:fffee000       .debug$S                   10000000     kernel32:KERNEL32.dll
 0000:fffee000       .debug$S                   10000000     U2Gui:U2Gui.dll
 0000:fffee000       .debug$S                   10000000     kernel32:KERNEL32.dll
 0000:fffee000       .debug$S                   10000000     U2Gui:U2Gui.dll
 0000:fffee000       .debug$S                   10000000     kernel32:KERNEL32.dll
 0000:fffee000       .debug$S                   10000000     U2Gui:U2Gui.dll
 0000:fffee000       .debug$S                   10000000     kernel32:KERNEL32.dll
 0000:fffee000       .debug$S                   10000000     U2Gui:U2Gui.dll
 0000:fffee000       .debug$S                   10000000     kernel32:KERNEL32.dll
 0000:fffee000       .debug$S                   10000000     U2Gui:U2Gui.dll
 0000:fffee000       .debug$S                   10000000     kernel32:KERNEL32.dll
 0000:fffee000       .debug$S                   10000000     U2Gui:U2Gui.dll
 0000:fffee000       .debug$S                   10000000     kernel32:KERNEL32.dll
 0000:fffee000       .debug$S                   10000000     U2Gui:U2Gui.dll
 0000:fffee000       .debug$S                   10000000     kernel32:KERNEL32.dll
 0000:fffee000       .debug$S                   10000000     U2Gui:U2Gui.dll
 0000:fffee000       .debug$S                   10000000     kernel32:KERNEL32.dll
 0000:fffee000       .debug$S                   10000000     U2Gui:U2Gui.dll
 0000:fffee000       .debug$S                   10000000     Qt5Core:Qt5Core.dll
 0000:fffee000       .debug$S                   10000000     U2Gui:U2Gui.dll
 0000:fffee000       .debug$S                   10000000     Qt5Core:Qt5Core.dll
 0001:fffff000       __ehhandler$?_Copy@?$basic_string@DU?$char_traits@D@std@@V?$allocator@D@2@@std@@QAEXII@Z 10000000 f   CudaSupportSettingsController.obj
 0000:fffee000       .debug$S                   10000000     U2Gui:U2Gui.dll
 0000:fffee000       .debug$S                   10000000     Qt5Widgets:Qt5Widgets.dll
 0000:fffee000       .debug$S                   10000000     Qt5Widgets:Qt5Widgets.dll
 0001:fffff000       __unwindfunclet$??H@YA?BVQString@@ABV0@0@Z$0 10000000 f   CudaSupportSettingsController.obj
 0000:fffee000       .debug$S                   10000000     Qt5Widgets:Qt5Widgets.dll
 0001:fffff000       __unwindfunclet$??H@YA?BVQString@@ABV0@PBD@Z$0 10000000 f   CudaSupportSettingsController.obj
 0000:fffee000       .debug$S                   10000000     Qt5Widgets:Qt5Widgets.dll
 0000:fffee000       .debug$S                   10000000     Qt5Core:Qt5Core.dll
 0000:fffee000       .debug$S                   10000000     Qt5Core:Qt5Core.dll
 0000:fffee000       .debug$S                   10000000     Qt5Core:Qt5Core.dll
 0000:fffee000       .debug$S                   10000000     Qt5Core:Qt5Core.dll
 0000:fffee000       .debug$S                   10000000     Qt5Core:Qt5Core.dll
 0000:fffee000       .debug$S                   10000000     Qt5Core:Qt5Core.dll
 0000:fffee000       .debug$S                   10000000     Qt5Core:Qt5Core.dll
 0000:fffee000       .debug$S                   10000000     Qt5Core:Qt5Core.dll
 0000:fffee000       .debug$S                   10000000     Qt5Core:Qt5Core.dll
 0000:fffee000       .debug$S                   10000000     Qt5Core:Qt5Core.dll
 0000:fffee000       .debug$S                   10000000     Qt5Core:Qt5Core.dll
 0000:fffee000       .debug$S                   10000000     Qt5Core:Qt5Core.dll
 0000:fffee000       .debug$S                   10000000     Qt5Core:Qt5Core.dll
 0000:fffee000       .debug$S                   10000000     Qt5Core:Qt5Core.dll
 0000:fffee000       .debug$S                   10000000     Qt5Core:Qt5Core.dll
 0000:fffee000       .debug$S                   10000000     Qt5Core:Qt5Core.dll
 0000:fffee000       .debug$S                   10000000     Qt5Core:Qt5Core.dll
 0000:fffee000       .debug$S                   10000000     Qt5Core:Qt5Core.dll
 0000:fffee000       .debug$S                   10000000     Qt5Core:Qt5Core.dll
 0000:fffee000       .debug$S                   10000000     Qt5Core:Qt5Core.dll
 0000:fffee000       .debug$S                   10000000     Qt5Core:Qt5Core.dll
 0000:fffee000       .debug$S                   10000000     Qt5Core:Qt5Core.dll
 0000:fffee000       .debug$S                   10000000     Qt5Core:Qt5Core.dll
 0000:fffee000       .debug$S                   10000000     Qt5Core:Qt5Core.dll
 0000:fffee000       .debug$S                   10000000     Qt5Core:Qt5Core.dll
 0000:fffee000       .debug$S                   10000000     Qt5Core:Qt5Core.dll
 0000:fffee000       .debug$S                   10000000     Qt5Core:Qt5Core.dll
 0000:fffee000       .debug$S                   10000000     Qt5Core:Qt5Core.dll
 0000:fffee000       .debug$S                   10000000     Qt5Core:Qt5Core.dll
 0000:fffee000       .debug$S                   10000000     Qt5Core:Qt5Core.dll
 0000:fffee000       .debug$S                   10000000     Qt5Core:Qt5Core.dll
 0000:fffee000       .debug$S                   10000000     Qt5Core:Qt5Core.dll
 0000:fffee000       .debug$S                   10000000     Qt5Core:Qt5Core.dll
 0000:fffee000       .debug$S                   10000000     Qt5Core:Qt5Core.dll
 0000:fffee000       .debug$S                   10000000     Qt5Core:Qt5Core.dll
 0000:fffee000       .debug$S                   10000000     Qt5Core:Qt5Core.dll
 0000:fffee000       .debug$S                   10000000     Qt5Core:Qt5Core.dll
 0000:fffee000       .debug$S                   10000000     Qt5Widgets:Qt5Widgets.dll
 0000:fffee000       .debug$S                   10000000     Qt5Widgets:Qt5Widgets.dll
 0000:fffee000       .debug$S                   10000000     Qt5Core:Qt5Core.dll
 0000:fffee000       .debug$S                   10000000     Qt5Core:Qt5Core.dll
 0000:fffee000       .debug$S                   10000000     Qt5Core:Qt5Core.dll
 0000:fffee000       .debug$S                   10000000     Qt5Core:Qt5Core.dll
 0000:fffee000       .debug$S                   10000000     Qt5Core:Qt5Core.dll
 0000:fffee000       .debug$S                   10000000     Qt5Core:Qt5Core.dll
 0000:fffee000       .debug$S                   10000000     Qt5Core:Qt5Core.dll
 0000:fffee000       .debug$S                   10000000     Qt5Core:Qt5Core.dll
 0000:fffee000       .debug$S                   10000000     Qt5Core:Qt5Core.dll
 0000:fffee000       .debug$S                   10000000     Qt5Core:Qt5Core.dll
 0000:fffee000       .debug$S                   10000000     Qt5Core:Qt5Core.dll
 0000:fffee000       .debug$S                   10000000     Qt5Core:Qt5Core.dll
 0000:fffee000       .debug$S                   10000000     Qt5Widgets:Qt5Widgets.dll
 0000:fffee000       .debug$S                   10000000     Qt5Widgets:Qt5Widgets.dll
 0000:fffee000       .debug$S                   10000000     Qt5Widgets:Qt5Widgets.dll
 0000:fffee000       .debug$S                   10000000     Qt5Widgets:Qt5Widgets.dll
 0000:fffee000       .debug$S                   10000000     Qt5Widgets:Qt5Widgets.dll
 0000:fffee000       .debug$S                   10000000     Qt5Widgets:Qt5Widgets.dll
 0000:fffee000       .debug$S                   10000000     Qt5Widgets:Qt5Widgets.dll
 0000:fffee000       .debug$S                   10000000     Qt5Widgets:Qt5Widgets.dll
 0000:fffee000       .debug$S                   10000000     Qt5Widgets:Qt5Widgets.dll
 0000:fffee000       .debug$S                   10000000     Qt5Widgets:Qt5Widgets.dll
 0000:fffee000       .debug$S                   10000000     Qt5Widgets:Qt5Widgets.dll
 0000:fffee000       .debug$S                   10000000     Qt5Widgets:Qt5Widgets.dll
 0000:fffee000       .debug$S                   10000000     Qt5Widgets:Qt5Widgets.dll
 0000:fffee000       .debug$S                   10000000     Qt5Widgets:Qt5Widgets.dll
 0000:fffee000       .debug$S                   10000000     Qt5Widgets:Qt5Widgets.dll
 0000:fffee000       .debug$S                   10000000     Qt5Widgets:Qt5Widgets.dll
 0000:fffee000       .debug$S                   10000000     Qt5Widgets:Qt5Widgets.dll
 0000:fffee000       .debug$S                   10000000     Qt5Widgets:Qt5Widgets.dll
 0000:fffee000       .debug$S                   10000000     Qt5Widgets:Qt5Widgets.dll
 0000:fffee000       .debug$S                   10000000     Qt5Widgets:Qt5Widgets.dll
 0000:fffee000       .debug$S                   10000000     Qt5Widgets:Qt5Widgets.dll
 0000:fffee000       .debug$S                   10000000     Qt5Widgets:Qt5Widgets.dll
 0000:fffee000       .debug$S                   10000000     Qt5Widgets:Qt5Widgets.dll
 0000:fffee000       .debug$S                   10000000     Qt5Widgets:Qt5Widgets.dll
 0000:fffee000       .debug$S                   10000000     Qt5Widgets:Qt5Widgets.dll
 0001:fffff000       __ehhandler$??0?$QList@PAVCudaGpuModel@U2@@@@QAE@ABV0@@Z 10000000 f   CudaSupportSettingsController.obj
 0000:fffee000       .debug$S                   10000000     Qt5Widgets:Qt5Widgets.dll
 0000:fffee000       .debug$S                   10000000     Qt5Widgets:Qt5Widgets.dll
 0000:fffee000       .debug$S                   10000000     Qt5Widgets:Qt5Widgets.dll
 0000:fffee000       .debug$S                   10000000     Qt5Widgets:Qt5Widgets.dll
 0000:fffee000       .debug$S                   10000000     Qt5Widgets:Qt5Widgets.dll
 0002:ffff8000       ?_System_object$initializer$@?$_Error_objects@H@std@@2P6AXXZA 10000000     CudaSupportSettingsController.obj
 0002:ffff8000       ?_Iostream_object$initializer$@?$_Error_objects@H@std@@2P6AXXZA 10000000     CudaSupportSettingsController.obj
 0002:ffff8000       __catchsym$?_Copy@?$basic_string@DU?$char_traits@D@std@@V?$allocator@D@2@@std@@QAEXII@Z$5 10000000     CudaSupportSettingsController.obj
 0002:ffff8000       ?_Generic_object$initializer$@?$_Error_objects@H@std@@2P6AXXZA 10000000     CudaSupportSettingsController.obj
 0002:ffff8000       __unwindtable$??H@YA?BVQString@@ABV0@0@Z 10000000     CudaSupportSettingsController.obj
 0000:fffee000       .debug$S                   10000000     Qt5Widgets:Qt5Widgets.dll
 0002:ffff8000       __unwindtable$??H@YA?BVQString@@ABV0@PBD@Z 10000000     CudaSupportSettingsController.obj
 0000:fffee000       .debug$S                   10000000     Qt5Widgets:Qt5Widgets.dll
 0000:fffee000       .debug$S                   10000000     Qt5Widgets:Qt5Widgets.dll
 0000:fffee000       .debug$S                   10000000     Qt5Widgets:Qt5Widgets.dll
 0000:fffee000       .debug$S                   10000000     Qt5Widgets:Qt5Widgets.dll
 0000:fffee000       .debug$S                   10000000     Qt5Widgets:Qt5Widgets.dll
 0000:fffee000       .debug$S                   10000000     Qt5Widgets:Qt5Widgets.dll
 0000:fffee000       .debug$S                   10000000     Qt5Widgets:Qt5Widgets.dll
 0000:fffee000       .debug$S                   10000000     Qt5Widgets:Qt5Widgets.dll
 0000:fffee000       .debug$S                   10000000     Qt5Widgets:Qt5Widgets.dll
 0000:fffee000       .debug$S                   10000000     Qt5Widgets:Qt5Widgets.dll
 0000:fffee000       .debug$S                   10000000     Qt5Widgets:Qt5Widgets.dll
 0000:fffee000       .debug$S                   10000000     Qt5Widgets:Qt5Widgets.dll
 0000:fffee000       .debug$S                   10000000     Qt5Widgets:Qt5Widgets.dll
 0000:fffee000       .debug$S                   10000000     Qt5Widgets:Qt5Widgets.dll
 0000:fffee000       .debug$S                   10000000     Qt5Widgets:Qt5Widgets.dll
 0000:fffee000       .debug$S                   10000000     Qt5Widgets:Qt5Widgets.dll
 0000:fffee000       .debug$S                   10000000     Qt5Widgets:Qt5Widgets.dll
 0000:fffee000       .debug$S                   10000000     Qt5Widgets:Qt5Widgets.dll
 0000:fffee000       .debug$S                   10000000     Qt5Widgets:Qt5Widgets.dll
 0000:fffee000       .debug$S                   10000000     Qt5Widgets:Qt5Widgets.dll
 0000:fffee000       .debug$S                   10000000     Qt5Widgets:Qt5Widgets.dll
 0000:fffee000       .debug$S                   10000000     Qt5Widgets:Qt5Widgets.dll
 0000:fffee000       .debug$S                   10000000     Qt5Widgets:Qt5Widgets.dll
 0000:fffee000       .debug$S                   10000000     Qt5Widgets:Qt5Widgets.dll
 0000:fffee000       .debug$S                   10000000     Qt5Widgets:Qt5Widgets.dll
 0000:fffee000       .debug$S                   10000000     Qt5Widgets:Qt5Widgets.dll
 0000:fffee000       .debug$S                   10000000     Qt5Widgets:Qt5Widgets.dll
 0000:fffee000       .debug$S                   10000000     Qt5Widgets:Qt5Widgets.dll
 0000:fffee000       .debug$S                   10000000     Qt5Widgets:Qt5Widgets.dll
 0000:fffee000       .debug$S                   10000000     Qt5Widgets:Qt5Widgets.dll
 0000:fffee000       .debug$S                   10000000     Qt5Widgets:Qt5Widgets.dll
 0000:fffee000       .debug$S                   10000000     Qt5Widgets:Qt5Widgets.dll
 0000:fffee000       .debug$S                   10000000     Qt5Widgets:Qt5Widgets.dll
 0000:fffee000       .debug$S                   10000000     Qt5Widgets:Qt5Widgets.dll
 0000:fffee000       .debug$S                   10000000     Qt5Widgets:Qt5Widgets.dll
 0000:fffee000       .debug$S                   10000000     Qt5Widgets:Qt5Widgets.dll
 0000:fffee000       .debug$S                   10000000     Qt5Widgets:Qt5Widgets.dll
 0000:fffee000       .debug$S                   10000000     Qt5Widgets:Qt5Widgets.dll
 0000:fffee000       .debug$S                   10000000     Qt5Widgets:Qt5Widgets.dll
 0000:fffee000       .debug$S                   10000000     Qt5Widgets:Qt5Widgets.dll
 0000:fffee000       .debug$S                   10000000     Qt5Widgets:Qt5Widgets.dll
 0000:fffee000       .debug$S                   10000000     Qt5Widgets:Qt5Widgets.dll
 0000:fffee000       .debug$S                   10000000     Qt5Widgets:Qt5Widgets.dll
 0000:fffee000       .debug$S                   10000000     Qt5Widgets:Qt5Widgets.dll
 0000:fffee000       .debug$S                   10000000     Qt5Widgets:Qt5Widgets.dll
 0000:fffee000       .debug$S                   10000000     Qt5Widgets:Qt5Widgets.dll
 0000:fffee000       .debug$S                   10000000     Qt5Widgets:Qt5Widgets.dll
 0000:fffee000       .debug$S                   10000000     Qt5Widgets:Qt5Widgets.dll
 0000:fffee000       .debug$S                   10000000     Qt5Widgets:Qt5Widgets.dll
 0000:fffee000       .debug$S                   10000000     Qt5Widgets:Qt5Widgets.dll
 0000:fffee000       .debug$S                   10000000     Qt5Widgets:Qt5Widgets.dll
 0000:fffee000       .debug$S                   10000000     Qt5Widgets:Qt5Widgets.dll
 0000:fffee000       .debug$S                   10000000     Qt5Widgets:Qt5Widgets.dll
 0000:fffee000       .debug$S                   10000000     Qt5Widgets:Qt5Widgets.dll
 0000:fffee000       .debug$S                   10000000     Qt5Widgets:Qt5Widgets.dll
 0000:fffee000       .debug$S                   10000000     Qt5Widgets:Qt5Widgets.dll
 0000:fffee000       .debug$S                   10000000     Qt5Widgets:Qt5Widgets.dll
 0000:fffee000       .debug$S                   10000000     Qt5Widgets:Qt5Widgets.dll
 0000:fffee000       .debug$S                   10000000     Qt5Widgets:Qt5Widgets.dll
 0000:fffee000       .debug$S                   10000000     Qt5Widgets:Qt5Widgets.dll
 0000:fffee000       .debug$S                   10000000     Qt5Widgets:Qt5Widgets.dll
 0002:ffff8000       __catchsym$??0?$QList@PAVCudaGpuModel@U2@@@@QAE@ABV0@@Z$2 10000000     CudaSupportSettingsController.obj
 0000:fffee000       .debug$S                   10000000     Qt5Widgets:Qt5Widgets.dll
 0000:fffee000       .debug$S                   10000000     Qt5Widgets:Qt5Widgets.dll
 0000:fffee000       .debug$S                   10000000     Qt5Widgets:Qt5Widgets.dll
 0000:fffee000       .debug$S                   10000000     Qt5Widgets:Qt5Widgets.dll
 0000:fffee000       .debug$S                   10000000     Qt5Widgets:Qt5Widgets.dll
 0000:fffee000       .debug$S                   10000000     Qt5Widgets:Qt5Widgets.dll
 0000:fffee000       .debug$S                   10000000     Qt5Widgets:Qt5Widgets.dll
 0000:fffee000       .debug$S                   10000000     Qt5Widgets:Qt5Widgets.dll
 0000:fffee000       .debug$S                   10000000     Qt5Widgets:Qt5Widgets.dll
 0000:fffee000       .debug$S                   10000000     Qt5Widgets:Qt5Widgets.dll
 0000:fffee000       .debug$S                   10000000     Qt5Widgets:Qt5Widgets.dll
 0000:fffee000       .debug$S                   10000000     Qt5Widgets:Qt5Widgets.dll
 0000:fffee000       .debug$S                   10000000     Qt5Widgets:Qt5Widgets.dll
 0000:fffee000       .debug$S                   10000000     Qt5Widgets:Qt5Widgets.dll
 0000:fffee000       .debug$S                   10000000     Qt5Widgets:Qt5Widgets.dll
 0000:fffee000       .debug$S                   10000000     Qt5Widgets:Qt5Widgets.dll
 0000:fffee000       .debug$S                   10000000     Qt5Widgets:Qt5Widgets.dll
 0000:fffee000       .debug$S                   10000000     Qt5Widgets:Qt5Widgets.dll
 0000:fffee000       .debug$S                   10000000     Qt5Widgets:Qt5Widgets.dll
 0000:fffee000       .debug$S                   10000000     Qt5Widgets:Qt5Widgets.dll
 0000:fffee000       .debug$S                   10000000     Qt5Widgets:Qt5Widgets.dll
 0000:fffee000       .debug$S                   10000000     Qt5Widgets:Qt5Widgets.dll
 0000:fffee000       .debug$S                   10000000     Qt5Widgets:Qt5Widgets.dll
 0000:fffee000       .debug$S                   10000000     U2Core:U2Core.dll
 0002:ffff8008       __ehfuncinfo$??H@YA?BVQString@@ABV0@0@Z 10000008     CudaSupportSettingsController.obj
 0002:ffff8010       __ehfuncinfo$??H@YA?BVQString@@ABV0@PBD@Z 10000010     CudaSupportSettingsController.obj
 0002:ffff8010       __catchsym$?_Copy@?$basic_string@DU?$char_traits@D@std@@V?$allocator@D@2@@std@@QAEXII@Z$4 10000010     moc_CudaSupportPlugin.obj
 0002:ffff8010       __unwindtable$??0?$QList@PAVCudaGpuModel@U2@@@@QAE@ABV0@@Z 10000010     CudaSupportSettingsController.obj
 0002:ffff8010       __catchsym$?_Copy@?$basic_string@DU?$char_traits@D@std@@V?$allocator@D@2@@std@@QAEXII@Z$4 10000010     CudaSupportSettingsController.obj
 0002:ffff8010       __catchsym$?_Copy@?$basic_string@DU?$char_traits@D@std@@V?$allocator@D@2@@std@@QAEXII@Z$4 10000010     moc_CudaSupportSettingsController.obj
 0001:fffff01a       __ehhandler$??H@YA?BVQString@@ABV0@0@Z 1000001a f   CudaSupportSettingsController.obj
 0001:fffff01a       __unwindfunclet$??H@YA?BVQString@@ABV0@PBD@Z$1 1000001a f   CudaSupportSettingsController.obj
 0002:ffff8020       __tryblocktable$??0?$QList@PAVCudaGpuModel@U2@@@@QAE@ABV0@@Z 10000020     CudaSupportSettingsController.obj
 0002:ffff8020       __unwindtable$?_Copy@?$basic_string@DU?$char_traits@D@std@@V?$allocator@D@2@@std@@QAEXII@Z 10000020     moc_CudaSupportSettingsController.obj
 0002:ffff8020       __unwindtable$?_Copy@?$basic_string@DU?$char_traits@D@std@@V?$allocator@D@2@@std@@QAEXII@Z 10000020     moc_CudaSupportPlugin.obj
 0002:ffff8020       __unwindtable$?_Copy@?$basic_string@DU?$char_traits@D@std@@V?$allocator@D@2@@std@@QAEXII@Z 10000020     CudaSupportSettingsController.obj
 0001:fffff023       __ehhandler$??H@YA?BVQString@@ABV0@PBD@Z 10000023 f   CudaSupportSettingsController.obj
 0002:ffff8034       __ehfuncinfo$??0?$QList@PAVCudaGpuModel@U2@@@@QAE@ABV0@@Z 10000034     CudaSupportSettingsController.obj
 0002:ffff8040       __ehfuncinfo$?_Copy@?$basic_string@DU?$char_traits@D@std@@V?$allocator@D@2@@std@@QAEXII@Z 10000040     moc_CudaSupportSettingsController.obj
 0002:ffff8040       __ehfuncinfo$?_Copy@?$basic_string@DU?$char_traits@D@std@@V?$allocator@D@2@@std@@QAEXII@Z 10000040     CudaSupportSettingsController.obj
 0002:ffff8040       __ehfuncinfo$?_Copy@?$basic_string@DU?$char_traits@D@std@@V?$allocator@D@2@@std@@QAEXII@Z 10000040     moc_CudaSupportPlugin.obj
 0002:ffff8064       __tryblocktable$?_Copy@?$basic_string@DU?$char_traits@D@std@@V?$allocator@D@2@@std@@QAEXII@Z 10000064     moc_CudaSupportSettingsController.obj
 0002:ffff8064       __tryblocktable$?_Copy@?$basic_string@DU?$char_traits@D@std@@V?$allocator@D@2@@std@@QAEXII@Z 10000064     moc_CudaSupportPlugin.obj
 0002:ffff8064       __tryblocktable$?_Copy@?$basic_string@DU?$char_traits@D@std@@V?$allocator@D@2@@std@@QAEXII@Z 10000064     CudaSupportSettingsController.obj
 0001:fffff096       __catch$?_Copy@?$basic_string@DU?$char_traits@D@std@@V?$allocator@D@2@@std@@QAEXII@Z$0 10000096 f   moc_CudaSupportPlugin.obj
 0001:fffff096       __catch$?_Copy@?$basic_string@DU?$char_traits@D@std@@V?$allocator@D@2@@std@@QAEXII@Z$0 10000096 f   moc_CudaSupportSettingsController.obj
 0001:fffff096       __catch$?_Copy@?$basic_string@DU?$char_traits@D@std@@V?$allocator@D@2@@std@@QAEXII@Z$0 10000096 f   CudaSupportSettingsController.obj
 0001:fffff09e       __catch$??0?$QList@PAVCudaGpuModel@U2@@@@QAE@ABV0@@Z$0 1000009e f   CudaSupportSettingsController.obj
 0001:fffff0d3       __catch$?_Copy@?$basic_string@DU?$char_traits@D@std@@V?$allocator@D@2@@std@@QAEXII@Z$1 100000d3 f   CudaSupportSettingsController.obj
 0001:fffff0d3       __catch$?_Copy@?$basic_string@DU?$char_traits@D@std@@V?$allocator@D@2@@std@@QAEXII@Z$1 100000d3 f   moc_CudaSupportPlugin.obj
 0001:fffff0d3       __catch$?_Copy@?$basic_string@DU?$char_traits@D@std@@V?$allocator@D@2@@std@@QAEXII@Z$1 100000d3 f   moc_CudaSupportSettingsController.obj
 0001:00000000       ??__E?_Generic_object@?$_Error_objects@H@std@@2V_Generic_error_category@2@A@@YAXXZ 10001000 f   CudaSupportPlugin.obj
 0001:00000010       ??__E?_Iostream_object@?$_Error_objects@H@std@@2V_Iostream_error_category@2@A@@YAXXZ 10001010 f   CudaSupportPlugin.obj
 0001:00000020       ??__E?_System_object@?$_Error_objects@H@std@@2V_System_error_category@2@A@@YAXXZ 10001020 f   CudaSupportPlugin.obj
 0001:00000030       ??__EalgoLog@U2@@YAXXZ     10001030 f   CudaSupportPlugin.obj
 0001:000000b0       ??__EcmdLog@U2@@YAXXZ      100010b0 f   CudaSupportPlugin.obj
 0001:00000130       ??__EcoreLog@U2@@YAXXZ     10001130 f   CudaSupportPlugin.obj
 0001:000001b0       ??__EioLog@U2@@YAXXZ       100011b0 f   CudaSupportPlugin.obj
 0001:00000230       ??__EperfLog@U2@@YAXXZ     10001230 f   CudaSupportPlugin.obj
 0001:000002b0       ??__EscriptLog@U2@@YAXXZ   100012b0 f   CudaSupportPlugin.obj
 0001:00000330       ??__EtaskLog@U2@@YAXXZ     10001330 f   CudaSupportPlugin.obj
 0001:000003b0       ??__EuiLog@U2@@YAXXZ       100013b0 f   CudaSupportPlugin.obj
 0001:00000430       ??__EuserActLog@U2@@YAXXZ  10001430 f   CudaSupportPlugin.obj
 0001:000004b0       ??__E?_Generic_object@?$_Error_objects@H@std@@2V_Generic_error_category@2@A@@YAXXZ 100014b0 f   CudaSupportSettingsController.obj
 0001:000004c0       ??__E?_Iostream_object@?$_Error_objects@H@std@@2V_Iostream_error_category@2@A@@YAXXZ 100014c0 f   CudaSupportSettingsController.obj
 0001:000004d0       ??__E?_System_object@?$_Error_objects@H@std@@2V_System_error_category@2@A@@YAXXZ 100014d0 f   CudaSupportSettingsController.obj
 0001:000004e0       ??__E?helpPageId@CudaSupportSettingsPageController@U2@@0VQString@@B@@YAXXZ 100014e0 f   CudaSupportSettingsController.obj
 0001:00000500       ??__EalgoLog@U2@@YAXXZ     10001500 f   CudaSupportSettingsController.obj
 0001:00000580       ??__EcmdLog@U2@@YAXXZ      10001580 f   CudaSupportSettingsController.obj
 0001:00000600       ??__EcoreLog@U2@@YAXXZ     10001600 f   CudaSupportSettingsController.obj
 0001:00000680       ??__EioLog@U2@@YAXXZ       10001680 f   CudaSupportSettingsController.obj
 0001:00000700       ??__EperfLog@U2@@YAXXZ     10001700 f   CudaSupportSettingsController.obj
 0001:00000780       ??__EscriptLog@U2@@YAXXZ   10001780 f   CudaSupportSettingsController.obj
 0001:00000800       ??__EtaskLog@U2@@YAXXZ     10001800 f   CudaSupportSettingsController.obj
 0001:00000880       ??__EuiLog@U2@@YAXXZ       10001880 f   CudaSupportSettingsController.obj
 0001:00000900       ??__EuserActLog@U2@@YAXXZ  10001900 f   CudaSupportSettingsController.obj
 0001:00000980       ??__E?_Generic_object@?$_Error_objects@H@std@@2V_Generic_error_category@2@A@@YAXXZ 10001980 f   moc_CudaSupportPlugin.obj
 0001:00000990       ??__E?_Iostream_object@?$_Error_objects@H@std@@2V_Iostream_error_category@2@A@@YAXXZ 10001990 f   moc_CudaSupportPlugin.obj
 0001:000009a0       ??__E?_System_object@?$_Error_objects@H@std@@2V_System_error_category@2@A@@YAXXZ 100019a0 f   moc_CudaSupportPlugin.obj
 0001:000009b0       ??__E?staticMetaObject@CudaSupportPlugin@U2@@2UQMetaObject@@B@@YAXXZ 100019b0 f   moc_CudaSupportPlugin.obj
 0001:000009c0       ??__E?_Generic_object@?$_Error_objects@H@std@@2V_Generic_error_category@2@A@@YAXXZ 100019c0 f   moc_CudaSupportSettingsController.obj
 0001:000009d0       ??__E?_Iostream_object@?$_Error_objects@H@std@@2V_Iostream_error_category@2@A@@YAXXZ 100019d0 f   moc_CudaSupportSettingsController.obj
 0001:000009e0       ??__E?_System_object@?$_Error_objects@H@std@@2V_System_error_category@2@A@@YAXXZ 100019e0 f   moc_CudaSupportSettingsController.obj
 0001:000009f0       ??__E?staticMetaObject@CudaSupportSettingsPageController@U2@@2UQMetaObject@@B@@YAXXZ 100019f0 f   moc_CudaSupportSettingsController.obj
 0001:00000a00       ??__E?staticMetaObject@CudaSupportSettingsPageState@U2@@2UQMetaObject@@B@@YAXXZ 10001a00 f   moc_CudaSupportSettingsController.obj
 0001:00000a10       ??__E?staticMetaObject@CudaSupportSettingsPageWidget@U2@@2UQMetaObject@@B@@YAXXZ 10001a10 f   moc_CudaSupportSettingsController.obj
 0001:00000c3e       __catch$??0?$QList@PAVCudaGpuModel@U2@@@@QAE@ABV0@@Z$0 10001c3e f i CudaSupportPlugin.obj
 0001:000015b6       __catch$?_Copy@?$basic_string@DU?$char_traits@D@std@@V?$allocator@D@2@@std@@QAEXII@Z$0 100025b6 f i CudaSupportPlugin.obj
 0001:000015f3       __catch$?_Copy@?$basic_string@DU?$char_traits@D@std@@V?$allocator@D@2@@std@@QAEXII@Z$1 100025f3 f i CudaSupportPlugin.obj
 0001:00001915       __catch$?append@?$QList@PAVCudaGpuModel@U2@@@@QAEXABQAVCudaGpuModel@U2@@@Z$4 10002915 f i CudaSupportPlugin.obj
 0001:00001dd1       __catch$?detach_helper_grow@?$QList@PAVCudaGpuModel@U2@@@@AAEPAUNode@1@HH@Z$2 10002dd1 f i CudaSupportPlugin.obj
 0001:00001dd1       __catch$?detach_helper_grow@?$QList@PAVCudaGpuModel@U2@@@@AAEPAUNode@1@HH@Z$0 10002dd1 f i CudaSupportPlugin.obj
 0001:0000208c       $LN17                      1000308c     CudaSupportPlugin.obj
 0001:00003b85       __catch$?append@?$QList@PAVQCheckBox@@@@QAEXABQAVQCheckBox@@@Z$4 10004b85 f i CudaSupportSettingsController.obj
 0001:00003edc       __catch$?detach_helper@?$QList@PAVCudaGpuModel@U2@@@@AAEXH@Z$0 10004edc f i CudaSupportSettingsController.obj
 0001:00004001       __catch$?detach_helper_grow@?$QList@PAVQCheckBox@@@@AAEPAUNode@1@HH@Z$0 10005001 f i CudaSupportSettingsController.obj
 0001:00004001       __catch$?detach_helper_grow@?$QList@PAVQCheckBox@@@@AAEPAUNode@1@HH@Z$2 10005001 f i CudaSupportSettingsController.obj
 0001:00004543       __catch$?reallocData@?$QVector@_N@@AAEXHHV?$QFlags@W4AllocationOption@QArrayData@@@@@Z$0 10005543 f i CudaSupportSettingsController.obj
 0001:00004555       __catch$?reallocData@?$QVector@_N@@AAEXHHV?$QFlags@W4AllocationOption@QArrayData@@@@@Z$2 10005555 f i CudaSupportSettingsController.obj
 0001:0000520c       _pre_c_init                1000620c f   MSVCRT:crtdll.obj
 0001:00005479       ___DllMainCRTStartup       10006479 f   MSVCRT:crtdll.obj
 0001:000055d0       $$000000                   100065d0     MSVCRT:sehprolg4.obj
 0001:000059e5       ?ArrayUnwindFilter@@YAHPAU_EXCEPTION_POINTERS@@@Z 100069e5 f   MSVCRT:ehvecdtr.obj
 0001:00005d30       __ehhandler$??0?$QList@PAVCudaGpuModel@U2@@@@QAE@ABV0@@Z 10006d30 f   CudaSupportPlugin.obj
 0001:00005d50       __unwindfunclet$??0CudaSupportPlugin@U2@@QAE@XZ$0 10006d50 f   CudaSupportPlugin.obj
 0001:00005d59       __unwindfunclet$??0CudaSupportPlugin@U2@@QAE@XZ$1 10006d59 f   CudaSupportPlugin.obj
 0001:00005d62       __unwindfunclet$??0CudaSupportPlugin@U2@@QAE@XZ$2 10006d62 f   CudaSupportPlugin.obj
 0001:00005d6b       __unwindfunclet$??0CudaSupportPlugin@U2@@QAE@XZ$3 10006d6b f   CudaSupportPlugin.obj
 0001:00005d76       __unwindfunclet$??0CudaSupportPlugin@U2@@QAE@XZ$4 10006d76 f   CudaSupportPlugin.obj
 0001:00005d7f       __unwindfunclet$??0CudaSupportPlugin@U2@@QAE@XZ$5 10006d7f f   CudaSupportPlugin.obj
 0001:00005d88       __unwindfunclet$??0CudaSupportPlugin@U2@@QAE@XZ$6 10006d88 f   CudaSupportPlugin.obj
 0001:00005d93       __unwindfunclet$??0CudaSupportPlugin@U2@@QAE@XZ$7 10006d93 f   CudaSupportPlugin.obj
 0001:00005d9c       __unwindfunclet$??0CudaSupportPlugin@U2@@QAE@XZ$8 10006d9c f   CudaSupportPlugin.obj
 0001:00005da7       __unwindfunclet$??0CudaSupportPlugin@U2@@QAE@XZ$9 10006da7 f   CudaSupportPlugin.obj
 0001:00005dc1       __unwindfunclet$??0CudaSupportPlugin@U2@@QAE@XZ$10 10006dc1 f   CudaSupportPlugin.obj
 0001:00005ddb       __ehhandler$??0CudaSupportPlugin@U2@@QAE@XZ 10006ddb f   CudaSupportPlugin.obj
 0001:00005e00       __unwindfunclet$??1CudaSupportPlugin@U2@@UAE@XZ$0 10006e00 f   CudaSupportPlugin.obj
 0001:00005e09       __ehhandler$??1CudaSupportPlugin@U2@@UAE@XZ 10006e09 f   CudaSupportPlugin.obj
 0001:00005e30       __unwindfunclet$??H@YA?BVQString@@ABV0@0@Z$0 10006e30 f   CudaSupportPlugin.obj
 0001:00005e4a       __ehhandler$??H@YA?BVQString@@ABV0@0@Z 10006e4a f   CudaSupportPlugin.obj
 0001:00005e70       __unwindfunclet$??H@YA?BVQString@@ABV0@PBD@Z$0 10006e70 f   CudaSupportPlugin.obj
 0001:00005e8a       __unwindfunclet$??H@YA?BVQString@@ABV0@PBD@Z$1 10006e8a f   CudaSupportPlugin.obj
 0001:00005e93       __ehhandler$??H@YA?BVQString@@ABV0@PBD@Z 10006e93 f   CudaSupportPlugin.obj
 0001:00005eb0       __unwindfunclet$??H@YA?BVQString@@PBDABV0@@Z$0 10006eb0 f   CudaSupportPlugin.obj
 0001:00005eca       __ehhandler$??H@YA?BVQString@@PBDABV0@@Z 10006eca f   CudaSupportPlugin.obj
 0001:00005ef0       __unwindfunclet$??_GCudaSupportPlugin@U2@@UAEPAXI@Z$0 10006ef0 f   CudaSupportPlugin.obj
 0001:00005ef9       __ehhandler$??_GCudaSupportPlugin@U2@@UAEPAXI@Z 10006ef9 f   CudaSupportPlugin.obj
 0001:00005f20       __unwindfunclet$??__EalgoLog@U2@@YAXXZ$0 10006f20 f   CudaSupportPlugin.obj
 0001:00005f29       __ehhandler$??__EalgoLog@U2@@YAXXZ 10006f29 f   CudaSupportPlugin.obj
 0001:00005f50       __unwindfunclet$??__EcmdLog@U2@@YAXXZ$0 10006f50 f   CudaSupportPlugin.obj
 0001:00005f59       __ehhandler$??__EcmdLog@U2@@YAXXZ 10006f59 f   CudaSupportPlugin.obj
 0001:00005f80       __unwindfunclet$??__EcoreLog@U2@@YAXXZ$0 10006f80 f   CudaSupportPlugin.obj
 0001:00005f89       __ehhandler$??__EcoreLog@U2@@YAXXZ 10006f89 f   CudaSupportPlugin.obj
 0001:00005fb0       __unwindfunclet$??__EioLog@U2@@YAXXZ$0 10006fb0 f   CudaSupportPlugin.obj
 0001:00005fb9       __ehhandler$??__EioLog@U2@@YAXXZ 10006fb9 f   CudaSupportPlugin.obj
 0001:00005fe0       __unwindfunclet$??__EperfLog@U2@@YAXXZ$0 10006fe0 f   CudaSupportPlugin.obj
 0001:00005fe9       __ehhandler$??__EperfLog@U2@@YAXXZ 10006fe9 f   CudaSupportPlugin.obj
 0001:00006010       __unwindfunclet$??__EscriptLog@U2@@YAXXZ$0 10007010 f   CudaSupportPlugin.obj
 0001:00006019       __ehhandler$??__EscriptLog@U2@@YAXXZ 10007019 f   CudaSupportPlugin.obj
 0001:00006040       __unwindfunclet$??__EtaskLog@U2@@YAXXZ$0 10007040 f   CudaSupportPlugin.obj
 0001:00006049       __ehhandler$??__EtaskLog@U2@@YAXXZ 10007049 f   CudaSupportPlugin.obj
 0001:00006070       __unwindfunclet$??__EuiLog@U2@@YAXXZ$0 10007070 f   CudaSupportPlugin.obj
 0001:00006079       __ehhandler$??__EuiLog@U2@@YAXXZ 10007079 f   CudaSupportPlugin.obj
 0001:000060a0       __unwindfunclet$??__EuserActLog@U2@@YAXXZ$0 100070a0 f   CudaSupportPlugin.obj
 0001:000060a9       __ehhandler$??__EuserActLog@U2@@YAXXZ 100070a9 f   CudaSupportPlugin.obj
 0001:000060d0       __ehhandler$?_Copy@?$basic_string@DU?$char_traits@D@std@@V?$allocator@D@2@@std@@QAEXII@Z 100070d0 f   CudaSupportPlugin.obj
 0001:000060f0       __ehhandler$?append@?$QList@PAVCudaGpuModel@U2@@@@QAEXABQAVCudaGpuModel@U2@@@Z 100070f0 f   CudaSupportPlugin.obj
 0001:00006110       __ehhandler$?detach_helper_grow@?$QList@PAVCudaGpuModel@U2@@@@AAEPAUNode@1@HH@Z 10007110 f   CudaSupportPlugin.obj
 0001:00006130       __unwindfunclet$?loadGpusSettings@CudaSupportPlugin@U2@@AAEXXZ$0 10007130 f   CudaSupportPlugin.obj
 0001:00006138       __unwindfunclet$?loadGpusSettings@CudaSupportPlugin@U2@@AAEXXZ$1 10007138 f   CudaSupportPlugin.obj
 0001:00006141       __unwindfunclet$?loadGpusSettings@CudaSupportPlugin@U2@@AAEXXZ$2 10007141 f   CudaSupportPlugin.obj
 0001:0000614a       __unwindfunclet$?loadGpusSettings@CudaSupportPlugin@U2@@AAEXXZ$3 1000714a f   CudaSupportPlugin.obj
 0001:00006153       __unwindfunclet$?loadGpusSettings@CudaSupportPlugin@U2@@AAEXXZ$4 10007153 f   CudaSupportPlugin.obj
 0001:0000615c       __unwindfunclet$?loadGpusSettings@CudaSupportPlugin@U2@@AAEXXZ$5 1000715c f   CudaSupportPlugin.obj
 0001:00006165       __ehhandler$?loadGpusSettings@CudaSupportPlugin@U2@@AAEXXZ 10007165 f   CudaSupportPlugin.obj
 0001:00006180       __unwindfunclet$?obtainGpusInfo@CudaSupportPlugin@U2@@AAE?AW4Error@12@AAVQString@@@Z$0 10007180 f   CudaSupportPlugin.obj
 0001:00006189       __unwindfunclet$?obtainGpusInfo@CudaSupportPlugin@U2@@AAE?AW4Error@12@AAVQString@@@Z$1 10007189 f   CudaSupportPlugin.obj
 0001:00006192       __unwindfunclet$?obtainGpusInfo@CudaSupportPlugin@U2@@AAE?AW4Error@12@AAVQString@@@Z$2 10007192 f   CudaSupportPlugin.obj
 0001:0000619e       __unwindfunclet$?obtainGpusInfo@CudaSupportPlugin@U2@@AAE?AW4Error@12@AAVQString@@@Z$3 1000719e f   CudaSupportPlugin.obj
 0001:000061a7       __unwindfunclet$?obtainGpusInfo@CudaSupportPlugin@U2@@AAE?AW4Error@12@AAVQString@@@Z$4 100071a7 f   CudaSupportPlugin.obj
 0001:000061b0       __unwindfunclet$?obtainGpusInfo@CudaSupportPlugin@U2@@AAE?AW4Error@12@AAVQString@@@Z$5 100071b0 f   CudaSupportPlugin.obj
 0001:000061b9       __unwindfunclet$?obtainGpusInfo@CudaSupportPlugin@U2@@AAE?AW4Error@12@AAVQString@@@Z$6 100071b9 f   CudaSupportPlugin.obj
 0001:000061c2       __unwindfunclet$?obtainGpusInfo@CudaSupportPlugin@U2@@AAE?AW4Error@12@AAVQString@@@Z$7 100071c2 f   CudaSupportPlugin.obj
 0001:000061cb       __unwindfunclet$?obtainGpusInfo@CudaSupportPlugin@U2@@AAE?AW4Error@12@AAVQString@@@Z$8 100071cb f   CudaSupportPlugin.obj
 0001:000061d4       __unwindfunclet$?obtainGpusInfo@CudaSupportPlugin@U2@@AAE?AW4Error@12@AAVQString@@@Z$9 100071d4 f   CudaSupportPlugin.obj
 0001:000061dd       __unwindfunclet$?obtainGpusInfo@CudaSupportPlugin@U2@@AAE?AW4Error@12@AAVQString@@@Z$10 100071dd f   CudaSupportPlugin.obj
 0001:000061e6       __unwindfunclet$?obtainGpusInfo@CudaSupportPlugin@U2@@AAE?AW4Error@12@AAVQString@@@Z$11 100071e6 f   CudaSupportPlugin.obj
 0001:000061ef       __unwindfunclet$?obtainGpusInfo@CudaSupportPlugin@U2@@AAE?AW4Error@12@AAVQString@@@Z$12 100071ef f   CudaSupportPlugin.obj
 0001:000061f8       __unwindfunclet$?obtainGpusInfo@CudaSupportPlugin@U2@@AAE?AW4Error@12@AAVQString@@@Z$13 100071f8 f   CudaSupportPlugin.obj
 0001:00006201       __unwindfunclet$?obtainGpusInfo@CudaSupportPlugin@U2@@AAE?AW4Error@12@AAVQString@@@Z$14 10007201 f   CudaSupportPlugin.obj
 0001:0000620a       __unwindfunclet$?obtainGpusInfo@CudaSupportPlugin@U2@@AAE?AW4Error@12@AAVQString@@@Z$15 1000720a f   CudaSupportPlugin.obj
 0001:00006213       __unwindfunclet$?obtainGpusInfo@CudaSupportPlugin@U2@@AAE?AW4Error@12@AAVQString@@@Z$19 10007213 f   CudaSupportPlugin.obj
 0001:0000621c       __unwindfunclet$?obtainGpusInfo@CudaSupportPlugin@U2@@AAE?AW4Error@12@AAVQString@@@Z$29 1000721c f   CudaSupportPlugin.obj
 0001:0000622a       __unwindfunclet$?obtainGpusInfo@CudaSupportPlugin@U2@@AAE?AW4Error@12@AAVQString@@@Z$30 1000722a f   CudaSupportPlugin.obj
 0001:00006244       __unwindfunclet$?obtainGpusInfo@CudaSupportPlugin@U2@@AAE?AW4Error@12@AAVQString@@@Z$31 10007244 f   CudaSupportPlugin.obj
 0001:0000624d       __unwindfunclet$?obtainGpusInfo@CudaSupportPlugin@U2@@AAE?AW4Error@12@AAVQString@@@Z$32 1000724d f   CudaSupportPlugin.obj
 0001:00006259       __unwindfunclet$?obtainGpusInfo@CudaSupportPlugin@U2@@AAE?AW4Error@12@AAVQString@@@Z$33 10007259 f   CudaSupportPlugin.obj
 0001:00006265       __unwindfunclet$?obtainGpusInfo@CudaSupportPlugin@U2@@AAE?AW4Error@12@AAVQString@@@Z$34 10007265 f   CudaSupportPlugin.obj
 0001:00006271       __unwindfunclet$?obtainGpusInfo@CudaSupportPlugin@U2@@AAE?AW4Error@12@AAVQString@@@Z$28 10007271 f   CudaSupportPlugin.obj
 0001:0000627a       __unwindfunclet$?obtainGpusInfo@CudaSupportPlugin@U2@@AAE?AW4Error@12@AAVQString@@@Z$26 1000727a f   CudaSupportPlugin.obj
 0001:00006283       __unwindfunclet$?obtainGpusInfo@CudaSupportPlugin@U2@@AAE?AW4Error@12@AAVQString@@@Z$27 10007283 f   CudaSupportPlugin.obj
 0001:0000628c       __unwindfunclet$?obtainGpusInfo@CudaSupportPlugin@U2@@AAE?AW4Error@12@AAVQString@@@Z$25 1000728c f   CudaSupportPlugin.obj
 0001:00006295       __unwindfunclet$?obtainGpusInfo@CudaSupportPlugin@U2@@AAE?AW4Error@12@AAVQString@@@Z$23 10007295 f   CudaSupportPlugin.obj
 0001:0000629e       __unwindfunclet$?obtainGpusInfo@CudaSupportPlugin@U2@@AAE?AW4Error@12@AAVQString@@@Z$24 1000729e f   CudaSupportPlugin.obj
 0001:000062a7       __unwindfunclet$?obtainGpusInfo@CudaSupportPlugin@U2@@AAE?AW4Error@12@AAVQString@@@Z$22 100072a7 f   CudaSupportPlugin.obj
 0001:000062b0       __unwindfunclet$?obtainGpusInfo@CudaSupportPlugin@U2@@AAE?AW4Error@12@AAVQString@@@Z$20 100072b0 f   CudaSupportPlugin.obj
 0001:000062b9       __unwindfunclet$?obtainGpusInfo@CudaSupportPlugin@U2@@AAE?AW4Error@12@AAVQString@@@Z$21 100072b9 f   CudaSupportPlugin.obj
 0001:000062c2       __unwindfunclet$?obtainGpusInfo@CudaSupportPlugin@U2@@AAE?AW4Error@12@AAVQString@@@Z$18 100072c2 f   CudaSupportPlugin.obj
 0001:000062cb       __unwindfunclet$?obtainGpusInfo@CudaSupportPlugin@U2@@AAE?AW4Error@12@AAVQString@@@Z$16 100072cb f   CudaSupportPlugin.obj
 0001:000062d4       __unwindfunclet$?obtainGpusInfo@CudaSupportPlugin@U2@@AAE?AW4Error@12@AAVQString@@@Z$17 100072d4 f   CudaSupportPlugin.obj
 0001:000062dd       __ehhandler$?obtainGpusInfo@CudaSupportPlugin@U2@@AAE?AW4Error@12@AAVQString@@@Z 100072dd f   CudaSupportPlugin.obj
 0001:00006310       __unwindfunclet$?registerAvailableGpus@CudaSupportPlugin@U2@@AAEXXZ$0 10007310 f   CudaSupportPlugin.obj
 0001:00006318       __ehhandler$?registerAvailableGpus@CudaSupportPlugin@U2@@AAEXXZ 10007318 f   CudaSupportPlugin.obj
 0001:00006340       __unwindfunclet$??0CudaSupportSettingsPageController@U2@@QAE@ABVQString@@PAVQObject@@@Z$0 10007340 f   CudaSupportSettingsController.obj
 0001:00006349       __unwindfunclet$??0CudaSupportSettingsPageController@U2@@QAE@ABVQString@@PAVQObject@@@Z$1 10007349 f   CudaSupportSettingsController.obj
 0001:00006352       __unwindfunclet$??0CudaSupportSettingsPageController@U2@@QAE@ABVQString@@PAVQObject@@@Z$2 10007352 f   CudaSupportSettingsController.obj
 0001:0000635b       __ehhandler$??0CudaSupportSettingsPageController@U2@@QAE@ABVQString@@PAVQObject@@@Z 1000735b f   CudaSupportSettingsController.obj
 0001:00006380       __unwindfunclet$??0CudaSupportSettingsPageState@U2@@QAE@H@Z$0 10007380 f   CudaSupportSettingsController.obj
 0001:00006389       __unwindfunclet$??0CudaSupportSettingsPageState@U2@@QAE@H@Z$1 10007389 f   CudaSupportSettingsController.obj
 0001:00006394       __ehhandler$??0CudaSupportSettingsPageState@U2@@QAE@H@Z 10007394 f   CudaSupportSettingsController.obj
 0001:000063b0       __unwindfunclet$??0CudaSupportSettingsPageWidget@U2@@QAE@ABVQString@@PAVCudaSupportSettingsPageController@1@@Z$0 100073b0 f   CudaSupportSettingsController.obj
 0001:000063b9       __unwindfunclet$??0CudaSupportSettingsPageWidget@U2@@QAE@ABVQString@@PAVCudaSupportSettingsPageController@1@@Z$1 100073b9 f   CudaSupportSettingsController.obj
 0001:000063c5       __unwindfunclet$??0CudaSupportSettingsPageWidget@U2@@QAE@ABVQString@@PAVCudaSupportSettingsPageController@1@@Z$2 100073c5 f   CudaSupportSettingsController.obj
 0001:000063d0       __unwindfunclet$??0CudaSupportSettingsPageWidget@U2@@QAE@ABVQString@@PAVCudaSupportSettingsPageController@1@@Z$3 100073d0 f   CudaSupportSettingsController.obj
 0001:000063db       __unwindfunclet$??0CudaSupportSettingsPageWidget@U2@@QAE@ABVQString@@PAVCudaSupportSettingsPageController@1@@Z$4 100073db f   CudaSupportSettingsController.obj
 0001:000063e6       __unwindfunclet$??0CudaSupportSettingsPageWidget@U2@@QAE@ABVQString@@PAVCudaSupportSettingsPageController@1@@Z$5 100073e6 f   CudaSupportSettingsController.obj
 0001:000063f1       __unwindfunclet$??0CudaSupportSettingsPageWidget@U2@@QAE@ABVQString@@PAVCudaSupportSettingsPageController@1@@Z$6 100073f1 f   CudaSupportSettingsController.obj
 0001:000063f9       __unwindfunclet$??0CudaSupportSettingsPageWidget@U2@@QAE@ABVQString@@PAVCudaSupportSettingsPageController@1@@Z$7 100073f9 f   CudaSupportSettingsController.obj
 0001:00006413       __unwindfunclet$??0CudaSupportSettingsPageWidget@U2@@QAE@ABVQString@@PAVCudaSupportSettingsPageController@1@@Z$8 10007413 f   CudaSupportSettingsController.obj
 0001:0000642d       __unwindfunclet$??0CudaSupportSettingsPageWidget@U2@@QAE@ABVQString@@PAVCudaSupportSettingsPageController@1@@Z$9 1000742d f   CudaSupportSettingsController.obj
 0001:00006436       __unwindfunclet$??0CudaSupportSettingsPageWidget@U2@@QAE@ABVQString@@PAVCudaSupportSettingsPageController@1@@Z$10 10007436 f   CudaSupportSettingsController.obj
 0001:00006441       __unwindfunclet$??0CudaSupportSettingsPageWidget@U2@@QAE@ABVQString@@PAVCudaSupportSettingsPageController@1@@Z$11 10007441 f   CudaSupportSettingsController.obj
 0001:00006449       __unwindfunclet$??0CudaSupportSettingsPageWidget@U2@@QAE@ABVQString@@PAVCudaSupportSettingsPageController@1@@Z$12 10007449 f   CudaSupportSettingsController.obj
 0001:00006454       __unwindfunclet$??0CudaSupportSettingsPageWidget@U2@@QAE@ABVQString@@PAVCudaSupportSettingsPageController@1@@Z$13 10007454 f   CudaSupportSettingsController.obj
 0001:0000645d       __unwindfunclet$??0CudaSupportSettingsPageWidget@U2@@QAE@ABVQString@@PAVCudaSupportSettingsPageController@1@@Z$14 1000745d f   CudaSupportSettingsController.obj
 0001:00006466       __unwindfunclet$??0CudaSupportSettingsPageWidget@U2@@QAE@ABVQString@@PAVCudaSupportSettingsPageController@1@@Z$15 10007466 f   CudaSupportSettingsController.obj
 0001:0000646f       __unwindfunclet$??0CudaSupportSettingsPageWidget@U2@@QAE@ABVQString@@PAVCudaSupportSettingsPageController@1@@Z$16 1000746f f   CudaSupportSettingsController.obj
 0001:00006478       __unwindfunclet$??0CudaSupportSettingsPageWidget@U2@@QAE@ABVQString@@PAVCudaSupportSettingsPageController@1@@Z$17 10007478 f   CudaSupportSettingsController.obj
 0001:00006481       __unwindfunclet$??0CudaSupportSettingsPageWidget@U2@@QAE@ABVQString@@PAVCudaSupportSettingsPageController@1@@Z$18 10007481 f   CudaSupportSettingsController.obj
 0001:0000648c       __ehhandler$??0CudaSupportSettingsPageWidget@U2@@QAE@ABVQString@@PAVCudaSupportSettingsPageController@1@@Z 1000748c f   CudaSupportSettingsController.obj
 0001:000064b0       __unwindfunclet$??1CudaSupportSettingsPageController@U2@@UAE@XZ$0 100074b0 f   CudaSupportSettingsController.obj
 0001:000064b9       __ehhandler$??1CudaSupportSettingsPageController@U2@@UAE@XZ 100074b9 f   CudaSupportSettingsController.obj
 0001:000064e0       __unwindfunclet$??1CudaSupportSettingsPageState@U2@@UAE@XZ$0 100074e0 f   CudaSupportSettingsController.obj
 0001:000064e9       __ehhandler$??1CudaSupportSettingsPageState@U2@@UAE@XZ 100074e9 f   CudaSupportSettingsController.obj
 0001:00006510       __unwindfunclet$??1CudaSupportSettingsPageWidget@U2@@UAE@XZ$0 10007510 f   CudaSupportSettingsController.obj
 0001:00006519       __unwindfunclet$??1CudaSupportSettingsPageWidget@U2@@UAE@XZ$1 10007519 f   CudaSupportSettingsController.obj
 0001:00006525       __ehhandler$??1CudaSupportSettingsPageWidget@U2@@UAE@XZ 10007525 f   CudaSupportSettingsController.obj
 0001:00006540       __unwindfunclet$??_GCudaSupportSettingsPageController@U2@@UAEPAXI@Z$0 10007540 f   CudaSupportSettingsController.obj
 0001:00006549       __ehhandler$??_GCudaSupportSettingsPageController@U2@@UAEPAXI@Z 10007549 f   CudaSupportSettingsController.obj
 0001:00006570       __unwindfunclet$??_GCudaSupportSettingsPageState@U2@@UAEPAXI@Z$0 10007570 f   CudaSupportSettingsController.obj
 0001:00006579       __ehhandler$??_GCudaSupportSettingsPageState@U2@@UAEPAXI@Z 10007579 f   CudaSupportSettingsController.obj
 0001:000065a0       __unwindfunclet$??_GCudaSupportSettingsPageWidget@U2@@UAEPAXI@Z$0 100075a0 f   CudaSupportSettingsController.obj
 0001:000065a9       __unwindfunclet$??_GCudaSupportSettingsPageWidget@U2@@UAEPAXI@Z$1 100075a9 f   CudaSupportSettingsController.obj
 0001:000065b5       __ehhandler$??_GCudaSupportSettingsPageWidget@U2@@UAEPAXI@Z 100075b5 f   CudaSupportSettingsController.obj
 0001:000065d0       __unwindfunclet$??__EalgoLog@U2@@YAXXZ$0 100075d0 f   CudaSupportSettingsController.obj
 0001:000065d9       __ehhandler$??__EalgoLog@U2@@YAXXZ 100075d9 f   CudaSupportSettingsController.obj
 0001:00006600       __unwindfunclet$??__EcmdLog@U2@@YAXXZ$0 10007600 f   CudaSupportSettingsController.obj
 0001:00006609       __ehhandler$??__EcmdLog@U2@@YAXXZ 10007609 f   CudaSupportSettingsController.obj
 0001:00006630       __unwindfunclet$??__EcoreLog@U2@@YAXXZ$0 10007630 f   CudaSupportSettingsController.obj
 0001:00006639       __ehhandler$??__EcoreLog@U2@@YAXXZ 10007639 f   CudaSupportSettingsController.obj
 0001:00006660       __unwindfunclet$??__EioLog@U2@@YAXXZ$0 10007660 f   CudaSupportSettingsController.obj
 0001:00006669       __ehhandler$??__EioLog@U2@@YAXXZ 10007669 f   CudaSupportSettingsController.obj
 0001:00006690       __unwindfunclet$??__EperfLog@U2@@YAXXZ$0 10007690 f   CudaSupportSettingsController.obj
 0001:00006699       __ehhandler$??__EperfLog@U2@@YAXXZ 10007699 f   CudaSupportSettingsController.obj
 0001:000066c0       __unwindfunclet$??__EscriptLog@U2@@YAXXZ$0 100076c0 f   CudaSupportSettingsController.obj
 0001:000066c9       __ehhandler$??__EscriptLog@U2@@YAXXZ 100076c9 f   CudaSupportSettingsController.obj
 0001:000066f0       __unwindfunclet$??__EtaskLog@U2@@YAXXZ$0 100076f0 f   CudaSupportSettingsController.obj
 0001:000066f9       __ehhandler$??__EtaskLog@U2@@YAXXZ 100076f9 f   CudaSupportSettingsController.obj
 0001:00006720       __unwindfunclet$??__EuiLog@U2@@YAXXZ$0 10007720 f   CudaSupportSettingsController.obj
 0001:00006729       __ehhandler$??__EuiLog@U2@@YAXXZ 10007729 f   CudaSupportSettingsController.obj
 0001:00006750       __unwindfunclet$??__EuserActLog@U2@@YAXXZ$0 10007750 f   CudaSupportSettingsController.obj
 0001:00006759       __ehhandler$??__EuserActLog@U2@@YAXXZ 10007759 f   CudaSupportSettingsController.obj
 0001:00006780       __ehhandler$?append@?$QList@PAVQCheckBox@@@@QAEXABQAVQCheckBox@@@Z 10007780 f   CudaSupportSettingsController.obj
 0001:000067a0       __unwindfunclet$?createWidget@CudaSupportSettingsPageController@U2@@UAEPAVAppSettingsGUIPageWidget@2@PAVAppSettingsGUIPageState@2@@Z$0 100077a0 f   CudaSupportSettingsController.obj
 0001:000067ab       __ehhandler$?createWidget@CudaSupportSettingsPageController@U2@@UAEPAVAppSettingsGUIPageWidget@2@PAVAppSettingsGUIPageState@2@@Z 100077ab f   CudaSupportSettingsController.obj
 0001:000067d0       __ehhandler$?detach_helper@?$QList@PAVCudaGpuModel@U2@@@@AAEXH@Z 100077d0 f   CudaSupportSettingsController.obj
 0001:000067f0       __ehhandler$?detach_helper_grow@?$QList@PAVQCheckBox@@@@AAEPAUNode@1@HH@Z 100077f0 f   CudaSupportSettingsController.obj
 0001:00006810       __unwindfunclet$?getSavedState@CudaSupportSettingsPageController@U2@@UAEPAVAppSettingsGUIPageState@2@XZ$0 10007810 f   CudaSupportSettingsController.obj
 0001:00006818       __unwindfunclet$?getSavedState@CudaSupportSettingsPageController@U2@@UAEPAVAppSettingsGUIPageState@2@XZ$1 10007818 f   CudaSupportSettingsController.obj
 0001:00006823       __ehhandler$?getSavedState@CudaSupportSettingsPageController@U2@@UAEPAVAppSettingsGUIPageState@2@XZ 10007823 f   CudaSupportSettingsController.obj
 0001:00006840       __unwindfunclet$?getState@CudaSupportSettingsPageWidget@U2@@UBEPAVAppSettingsGUIPageState@2@AAVQString@@@Z$0 10007840 f   CudaSupportSettingsController.obj
 0001:0000684b       __ehhandler$?getState@CudaSupportSettingsPageWidget@U2@@UBEPAVAppSettingsGUIPageState@2@AAVQString@@@Z 1000784b f   CudaSupportSettingsController.obj
 0001:00006870       __ehhandler$?reallocData@?$QVector@_N@@AAEXHHV?$QFlags@W4AllocationOption@QArrayData@@@@@Z 10007870 f   CudaSupportSettingsController.obj
 0001:00006890       __unwindfunclet$?saveState@CudaSupportSettingsPageController@U2@@UAEXPAVAppSettingsGUIPageState@2@@Z$0 10007890 f   CudaSupportSettingsController.obj
 0001:00006898       __ehhandler$?saveState@CudaSupportSettingsPageController@U2@@UAEXPAVAppSettingsGUIPageState@2@@Z 10007898 f   CudaSupportSettingsController.obj
 0001:000068c0       ??__F?_Generic_object@?$_Error_objects@H@std@@2V_Generic_error_category@2@A@@YAXXZ 100078c0 f   CudaSupportPlugin.obj
 0001:000068d0       ??__F?_Iostream_object@?$_Error_objects@H@std@@2V_Iostream_error_category@2@A@@YAXXZ 100078d0 f   CudaSupportPlugin.obj
 0001:000068e0       ??__F?_System_object@?$_Error_objects@H@std@@2V_System_error_category@2@A@@YAXXZ 100078e0 f   CudaSupportPlugin.obj
 0001:000068f0       ??__FalgoLog@U2@@YAXXZ     100078f0 f   CudaSupportPlugin.obj
 0001:00006900       ??__FcmdLog@U2@@YAXXZ      10007900 f   CudaSupportPlugin.obj
 0001:00006910       ??__FcoreLog@U2@@YAXXZ     10007910 f   CudaSupportPlugin.obj
 0001:00006920       ??__FioLog@U2@@YAXXZ       10007920 f   CudaSupportPlugin.obj
 0001:00006930       ??__FperfLog@U2@@YAXXZ     10007930 f   CudaSupportPlugin.obj
 0001:00006940       ??__FscriptLog@U2@@YAXXZ   10007940 f   CudaSupportPlugin.obj
 0001:00006950       ??__FtaskLog@U2@@YAXXZ     10007950 f   CudaSupportPlugin.obj
 0001:00006960       ??__FuiLog@U2@@YAXXZ       10007960 f   CudaSupportPlugin.obj
 0001:00006970       ??__FuserActLog@U2@@YAXXZ  10007970 f   CudaSupportPlugin.obj
 0001:00006980       ??__F?_Generic_object@?$_Error_objects@H@std@@2V_Generic_error_category@2@A@@YAXXZ 10007980 f   CudaSupportSettingsController.obj
 0001:00006990       ??__F?_Iostream_object@?$_Error_objects@H@std@@2V_Iostream_error_category@2@A@@YAXXZ 10007990 f   CudaSupportSettingsController.obj
 0001:000069a0       ??__F?_System_object@?$_Error_objects@H@std@@2V_System_error_category@2@A@@YAXXZ 100079a0 f   CudaSupportSettingsController.obj
 0001:000069b0       ??__F?helpPageId@CudaSupportSettingsPageController@U2@@0VQString@@B@@YAXXZ 100079b0 f   CudaSupportSettingsController.obj
 0001:000069c0       ??__FalgoLog@U2@@YAXXZ     100079c0 f   CudaSupportSettingsController.obj
 0001:000069d0       ??__FcmdLog@U2@@YAXXZ      100079d0 f   CudaSupportSettingsController.obj
 0001:000069e0       ??__FcoreLog@U2@@YAXXZ     100079e0 f   CudaSupportSettingsController.obj
 0001:000069f0       ??__FioLog@U2@@YAXXZ       100079f0 f   CudaSupportSettingsController.obj
 0001:00006a00       ??__FperfLog@U2@@YAXXZ     10007a00 f   CudaSupportSettingsController.obj
 0001:00006a10       ??__FscriptLog@U2@@YAXXZ   10007a10 f   CudaSupportSettingsController.obj
 0001:00006a20       ??__FtaskLog@U2@@YAXXZ     10007a20 f   CudaSupportSettingsController.obj
 0001:00006a30       ??__FuiLog@U2@@YAXXZ       10007a30 f   CudaSupportSettingsController.obj
 0001:00006a40       ??__FuserActLog@U2@@YAXXZ  10007a40 f   CudaSupportSettingsController.obj
 0001:00006a50       ??__F?_Generic_object@?$_Error_objects@H@std@@2V_Generic_error_category@2@A@@YAXXZ 10007a50 f   moc_CudaSupportPlugin.obj
 0001:00006a60       ??__F?_Iostream_object@?$_Error_objects@H@std@@2V_Iostream_error_category@2@A@@YAXXZ 10007a60 f   moc_CudaSupportPlugin.obj
 0001:00006a70       ??__F?_System_object@?$_Error_objects@H@std@@2V_System_error_category@2@A@@YAXXZ 10007a70 f   moc_CudaSupportPlugin.obj
 0001:00006a80       ??__F?_Generic_object@?$_Error_objects@H@std@@2V_Generic_error_category@2@A@@YAXXZ 10007a80 f   moc_CudaSupportSettingsController.obj
 0001:00006a90       ??__F?_Iostream_object@?$_Error_objects@H@std@@2V_Iostream_error_category@2@A@@YAXXZ 10007a90 f   moc_CudaSupportSettingsController.obj
 0001:00006aa0       ??__F?_System_object@?$_Error_objects@H@std@@2V_System_error_category@2@A@@YAXXZ 10007aa0 f   moc_CudaSupportSettingsController.obj
 0002:00000420       _algoLog$initializer$      10008420     CudaSupportPlugin.obj
 0002:00000424       _cmdLog$initializer$       10008424     CudaSupportPlugin.obj
 0002:00000428       _coreLog$initializer$      10008428     CudaSupportPlugin.obj
 0002:0000042c       _ioLog$initializer$        1000842c     CudaSupportPlugin.obj
 0002:00000430       _perfLog$initializer$      10008430     CudaSupportPlugin.obj
 0002:00000434       _scriptLog$initializer$    10008434     CudaSupportPlugin.obj
 0002:00000438       _taskLog$initializer$      10008438     CudaSupportPlugin.obj
 0002:0000043c       _uiLog$initializer$        1000843c     CudaSupportPlugin.obj
 0002:00000440       _userActLog$initializer$   10008440     CudaSupportPlugin.obj
 0002:00000444       ?_Generic_object$initializer$@?$_Error_objects@H@std@@2P6AXXZA 10008444     CudaSupportPlugin.obj
 0002:00000448       ?_Iostream_object$initializer$@?$_Error_objects@H@std@@2P6AXXZA 10008448     CudaSupportPlugin.obj
 0002:0000044c       ?_System_object$initializer$@?$_Error_objects@H@std@@2P6AXXZA 1000844c     CudaSupportPlugin.obj
 0002:00000450       _algoLog$initializer$      10008450     CudaSupportSettingsController.obj
 0002:00000454       _cmdLog$initializer$       10008454     CudaSupportSettingsController.obj
 0002:00000458       _coreLog$initializer$      10008458     CudaSupportSettingsController.obj
 0002:0000045c       _ioLog$initializer$        1000845c     CudaSupportSettingsController.obj
 0002:00000460       _perfLog$initializer$      10008460     CudaSupportSettingsController.obj
 0002:00000464       _scriptLog$initializer$    10008464     CudaSupportSettingsController.obj
 0002:00000468       _taskLog$initializer$      10008468     CudaSupportSettingsController.obj
 0002:0000046c       _uiLog$initializer$        1000846c     CudaSupportSettingsController.obj
 0002:00000470       _userActLog$initializer$   10008470     CudaSupportSettingsController.obj
 0002:00000474       ?helpPageId$initializer$@CudaSupportSettingsPageController@U2@@0P6AXXZA 10008474     CudaSupportSettingsController.obj
 0002:00000478       ?staticMetaObject$initializer$@CudaSupportPlugin@U2@@2P6AXXZA 10008478     moc_CudaSupportPlugin.obj
 0002:0000047c       ?staticMetaObject$initializer$@CudaSupportSettingsPageController@U2@@2P6AXXZA 1000847c     moc_CudaSupportSettingsController.obj
 0002:00000480       ?staticMetaObject$initializer$@CudaSupportSettingsPageState@U2@@2P6AXXZA 10008480     moc_CudaSupportSettingsController.obj
 0002:00000484       ?staticMetaObject$initializer$@CudaSupportSettingsPageWidget@U2@@2P6AXXZA 10008484     moc_CudaSupportSettingsController.obj
 0002:00000490       _pcinit                    10008490     MSVCRT:crtdll.obj
 0002:00000494       _pinit                     10008494     MSVCRT:atonexit.obj
 0002:00000f1c       _qt_meta_stringdata_U2__CudaSupportPlugin 10008f1c     moc_CudaSupportPlugin.obj
 0002:00000f44       _qt_meta_data_U2__CudaSupportPlugin 10008f44     moc_CudaSupportPlugin.obj
 0002:00000f80       _qt_meta_stringdata_U2__CudaSupportSettingsPageController 10008f80     moc_CudaSupportSettingsController.obj
 0002:00000fb8       _qt_meta_data_U2__CudaSupportSettingsPageController 10008fb8     moc_CudaSupportSettingsController.obj
 0002:00000ff4       _qt_meta_stringdata_U2__CudaSupportSettingsPageState 10008ff4     moc_CudaSupportSettingsController.obj
 0002:00001028       _qt_meta_data_U2__CudaSupportSettingsPageState 10009028     moc_CudaSupportSettingsController.obj
 0002:00001064       _qt_meta_stringdata_U2__CudaSupportSettingsPageWidget 10009064     moc_CudaSupportSettingsController.obj
 0002:00001098       _qt_meta_data_U2__CudaSupportSettingsPageWidget 10009098     moc_CudaSupportSettingsController.obj
 0002:000010e4       _GS_ExceptionPointers      100090e4     MSVCRT:gs_report.obj
 0002:00001a98       __catchsym$?_Copy@?$basic_string@DU?$char_traits@D@std@@V?$allocator@D@2@@std@@QAEXII@Z$5 10009a98     CudaSupportPlugin.obj
 0002:00001aa8       __catchsym$?_Copy@?$basic_string@DU?$char_traits@D@std@@V?$allocator@D@2@@std@@QAEXII@Z$4 10009aa8     CudaSupportPlugin.obj
 0002:00001ab8       __unwindtable$?_Copy@?$basic_string@DU?$char_traits@D@std@@V?$allocator@D@2@@std@@QAEXII@Z 10009ab8     CudaSupportPlugin.obj
 0002:00001ad8       __ehfuncinfo$?_Copy@?$basic_string@DU?$char_traits@D@std@@V?$allocator@D@2@@std@@QAEXII@Z 10009ad8     CudaSupportPlugin.obj
 0002:00001afc       __tryblocktable$?_Copy@?$basic_string@DU?$char_traits@D@std@@V?$allocator@D@2@@std@@QAEXII@Z 10009afc     CudaSupportPlugin.obj
 0002:00001b24       __unwindtable$??H@YA?BVQString@@ABV0@0@Z 10009b24     CudaSupportPlugin.obj
 0002:00001b2c       __ehfuncinfo$??H@YA?BVQString@@ABV0@0@Z 10009b2c     CudaSupportPlugin.obj
 0002:00001b50       __unwindtable$??H@YA?BVQString@@ABV0@PBD@Z 10009b50     CudaSupportPlugin.obj
 0002:00001b60       __ehfuncinfo$??H@YA?BVQString@@ABV0@PBD@Z 10009b60     CudaSupportPlugin.obj
 0002:00001b84       __unwindtable$??H@YA?BVQString@@PBDABV0@@Z 10009b84     CudaSupportPlugin.obj
 0002:00001b8c       __ehfuncinfo$??H@YA?BVQString@@PBDABV0@@Z 10009b8c     CudaSupportPlugin.obj
 0002:00001bb0       __unwindtable$??__EalgoLog@U2@@YAXXZ 10009bb0     CudaSupportPlugin.obj
 0002:00001bb8       __ehfuncinfo$??__EalgoLog@U2@@YAXXZ 10009bb8     CudaSupportPlugin.obj
 0002:00001bdc       __unwindtable$??__EcmdLog@U2@@YAXXZ 10009bdc     CudaSupportPlugin.obj
 0002:00001be4       __ehfuncinfo$??__EcmdLog@U2@@YAXXZ 10009be4     CudaSupportPlugin.obj
 0002:00001c08       __unwindtable$??__EcoreLog@U2@@YAXXZ 10009c08     CudaSupportPlugin.obj
 0002:00001c10       __ehfuncinfo$??__EcoreLog@U2@@YAXXZ 10009c10     CudaSupportPlugin.obj
 0002:00001c34       __unwindtable$??__EioLog@U2@@YAXXZ 10009c34     CudaSupportPlugin.obj
 0002:00001c3c       __ehfuncinfo$??__EioLog@U2@@YAXXZ 10009c3c     CudaSupportPlugin.obj
 0002:00001c60       __unwindtable$??__EperfLog@U2@@YAXXZ 10009c60     CudaSupportPlugin.obj
 0002:00001c68       __ehfuncinfo$??__EperfLog@U2@@YAXXZ 10009c68     CudaSupportPlugin.obj
 0002:00001c8c       __unwindtable$??__EscriptLog@U2@@YAXXZ 10009c8c     CudaSupportPlugin.obj
 0002:00001c94       __ehfuncinfo$??__EscriptLog@U2@@YAXXZ 10009c94     CudaSupportPlugin.obj
 0002:00001cb8       __unwindtable$??__EtaskLog@U2@@YAXXZ 10009cb8     CudaSupportPlugin.obj
 0002:00001cc0       __ehfuncinfo$??__EtaskLog@U2@@YAXXZ 10009cc0     CudaSupportPlugin.obj
 0002:00001ce4       __unwindtable$??__EuiLog@U2@@YAXXZ 10009ce4     CudaSupportPlugin.obj
 0002:00001cec       __ehfuncinfo$??__EuiLog@U2@@YAXXZ 10009cec     CudaSupportPlugin.obj
 0002:00001d10       __unwindtable$??__EuserActLog@U2@@YAXXZ 10009d10     CudaSupportPlugin.obj
 0002:00001d18       __ehfuncinfo$??__EuserActLog@U2@@YAXXZ 10009d18     CudaSupportPlugin.obj
 0002:00001d3c       __ehfuncinfo$??0CudaSupportPlugin@U2@@QAE@XZ 10009d3c     CudaSupportPlugin.obj
 0002:00001d60       __unwindtable$??0CudaSupportPlugin@U2@@QAE@XZ 10009d60     CudaSupportPlugin.obj
 0002:00001dd8       __ehfuncinfo$?obtainGpusInfo@CudaSupportPlugin@U2@@AAE?AW4Error@12@AAVQString@@@Z 10009dd8     CudaSupportPlugin.obj
 0002:00001dfc       __unwindtable$?obtainGpusInfo@CudaSupportPlugin@U2@@AAE?AW4Error@12@AAVQString@@@Z 10009dfc     CudaSupportPlugin.obj
 0002:00001f44       __ehfuncinfo$?loadGpusSettings@CudaSupportPlugin@U2@@AAEXXZ 10009f44     CudaSupportPlugin.obj
 0002:00001f68       __unwindtable$?loadGpusSettings@CudaSupportPlugin@U2@@AAEXXZ 10009f68     CudaSupportPlugin.obj
 0002:00001fb0       __unwindtable$?registerAvailableGpus@CudaSupportPlugin@U2@@AAEXXZ 10009fb0     CudaSupportPlugin.obj
 0002:00001fb8       __ehfuncinfo$?registerAvailableGpus@CudaSupportPlugin@U2@@AAEXXZ 10009fb8     CudaSupportPlugin.obj
 0002:00001fdc       __catchsym$??0?$QList@PAVCudaGpuModel@U2@@@@QAE@ABV0@@Z$2 10009fdc     CudaSupportPlugin.obj
 0002:00001fec       __unwindtable$??0?$QList@PAVCudaGpuModel@U2@@@@QAE@ABV0@@Z 10009fec     CudaSupportPlugin.obj
 0002:00001ffc       __tryblocktable$??0?$QList@PAVCudaGpuModel@U2@@@@QAE@ABV0@@Z 10009ffc     CudaSupportPlugin.obj
 0002:00002010       __ehfuncinfo$??0?$QList@PAVCudaGpuModel@U2@@@@QAE@ABV0@@Z 1000a010     CudaSupportPlugin.obj
 0002:00002034       __catchsym$?append@?$QList@PAVCudaGpuModel@U2@@@@QAEXABQAVCudaGpuModel@U2@@@Z$6 1000a034     CudaSupportPlugin.obj
 0002:00002044       __tryblocktable$?append@?$QList@PAVCudaGpuModel@U2@@@@QAEXABQAVCudaGpuModel@U2@@@Z 1000a044     CudaSupportPlugin.obj
 0002:00002058       __ehfuncinfo$?append@?$QList@PAVCudaGpuModel@U2@@@@QAEXABQAVCudaGpuModel@U2@@@Z 1000a058     CudaSupportPlugin.obj
 0002:0000207c       __unwindtable$?append@?$QList@PAVCudaGpuModel@U2@@@@QAEXABQAVCudaGpuModel@U2@@@Z 1000a07c     CudaSupportPlugin.obj
 0002:000020ac       __catchsym$?detach_helper_grow@?$QList@PAVCudaGpuModel@U2@@@@AAEPAUNode@1@HH@Z$5 1000a0ac     CudaSupportPlugin.obj
 0002:000020bc       __catchsym$?detach_helper_grow@?$QList@PAVCudaGpuModel@U2@@@@AAEPAUNode@1@HH@Z$4 1000a0bc     CudaSupportPlugin.obj
 0002:000020cc       __unwindtable$?detach_helper_grow@?$QList@PAVCudaGpuModel@U2@@@@AAEPAUNode@1@HH@Z 1000a0cc     CudaSupportPlugin.obj
 0002:000020ec       __ehfuncinfo$?detach_helper_grow@?$QList@PAVCudaGpuModel@U2@@@@AAEPAUNode@1@HH@Z 1000a0ec     CudaSupportPlugin.obj
 0002:00002110       __tryblocktable$?detach_helper_grow@?$QList@PAVCudaGpuModel@U2@@@@AAEPAUNode@1@HH@Z 1000a110     CudaSupportPlugin.obj
 0002:00002138       __unwindtable$??1CudaSupportPlugin@U2@@UAE@XZ 1000a138     CudaSupportPlugin.obj
 0002:00002140       __ehfuncinfo$??1CudaSupportPlugin@U2@@UAE@XZ 1000a140     CudaSupportPlugin.obj
 0002:00002164       __unwindtable$??_GCudaSupportPlugin@U2@@UAEPAXI@Z 1000a164     CudaSupportPlugin.obj
 0002:0000216c       __ehfuncinfo$??_GCudaSupportPlugin@U2@@UAEPAXI@Z 1000a16c     CudaSupportPlugin.obj
 0002:00002190       __unwindtable$??__EalgoLog@U2@@YAXXZ 1000a190     CudaSupportSettingsController.obj
 0002:00002198       __ehfuncinfo$??__EalgoLog@U2@@YAXXZ 1000a198     CudaSupportSettingsController.obj
 0002:000021bc       __unwindtable$??__EcmdLog@U2@@YAXXZ 1000a1bc     CudaSupportSettingsController.obj
 0002:000021c4       __ehfuncinfo$??__EcmdLog@U2@@YAXXZ 1000a1c4     CudaSupportSettingsController.obj
 0002:000021e8       __unwindtable$??__EcoreLog@U2@@YAXXZ 1000a1e8     CudaSupportSettingsController.obj
 0002:000021f0       __ehfuncinfo$??__EcoreLog@U2@@YAXXZ 1000a1f0     CudaSupportSettingsController.obj
 0002:00002214       __unwindtable$??__EioLog@U2@@YAXXZ 1000a214     CudaSupportSettingsController.obj
 0002:0000221c       __ehfuncinfo$??__EioLog@U2@@YAXXZ 1000a21c     CudaSupportSettingsController.obj
 0002:00002240       __unwindtable$??__EperfLog@U2@@YAXXZ 1000a240     CudaSupportSettingsController.obj
 0002:00002248       __ehfuncinfo$??__EperfLog@U2@@YAXXZ 1000a248     CudaSupportSettingsController.obj
 0002:0000226c       __unwindtable$??__EscriptLog@U2@@YAXXZ 1000a26c     CudaSupportSettingsController.obj
 0002:00002274       __ehfuncinfo$??__EscriptLog@U2@@YAXXZ 1000a274     CudaSupportSettingsController.obj
 0002:00002298       __unwindtable$??__EtaskLog@U2@@YAXXZ 1000a298     CudaSupportSettingsController.obj
 0002:000022a0       __ehfuncinfo$??__EtaskLog@U2@@YAXXZ 1000a2a0     CudaSupportSettingsController.obj
 0002:000022c4       __unwindtable$??__EuiLog@U2@@YAXXZ 1000a2c4     CudaSupportSettingsController.obj
 0002:000022cc       __ehfuncinfo$??__EuiLog@U2@@YAXXZ 1000a2cc     CudaSupportSettingsController.obj
 0002:000022f0       __unwindtable$??__EuserActLog@U2@@YAXXZ 1000a2f0     CudaSupportSettingsController.obj
 0002:000022f8       __ehfuncinfo$??__EuserActLog@U2@@YAXXZ 1000a2f8     CudaSupportSettingsController.obj
 0002:0000231c       __ehfuncinfo$??0CudaSupportSettingsPageController@U2@@QAE@ABVQString@@PAVQObject@@@Z 1000a31c     CudaSupportSettingsController.obj
 0002:00002340       __unwindtable$??0CudaSupportSettingsPageController@U2@@QAE@ABVQString@@PAVQObject@@@Z 1000a340     CudaSupportSettingsController.obj
 0002:00002368       __unwindtable$?getSavedState@CudaSupportSettingsPageController@U2@@UAEPAVAppSettingsGUIPageState@2@XZ 1000a368     CudaSupportSettingsController.obj
 0002:00002378       __ehfuncinfo$?getSavedState@CudaSupportSettingsPageController@U2@@UAEPAVAppSettingsGUIPageState@2@XZ 1000a378     CudaSupportSettingsController.obj
 0002:0000239c       __unwindtable$?saveState@CudaSupportSettingsPageController@U2@@UAEXPAVAppSettingsGUIPageState@2@@Z 1000a39c     CudaSupportSettingsController.obj
 0002:000023a4       __ehfuncinfo$?saveState@CudaSupportSettingsPageController@U2@@UAEXPAVAppSettingsGUIPageState@2@@Z 1000a3a4     CudaSupportSettingsController.obj
 0002:000023c8       __unwindtable$?createWidget@CudaSupportSettingsPageController@U2@@UAEPAVAppSettingsGUIPageWidget@2@PAVAppSettingsGUIPageState@2@@Z 1000a3c8     CudaSupportSettingsController.obj
 0002:000023d0       __ehfuncinfo$?createWidget@CudaSupportSettingsPageController@U2@@UAEPAVAppSettingsGUIPageWidget@2@PAVAppSettingsGUIPageState@2@@Z 1000a3d0     CudaSupportSettingsController.obj
 0002:000023f4       __unwindtable$??1CudaSupportSettingsPageController@U2@@UAE@XZ 1000a3f4     CudaSupportSettingsController.obj
 0002:000023fc       __ehfuncinfo$??1CudaSupportSettingsPageController@U2@@UAE@XZ 1000a3fc     CudaSupportSettingsController.obj
 0002:00002420       __unwindtable$??_GCudaSupportSettingsPageController@U2@@UAEPAXI@Z 1000a420     CudaSupportSettingsController.obj
 0002:00002428       __ehfuncinfo$??_GCudaSupportSettingsPageController@U2@@UAEPAXI@Z 1000a428     CudaSupportSettingsController.obj
 0002:0000244c       __unwindtable$??0CudaSupportSettingsPageState@U2@@QAE@H@Z 1000a44c     CudaSupportSettingsController.obj
 0002:0000245c       __ehfuncinfo$??0CudaSupportSettingsPageState@U2@@QAE@H@Z 1000a45c     CudaSupportSettingsController.obj
 0002:00002480       __catchsym$?reallocData@?$QVector@_N@@AAEXHHV?$QFlags@W4AllocationOption@QArrayData@@@@@Z$5 1000a480     CudaSupportSettingsController.obj
 0002:00002490       __catchsym$?reallocData@?$QVector@_N@@AAEXHHV?$QFlags@W4AllocationOption@QArrayData@@@@@Z$4 1000a490     CudaSupportSettingsController.obj
 0002:000024a0       __unwindtable$?reallocData@?$QVector@_N@@AAEXHHV?$QFlags@W4AllocationOption@QArrayData@@@@@Z 1000a4a0     CudaSupportSettingsController.obj
 0002:000024c0       __ehfuncinfo$?reallocData@?$QVector@_N@@AAEXHHV?$QFlags@W4AllocationOption@QArrayData@@@@@Z 1000a4c0     CudaSupportSettingsController.obj
 0002:000024e4       __tryblocktable$?reallocData@?$QVector@_N@@AAEXHHV?$QFlags@W4AllocationOption@QArrayData@@@@@Z 1000a4e4     CudaSupportSettingsController.obj
 0002:0000250c       __unwindtable$??1CudaSupportSettingsPageState@U2@@UAE@XZ 1000a50c     CudaSupportSettingsController.obj
 0002:00002514       __ehfuncinfo$??1CudaSupportSettingsPageState@U2@@UAE@XZ 1000a514     CudaSupportSettingsController.obj
 0002:00002538       __unwindtable$??_GCudaSupportSettingsPageState@U2@@UAEPAXI@Z 1000a538     CudaSupportSettingsController.obj
 0002:00002540       __ehfuncinfo$??_GCudaSupportSettingsPageState@U2@@UAEPAXI@Z 1000a540     CudaSupportSettingsController.obj
 0002:00002564       __ehfuncinfo$??0CudaSupportSettingsPageWidget@U2@@QAE@ABVQString@@PAVCudaSupportSettingsPageController@1@@Z 1000a564     CudaSupportSettingsController.obj
 0002:00002588       __unwindtable$??0CudaSupportSettingsPageWidget@U2@@QAE@ABVQString@@PAVCudaSupportSettingsPageController@1@@Z 1000a588     CudaSupportSettingsController.obj
 0002:00002650       __unwindtable$?getState@CudaSupportSettingsPageWidget@U2@@UBEPAVAppSettingsGUIPageState@2@AAVQString@@@Z 1000a650     CudaSupportSettingsController.obj
 0002:00002658       __ehfuncinfo$?getState@CudaSupportSettingsPageWidget@U2@@UBEPAVAppSettingsGUIPageState@2@AAVQString@@@Z 1000a658     CudaSupportSettingsController.obj
 0002:0000267c       __catchsym$?append@?$QList@PAVQCheckBox@@@@QAEXABQAVQCheckBox@@@Z$6 1000a67c     CudaSupportSettingsController.obj
 0002:0000268c       __tryblocktable$?append@?$QList@PAVQCheckBox@@@@QAEXABQAVQCheckBox@@@Z 1000a68c     CudaSupportSettingsController.obj
 0002:000026a0       __ehfuncinfo$?append@?$QList@PAVQCheckBox@@@@QAEXABQAVQCheckBox@@@Z 1000a6a0     CudaSupportSettingsController.obj
 0002:000026c4       __unwindtable$?append@?$QList@PAVQCheckBox@@@@QAEXABQAVQCheckBox@@@Z 1000a6c4     CudaSupportSettingsController.obj
 0002:000026f4       __catchsym$?detach_helper_grow@?$QList@PAVQCheckBox@@@@AAEPAUNode@1@HH@Z$5 1000a6f4     CudaSupportSettingsController.obj
 0002:00002704       __catchsym$?detach_helper_grow@?$QList@PAVQCheckBox@@@@AAEPAUNode@1@HH@Z$4 1000a704     CudaSupportSettingsController.obj
 0002:00002714       __unwindtable$?detach_helper_grow@?$QList@PAVQCheckBox@@@@AAEPAUNode@1@HH@Z 1000a714     CudaSupportSettingsController.obj
 0002:00002734       __ehfuncinfo$?detach_helper_grow@?$QList@PAVQCheckBox@@@@AAEPAUNode@1@HH@Z 1000a734     CudaSupportSettingsController.obj
 0002:00002758       __tryblocktable$?detach_helper_grow@?$QList@PAVQCheckBox@@@@AAEPAUNode@1@HH@Z 1000a758     CudaSupportSettingsController.obj
 0002:00002780       __unwindtable$??1CudaSupportSettingsPageWidget@U2@@UAE@XZ 1000a780     CudaSupportSettingsController.obj
 0002:00002790       __ehfuncinfo$??1CudaSupportSettingsPageWidget@U2@@UAE@XZ 1000a790     CudaSupportSettingsController.obj
 0002:000027b4       __unwindtable$??_GCudaSupportSettingsPageWidget@U2@@UAEPAXI@Z 1000a7b4     CudaSupportSettingsController.obj
 0002:000027c4       __ehfuncinfo$??_GCudaSupportSettingsPageWidget@U2@@UAEPAXI@Z 1000a7c4     CudaSupportSettingsController.obj
 0002:000027e8       __catchsym$?detach_helper@?$QList@PAVCudaGpuModel@U2@@@@AAEXH@Z$2 1000a7e8     CudaSupportSettingsController.obj
 0002:000027f8       __unwindtable$?detach_helper@?$QList@PAVCudaGpuModel@U2@@@@AAEXH@Z 1000a7f8     CudaSupportSettingsController.obj
 0002:00002808       __tryblocktable$?detach_helper@?$QList@PAVCudaGpuModel@U2@@@@AAEXH@Z 1000a808     CudaSupportSettingsController.obj
 0002:0000281c       __ehfuncinfo$?detach_helper@?$QList@PAVCudaGpuModel@U2@@@@AAEXH@Z 1000a81c     CudaSupportSettingsController.obj
 0002:00002840       __sehtable$__onexit        1000a840     MSVCRT:atonexit.obj
 0002:00002860       __sehtable$___DllMainCRTStartup 1000a860     MSVCRT:crtdll.obj
 0002:00002888       __sehtable$??_M@YGXPAXIHP6EX0@Z@Z 1000a888     MSVCRT:ehvecdtr.obj
 0002:000028a8       __sehtable$?__ArrayUnwind@@YGXPAXIHP6EX0@Z@Z 1000a8a8     MSVCRT:ehvecdtr.obj
 0002:000028c8       __sehtable$__IsNonwritableInCurrentImage 1000a8c8     MSVCRT:pesect.obj
 0002:000028f0       .edata                     1000a8f0     cuda_support.exp
 0002:00002918       rgpv                       1000a918     cuda_support.exp
 0002:0000291c       rgszName                   1000a91c     cuda_support.exp
 0002:00002920       rgwOrd                     1000a920     cuda_support.exp
 0002:00002922       szName                     1000a922     cuda_support.exp
 0002:00002933       $N00001                    1000a933     cuda_support.exp
 0002:000032da       .idata$6                   1000b2da     U2Core:U2Core.dll
 0002:000033d4       .idata$6                   1000b3d4     U2Algorithm:U2Algorithm.dll
 0002:00003742       .idata$6                   1000b742     U2Gui:U2Gui.dll
 0002:00004d30       .idata$6                   1000cd30     Qt5Widgets:Qt5Widgets.dll
 0002:0000546e       .idata$6                   1000d46e     Qt5Core:Qt5Core.dll
 0002:00005514       .idata$6                   1000d514     msvcprt:MSVCP120.dll
 0002:000055b4       .idata$6                   1000d5b4     MSVCRT:MSVCR120.dll
 0002:000057c8       .idata$6                   1000d7c8     kernel32:KERNEL32.dll
 0003:00000000       _RESOURCE_CUDA_GPU_NAME    1000e000     CudaSupportPlugin.obj
 0003:00000004       _cuinit_n                  1000e004     CudaSupportPlugin.obj
 0003:00000008       _cu_device_get_count_n     1000e008     CudaSupportPlugin.obj
 0003:0000000c       _cu_device_get_n           1000e00c     CudaSupportPlugin.obj
 0003:00000010       _cu_device_get_name_n      1000e010     CudaSupportPlugin.obj
 0003:00000014       _cu_device_total_mem_n     1000e014     CudaSupportPlugin.obj
 0003:00000018       _cu_device_get_properties_n 1000e018     CudaSupportPlugin.obj
 0003:00000028       _gpusDiscoveredText        1000e028     CudaSupportSettingsController.obj
 0003:0000002c       _noGpusDiscoveredText      1000e02c     CudaSupportSettingsController.obj
 0003:00000440       __Tuple_alloc              1000e440     CudaSupportPlugin.obj
 0003:00000441       _ignore                    1000e441     CudaSupportPlugin.obj
 0003:00000442       _allocator_arg             1000e442     CudaSupportPlugin.obj
 0003:00000443       _piecewise_construct       1000e443     CudaSupportPlugin.obj
 0003:00000444       _taskLog                   1000e444     CudaSupportPlugin.obj
 0003:0000044c       _algoLog                   1000e44c     CudaSupportPlugin.obj
 0003:00000454       _userActLog                1000e454     CudaSupportPlugin.obj
 0003:0000045c       _ioLog                     1000e45c     CudaSupportPlugin.obj
 0003:00000464       _coreLog                   1000e464     CudaSupportPlugin.obj
 0003:0000046c       _uiLog                     1000e46c     CudaSupportPlugin.obj
 0003:00000474       _scriptLog                 1000e474     CudaSupportPlugin.obj
 0003:0000047c       _perfLog                   1000e47c     CudaSupportPlugin.obj
 0003:00000484       _cmdLog                    1000e484     CudaSupportPlugin.obj
 0003:00000494       __Tuple_alloc              1000e494     CudaSupportSettingsController.obj
 0003:00000495       _ignore                    1000e495     CudaSupportSettingsController.obj
 0003:00000496       _allocator_arg             1000e496     CudaSupportSettingsController.obj
 0003:00000497       _piecewise_construct       1000e497     CudaSupportSettingsController.obj
 0003:00000498       _taskLog                   1000e498     CudaSupportSettingsController.obj
 0003:000004a0       _algoLog                   1000e4a0     CudaSupportSettingsController.obj
 0003:000004a8       _userActLog                1000e4a8     CudaSupportSettingsController.obj
 0003:000004b0       _ioLog                     1000e4b0     CudaSupportSettingsController.obj
 0003:000004b8       _coreLog                   1000e4b8     CudaSupportSettingsController.obj
 0003:000004c0       _uiLog                     1000e4c0     CudaSupportSettingsController.obj
 0003:000004c8       _scriptLog                 1000e4c8     CudaSupportSettingsController.obj
 0003:000004d4       _perfLog                   1000e4d4     CudaSupportSettingsController.obj
 0003:000004dc       _cmdLog                    1000e4dc     CudaSupportSettingsController.obj
 0003:000004e4       __Tuple_alloc              1000e4e4     moc_CudaSupportPlugin.obj
 0003:000004e5       _ignore                    1000e4e5     moc_CudaSupportPlugin.obj
 0003:000004e6       _allocator_arg             1000e4e6     moc_CudaSupportPlugin.obj
 0003:000004e7       _piecewise_construct       1000e4e7     moc_CudaSupportPlugin.obj
 0003:000004e8       __Tuple_alloc              1000e4e8     moc_CudaSupportSettingsController.obj
 0003:000004e9       _ignore                    1000e4e9     moc_CudaSupportSettingsController.obj
 0003:000004ea       _allocator_arg             1000e4ea     moc_CudaSupportSettingsController.obj
 0003:000004eb       _piecewise_construct       1000e4eb     moc_CudaSupportSettingsController.obj
 0003:000004ec       ___proc_attached           1000e4ec     MSVCRT:crtdll.obj
 0003:000004f0       _GS_ExceptionRecord        1000e4f0     MSVCRT:gs_report.obj
 0003:00000540       _GS_ContextRecord          1000e540     MSVCRT:gs_report.obj
 0003:0000080c       _DebuggerWasPresent        1000e80c     MSVCRT:gs_report.obj
 0004:00000060       $R000000                   1000f060     * linker generated manifest res *

 Exports

  ordinal    name

        1    _ugene_plugin_init
               exported name: ugene_plugin_init
